:020000040800F2
:1000000000000110393107087D2B0008297602080D
:10001000D9310708D9310708D93107080000000095
:100020000000000000000000000000000D4A000871
:10003000114A000800000000154A0008D50901080F
:10004000D9310708D9310708D9310708D93107084C
:10005000D9310708D9310708F5CB0008F9CB0008DA
:10006000D9310708FDCB000801CC00089532000803
:10007000A9320008BD320008D1320008E53200087C
:10008000F93200080D330008D9310708D9310708C3
:10009000D9310708D9310708D931070805CC00083C
:1000A0004131000869310008913100082D31000804
:1000B000B9310008CD310008E1310008D931070815
:1000C000D9310708D9310708D9310708D9310708CC
:1000D000D9310708E52C0008F12C0008D9310708B0
:1000E00009CC0008D9310708194A00081D32000858
:1000F000453200086D32000809320008213300083B
:10010000D931070861370008F5310008D9310708EF
:10011000FD2C0008D9310708D9310708D931070863
:1001200035330008493300085D3300087133000897
:1001300085330008D9310708D9310708D9310708B4
:10014000D9310708D9310708D93107086D4A0008A5
:1001500099330008AD330008C1330008092D0008A9
:10016000D9310708D9310708D9310708D93107082B
:10017000D9310708D9310708D9310708D93107081B
:08018000D9310708D931070845
:10019000D0E907239A422FBFD01AC0688018C01A2E
:1001A000704700BFD0E9092300699A4238BF12188E
:1001B000D31A0138C01A7047D0E90902101AB0FAF0
:1001C00080F04009704700BF0246036A4069D16869
:1001D000C05C01338B4228BF00231362704700BF0D
:1001E000436A8269D154436A0169426B01338B428D
:1001F00028BF00234362D36843F08003D360704775
:10020000436B188810F0100002D01A889B880120D8
:10021000704700BF436B99891A88890610B5044658
:100220000AD592B2900607D5E26A002A29D09888AA
:10023000216B80B29047636B99891A88090692B244
:100240000FD510060DD5D4E909128A4214D0A16940
:100250002069895C99800132B2FBF0F100FB112228
:10026000A262998A1A88C90592B204D5D20744BFFE
:100270004FF6F7721A8010BDDA6822F08002DA6059
:10028000EFE79B88E2696169DBB28B54E269E16860
:10029000636B0132B2FBF1F001FB1022E261CBE7AC
:1002A000036942681F2B10B40AD95468A3F1200CCB
:1002B000202101FA0CF1214207D15DF8044B70476F
:1002C0001468202199402142F7D081690024C86830
:1002D0000C7480684C68016821F00101016020689D
:1002E00094F805C00C4C818934F81C4089B221EA8D
:1002F00004011F2B818107D9A3F1200120238B400A
:100300005DF8044BD3607047202101FA03F35DF8D8
:10031000044B9360704700BFF4AC07084B1C10B44B
:1003200008BF4FF0800C4D4C18BF4FF0450C4FF4F8
:10033000003300E003B3626B12EA0C0F03F1FF33EA
:10034000F8D0002923DD626B52071CD403291ED08C
:10035000424A536B13F0010320D1022908D01369DC
:10036000DBB283421ED1012953692AD006291BD052
:1003700000205DF8044B7047002904DD636B5C07C7
:1003800001D40329E4D103205DF8044B7047002B0E
:1003900014BF002003205DF8044B704701205DF876
:1003A000044B70471020EFE713F4604F04BF2C4A52
:1003B0001360990431D45A04F4D41B04D8D50F2007
:1003C000E2E7284818400028DED0002B29DB5C003B
:1003D00025D4980029D4D90025D41A0129D45C0148
:1003E00025D4D8012FD41902E9D45A02DAD49C02B8
:1003F00027D4D8022FD419030FD45A0329D49C032D
:1004000025D4D80321D4190419D45A0415D49C0432
:1004100011D41807ACD51A20B6E71320B4E7092089
:10042000B2E71C20B0E70B20AEE70A20ACE70D20B6
:10043000AAE70C20A8E71920A6E71820A4E71720B0
:10044000A2E71120A0E70E209EE716209CE71520CA
:100450009AE7142098E7122096E700BF002C01408D
:10046000F01D002008E0FFFDF8B5154DEB6A93B1D3
:10047000696B0129044614D0124BDA6A22F0080293
:10048000DA6240F2FF5100229963EA62236823F0A6
:1004900001032360F8BD0B4AD36B43F48073D3632D
:1004A000F8BD084E40F2FF570023B763B36040F237
:1004B0004C43F3600C20FFF731FFB763DCE700BF6C
:1004C000F01D0020002C0140B34BD3E9011270B5A0
:1004D0008C0F83F83840C1F3836483F83940C1F34B
:1004E000016483F83A40100EC1F3074483F83B409F
:1004F0000001C1F30724C9B283F83C4083F83D10E2
:10050000D887D98FC2F3035089B20143C2F30344A1
:10051000D987C2F3C03083F84040C2F34031C2F300
:10052000803483F8410083F8424083F84310C2F3DB
:10053000003183F8441093F8901000200129C2F391
:10054000072C83F8450040F2D880022900F0B180E2
:10055000D9682A204FEA4C0C0CF07E0C83F85140ED
:1005600083F852C093F85240C1F3C01214431A6981
:1005700083F8524001F07F01D40F83F8531083F8C1
:100580005440910DC2F3417483F8554001F00C01C1
:10059000C2F3826483F8564083F8571093F85710DB
:1005A000C2F381542143C2F3405583F8571083F8B6
:1005B0005850002583F85950C2F3004583F85A502B
:1005C000C2F3C03583F85B50C2F3803583F85C50CA
:1005D000C2F3403583F85D505C69C2F3003583F89F
:1005E0005E50C2F3812583F85F50C4F30741C2F324
:1005F0000125C2F3460283F860504FF0010C83F8E6
:1006000061200902220E83F862C083F86420A3F8F7
:100610006610B3F86610C4F3072289B211432406AA
:10062000A3F8661099699C669A6E0C0E42EA044221
:100630009A669C6E0A0A02F47F4222439A669D6E75
:10064000DA69C1F307242C43C9B29C6683F86C10A5
:10065000110E83F86D10110C090619671C6F110239
:1006600001F47F0121431967196F120292B20A4304
:100670001A67196F1A6A41EA1261196793F87410C0
:10068000C2F30354214383F87410110A01F470611A
:10069000A3F87610B3F87610C2F3072489B2214389
:1006A000C2F34602A3F8761083F8782083F879C065
:1006B00070BD120402F47C129A64D9689A6C0C0E14
:1006C00042EA04229A649C6CC1F3074222439A6472
:1006D0009A6C013240F10004A40244EA925492025E
:1006E000C3F880204FF40072C3F88440C1F3072C94
:1006F000C3F88820C1F380342CE74FEA8C2C0CF42B
:1007000040619964996C920002F47F720A439A6482
:100710009C6CD96844EA91749C64C1F3C265C1F3CE
:10072000026483F84C50CA0B83F84D40C1F3425425
:1007300083F84E4002F00602C1F3824483F84F4032
:1007400083F8502093F85020C1F3C034224383F83B
:1007500050209D6C93F8502093F8404002F1020E17
:10076000012202FA04F602FA0EF24FEAE27EA2FB3E
:10077000062406FB0E4405F1010EA2FB0E2E05FB1E
:1007800004447444C3E92024C1F3072CC3F88860EF
:10079000C1F38034DEE600BFF01D00202F4B1A6845
:1007A000910102D59A6D52074BD42C4B1A68500216
:1007B00002D5DA6E11063CD4284B1A68D20102D554
:1007C0009A6D90072DD4254B1A68510102D59A6D68
:1007D000120717D4214B1A68120112D59A6DD00650
:1007E0000FD59A6D510334D49A6DD20503D49A6D06
:1007F00022F010029A65194B19484FF000629A6076
:1008000032E670479A6D500307D49A6DD10503D430
:100810009A6D22F008029A65104B4FF080629A6040
:10082000D8E79A6D4FF0807122F002029A659960C4
:10083000C9E7DA6E4FF4800122F08002DA6699602F
:10084000BAE79A6D4FF0007122F004029A65996040
:10085000ABE74FF000629A60704700BF006402404F
:1008600058640240384B5A68110303D5D3F8A020CE
:1008700052075BD4344B5A68D00303D5D3F8B42065
:10088000110649D4304B5A68520303D5D3F8A0203F
:10089000900737D42C4B5A68D10203D5D3F8A02047
:1008A00012071CD4284B5A68920217D5D3F8A020FF
:1008B000D00613D5D3F8A020510341D4D3F8A020FB
:1008C000D20505D4D3F8A02022F01002C3F8A0204E
:1008D0001D4B1E484FF40012DA60C5E57047D3F88F
:1008E000A02050030AD4D3F8A020D10505D4D3F812
:1008F000A02022F00802C3F8A020134B4FF480126E
:10090000DA60CFE7D3F8A0204FF4802122F0020272
:10091000C3F8A020D960BDE7D3F8B4204FF48031EC
:1009200022F08002C3F8B420D960ABE7D3F8A0204E
:100930004FF4002122F00402C3F8A020D96099E707
:100940004FF40012DA60704700640240A064024075
:1009500082B00922274B8DF80720DA68D00319D41A
:10096000DA68D10640D4DA68D20541D4DA6812F0E8
:10097000E00F3BD1DB6813F0020F14BF08230923FB
:100980008DF807309DF80730012B0AD09DF807003D
:1009900002B0704701238DF807309DF80730012B16
:1009A000F4D1144A12E0D368DB0519D4D36813F0EC
:1009B000E00F17D1D36813F0020F14BF08230923E7
:1009C0008DF807309DF80730012BDFD1D168C803BF
:1009D0004FF00103F4D4D368D906E4D50623EFE73A
:1009E0000223EDE70723EBE70623D4E70723D2E74B
:1009F0000223D0E7003C0240704700BF704700BFB1
:100A000001207047034BD3E92503C01AC0F30A0045
:100A1000704700BFF01D0020064AD2E925138B4223
:100A2000FDD0D1180133C3F30A0391F89C00C2F83A
:100A300098307047F01D0020064BD3F89C0800B991
:100A40007047D3F89C08A0F10500B0FA80F0400987
:100A5000704700BFF01D0020012380F84930704727
:100A6000044BD3E92503C01AC0F30A00C0F50060A7
:100A7000704700BFF01D002010B5D0F8E8350446DF
:100A80001B699847032384F81231002010BD00BF72
:100A900008B5042290F81211D0F8E83580F8131147
:100AA00080F81221DB689847002008BD08B5D0F80F
:100AB000E435DB6903B19847002008BD08B5D0F8DC
:100AC000E4351B6A9847002008BD00BF08B5D0F880
:100AD000E4355B6A9847002008BD00BF037830B456
:100AE00003B30446C0F1010C04EB0C0314F8015FDE
:100AF000DBB2002DF8D101335B00DCB2138003239D
:100B00000C704B7004785CB1022300255A1CD2B2E1
:100B1000CC548D5410F8014F0233DBB2002CF5D1C8
:100B200030BC704702242346E8E700BF10B5074CED
:100B30002068FF2808D00649D1F8A02801F6A401B2
:100B400000F080F8FF232360002010BD000000208B
:100B5000F01D0020432301480B8070470400002053
:100B6000122301480B8070474800002004230148ED
:100B70000B8070475C00002008B5044B04480A460F
:100B80001946FFF7ABFF084608BD00BF9C260020B2
:100B9000384E080808B5044B04480A461946FFF7C2
:100BA0009DFF084608BD00BF9C2600204C4E08084B
:100BB00008B5044B04480A461946FFF78FFF08465C
:100BC00008BD00BF9C260020544E080808B5044B01
:100BD00004480A461946FFF781FF084608BD00BFD2
:100BE0009C260020604E080808B5044B04480A46BD
:100BF0001946FFF773FF084608BD00BF9C2600207A
:100C00006C4E0808704700BF704700BF704700BFB8
:100C1000704700BF704700BF704700BF044B002003
:100C20000522C3F89C28C3F8AC09C3F8B009704783
:100C3000F01D0020024B0020C3F89C08704700BF45
:100C4000F01D0020212838B50C4605D022282DD0D3
:100C5000202813D0002038BD0029FBD0072AF9D165
:100C6000194BD3F8B40993F8B81993F8B92993F844
:100C7000BA39206021716271A371EBE70029E9D0D4
:100C8000072AE7D1104DD5F8B03913B10968002013
:100C90009847206821796279A379C5F8B40985F865
:100CA000B81985F8B92985F8BA39D3E70029D1D020
:100CB000022ACFD1044BD3F8AC39002BCAD0098813
:100CC00000209847C6E700BFF01D002010B4124C6A
:100CD000D4E925329A1AC2F30A020A44B2F5006F27
:100CE00014D8B9B101444A1E013810F801CFE118F7
:100CF000824203F1010381F89CC0C3F30A03F4D1DB
:100D0000C4F8943000205DF8044B704702205DF871
:100D1000044B70470846F6E7F01D0020034B93F89C
:100D2000E009003818BF0120704700BFF01D002007
:100D300070B5124D124C296840F2FF5640F24D43F7
:100D40000022A6630D20A160C5F8DC290121E36023
:100D5000FFF7E4FAA66320B96369C3F34323042BC6
:100D600008D0D5F8143AC5F8D039092285F8E02919
:100D7000002070BD85F8E039022070BDF01D002014
:100D8000002C014070B50F4D95F8E039042B044656
:100D90000E460BD0082B07D1D5F8D83983420ED098
:100DA000FFF7C6FF022801D0012070BD082385F897
:100DB000E039C5F8DC69C5F8D849022070BD0220C9
:100DC00070BD00BFF01D0020034B93F8E00903281D
:100DD00094BF002001207047F01D0020004870479C
:100DE000D427002030B4194B00209C7B14B11D681F
:100DF0008D4206D00130082803F11003F5D130BC34
:100E000070479AB1124B03EB40218A4219D0114B23
:100E100093F8B4218AB1104B01225A7000F5817009
:100E200003EB00100123837130BC70470A4B00F5BF
:100E3000817003EB00108271E1E7012283F8B42195
:100E4000E9E7022CE3D1183BE8E700BFD45A0020C1
:100E5000D44A0020BC5A0020BC4A002030B41D4CAB
:100E6000002384F8A03004F1180004E00133082BBB
:100E700000F110001ED005688D42F7D190F80EC029
:100E8000BCF1030FF2D1BAB1134901EB4320824206
:100E900009D094F8B42112B9012284F8B4210F4981
:100EA00001224A7000E0183903F5817301EB031346
:100EB00001229A7130BC70470849D4F89C2003F590
:100EC000817301EB0313013204219971C4F89C2052
:100ED000F0E700BFBC5A0020D44A0020BC4A0020E2
:100EE000A8B183681BB10E4B07229A7070470C4A59
:100EF0001178D36003294FF004000CBF80214FF418
:100F00008071C2E901111361137590707047044A32
:100F100002F580510123537081F8B431704700BF4E
:100F2000BC4A002010B58121044670F047FA2046E3
:100F3000012170F043FA2046822170F03FFAFFF75A
:100F400079FE002010BD00BFC169026910B4002302
:100F500040F20114A0F844410B60D169846D21F086
:100F600002014FF0010CD161A0F89CC32360D1694C
:100F7000044821F4003180F8183A5DF8044BD1613F
:100F800018467047F01D0020202301480B80704751
:100F900060000020122301480B8070478000002071
:100FA000042301480B807047940000200A4608B5CE
:100FB000054920B90548FFF791FD034808BD0448DD
:100FC000FFF78CFD004808BD0C2800207C4E080867
:100FD000944E080808B5044B04480A461946FFF722
:100FE0007DFD084608BD00BF0C280020AC4E080857
:100FF0002048D0F8E837D0F8EC2730B59B184FF0F0
:101000001A040C8001D11C4830BD1B4AD0F8EA17E5
:101010004FF0000E10467546B3F1204F4FEA137C97
:101020000CF130040EF1020E2ABF0CF1370C847063
:1010300080F802C0BEF1100FC5704FEA031300F133
:101040000200E9D100200446B1F1204F4FEA1173AC
:1010500003F1300C00F102002ABF373382F812C0CE
:1010600093740828D4744FEA011102F10202EBD103
:10107000014830BD00F0FF1F9800002008B5044B68
:1010800004480A461946FFF729FD084608BD00BF77
:101090000C280020C04E080808B5044B04480A4636
:1010A0001946FFF71BFD084608BD00BF0C280020AD
:1010B000CC4E080810B50F4C0F4BD4F8F41BB4F805
:1010C000F80B088303F1B402C4F8682DD3F8B430E8
:1010D000984702E01B69984720B9D4F8683D002B77
:1010E000F8D1FEE7D4F8F43BB4F8F82B5A8300208B
:1010F00010BD00BFF01D00200000002038B5084BD7
:10110000D3F8683D53B1DB6914460D4698474FF458
:10111000007302682A600020236038BD1B68FFDE70
:10112000F01D002008B5074BD3F8683D33B11B69AB
:10113000984780F00100404240B208BD4FF0FF30B8
:1011400008BD00BFF01D0020002070472DE9F041D0
:10115000164CD4F8B80B1646B4F8BC2B428303B334
:101160000F4603EB060806E000234D681A46394691
:101170003046A84738B9D4F8681D0029F4D1FEE7F5
:101180001B69984720B9D4F8683D002BF8D1FEE7D9
:101190000136B04507F50077EDD1D4F8B80BB4F8B7
:1011A000BC2B02830020BDE8F08100BFF01D0020B1
:1011B0002DE9F041184CD4F8B80B1646B4F8BC2B06
:1011C00042832BB30F4603EB060801E00B699847F7
:1011D000D4F8681D51B10023CD681A46394630460F
:1011E000A847D4F8681D08B10029EFD131B10B69C7
:1011F000984720B9D4F8681D0029F8D1FEE70136D8
:10120000B04507F50077E3D1D4F8B80BB4F8BC2BA0
:1012100002830020BDE8F081F01D0020A64A53683B
:1012200023F4FD4323F07F032DE9F04143F07603DF
:1012300053605368032123F48073536082B01160BC
:101240000FF014FC04460D460FF010FC031B61EB7D
:101250000502B3F57A7F72F10003F5D30FF006FCB7
:1012600004460D460FF002FC031B61EB0502B3F5CB
:101270007A7F72F10003F5D38F4C636840F2FF5020
:1012800043F4807300214FF480626360A0634FF4E5
:101290000033A160E26001E0002B6DD0626B1606A6
:1012A00003F1FF33F8D5002B66D040F2FF554FF421
:1012B000D5724FF48963A5630721A5630820A26056
:1012C000E360FFF72BF8A56300284ED000277A4C87
:1012D00040F2FF55002240F27743A5630121A2604E
:1012E0003720E360FFF71AF8A563002839D147F0EB
:1012F00000470646804647F4801701E0964230D00A
:1013000040F27743A5630121C4F808803720E360E9
:10131000FFF704F8034640F2694203212920013611
:10132000A563F3B9A563A760E260FEF7F7FF4FF688
:10133000FF72A563A8B96369002BDFDA4FF6FF726D
:1013400096420ED05D0000F1BF8023689B0708D055
:101350005A4D95F89000042840F0BE80FFF7B4F88D
:1013600090B1012002B0BDE8F081544B012283F816
:1013700090204FF08047AAE74F4B40F2FF520120E8
:101380009A6302B0BDE8F0814B4C2A6840F24743B3
:1013900040F2FF56A6630121A2600720E360FEF73A
:1013A000BDFFA663636823F4FD4323F07F036360FE
:1013B0000028D6D195F89030022BD2D8636913F06B
:1013C0000073CED1CDE9003308274FF48A63A663BA
:1013D0000121A7601020E360FEF7A0FFA6630028AC
:1013E000BFD12B68A663A36040F27743E36001217D
:1013F0003720FEF793FFA6630028B2D1304B63621B
:10140000A762E36A43F03303E36240F27343A663E7
:101410000121A060E3603320FEF780FFA66300286F
:101420009FD16B4640F22A4206E0616B880244BFBE
:10143000D4F8801043F8041B616B1142F5D0636B44
:1014400019078ED4636B9A078BD4636B9B0688D481
:10145000636B9F0285D4009B1BBA5E0381D52A680B
:1014600040F2774340F2FF55A5630121A260372087
:10147000E360FEF753FFA56300287FF472AF0222FA
:1014800040F24643A5630121A2600620E360FEF717
:1014900045FFA56300287FF464AF63681C0509D489
:1014A000054A084953680B4043F40063536053688E
:1014B0001805F7D5002055E7002C0140F01D00204D
:1014C00000E1F5050081FFFF314D022085F8900015
:1014D00023689C073FF445AF2E49002340F2FF529A
:1014E0008A638B6040F2C243CB604FF4003301E06B
:1014F000013B03D04A6B12F0450FF9D0254B5A6BD4
:10150000520741D45A6B12F0010F40F2FF529A6316
:101510007FF427AF5A696A619A69AA61DA69EA6158
:101520001B6A2B6201282AD81A4C40F2FF5600226F
:1015300040F24343A6630621A2600320E360FEF766
:10154000EDFEA66300287FF40CAF124C2A6840F22F
:10155000FF5640F2C943A6630221A2600920E3605E
:10156000FEF7DCFEA66300287FF4FBAE63696B60C8
:10157000A369AB60E369EB60236A2B61EEE600F0E0
:10158000FB000228D0D0E0E740F2FF529A63E8E681
:10159000F01D0020002C014008B5FFF73FFE58B1B8
:1015A0000E4A92F8D4390133DBB2072B82F8D439D2
:1015B00003D9002382F8E03908BDD2F80C3A23B1F0
:1015C0001868998803691942F3D00123D2F8141AD4
:1015D00082F8E039C2F8D01908BD00BFF01D002024
:1015E000F8B59F4CD4F8100A002800F0328194F826
:1015F000E0099C4D40F2FF5640F24D47431E082B38
:1016000063D8DFE813F04D005000D9006200950068
:1016100074002500620009002368AE630121AB60FD
:101620000D20EF60FEF77AFEAE6328B96B69C3F355
:101630004323042B00F00881D4F8D039D4F8142ABD
:10164000FA3393423ED2FFF7A7FF94F8E009D5E7BB
:101650002368AE630121AB600D20EF60FEF75EFEF4
:10166000AE630028E8D16B69C3F34323042BE3D1B5
:10167000D4F8DC3984F8D409012B40F2ED80D4F899
:10168000D8290820013B0132C4F8DC39C4F8D82934
:1016900084F8E009A0F10800B0FA80F04009F8BD34
:1016A000022384F8E0392368AE630121AB600D208A
:1016B000EF60FEF733FEAE6320B96B69C3F34323DB
:1016C000042B5AD094F8E009431EDBB2022B0AD84F
:1016D000D4F8143AD4F8D0299B1AC82BDAD9FFF7DA
:1016E0005BFF94F8E0090428D4D10120F8BD236BF6
:1016F000002BCFD1D4F8C859D4F8143AC4F8D03953
:10170000072084F8E009002DC4D0D4F8CC39D4F8EF
:10171000BC29D4F8C0190120A84794F8E009431E59
:10172000D3E7D4F8D039D4F8142A64339342B1D231
:10173000E36A002BF5D12368AE630121AB600D2075
:10174000EF60FEF7EBFDAE6300287FF47EAF6A69C1
:10175000C2F34322042A7FF478AFD4F8C85984F83E
:10176000E02984F8D409002DBFD0D4F8CC39D4F8BE
:10177000BC29D4F8C019A847A4E7FEF7A5FE0028A5
:10178000A0D194F89030002BA3F10203B3FA83F3B5
:1017900014BF022201225B0984F8D52984F8D639C6
:1017A000FEF792FE00287FF44EAFD4F88020C4F8F4
:1017B000E429032384F8E039FEF786FE002881D16E
:1017C00094F86420B4F86630A4F8E839A16EA36EEA
:1017D000C4F8DC09090E04201B0C84F8EA2984F8FB
:1017E000E009A26E84F8EB1984F8EC39A16E94F844
:1017F0006C0094F86D3084F8EE19120A1B0984F815
:10180000ED2984F8EF0994F86D2084F8F439216FFC
:10181000B4F87600B4F87630C4F8F01902F00F028C
:10182000C3F30B1384F8F52943EA1023B4F87620A8
:1018300003F00F0303F5FA6302F00F02A4F8F63980
:1018400084F8F8290120F8BD042384F8E039012048
:10185000F8BD84F8E009F8BDF6D1FFF769FA31E781
:10186000F01D0020002C01402DE9F0411E4E96F89D
:101870006C3D002BFBD199B3014400F1FF384F1EA2
:10188000D6F8703DD6F8742D0133C3F30A039A429B
:1018900016D10FF0EBF804460D460FF0E7F8031BE6
:1018A00061EB0501B3F57A7F71F10003F5D3D6F84A
:1018B000703DD6F8742D0133C3F30A039342E8D088
:1018C000D6F8702DD6F8703D18F8011F3244013358
:1018D000C3F30A03B84582F8781DC6F8703DCFD12E
:1018E0000020BDE8F08100BFF01D002090F84820E6
:1018F000531C0244DBB280F8483082F8341090F870
:1019000049200AB1132B03D9002280F8482003B9DB
:10191000704710B5084CD4F89C2802B910BDD4F813
:101920009C28052AFAD119463430D4F8143AFFF726
:101930009BFFD4F8143A10BDF01D002010B50A4CDE
:10194000D4F89C3803B910BDD4F89C38052BFAD1D3
:10195000002A0846D4F8143A1146F4DDFFF784FF54
:10196000D4F8143A10BD00BFF01D002090F84810C4
:101970000023A0F8483001B9704710B5084CD4F8DE
:101980009C381BB1D4F89C38052B00D010BD3430E6
:10199000D4F8143AFFF768FFD4F8143A10BD00BF2A
:1019A000F01D00202DE9F0475D4E1F4606EB800339
:1019B0009C68002C00F0AD8004F13E03A36104F5A7
:1019C0009F73E3614FF48073C4E9043328362368BE
:1019D00066600546E16094F83D00A36390460BF015
:1019E00015F9814694F8440294F83CA0261D00287D
:1019F0004FD194F8450268BBD4F8403283BB390715
:101A000034D418F0020F60D118F0010F44D194F9CA
:101A1000472294F84712D4F84832002A10DB414894
:101A20001B018418DBB284F800335209012301F052
:101A30001F0103FA01F140F822103046BDE8F0879B
:101A4000394A01F00F010A441B01DBB2137630461C
:101A5000BDE8F0876DF0F6FBD4F84032002BCED015
:101A6000324A116B0B4339071363CAD50135EDB206
:101A7000B9F1000FCBD040F20673FA0689F808508E
:101A8000A9F8063036D4BB0694F8462245D4322154
:101A900033E06DF0D7FBACE750460BF0B7F80135FB
:101AA000EDB20028B3D040F206620572C28094F80D
:101AB000462202210BF0AEFA94F9472294F847121D
:101AC000D4F84832002AAADABAE76B1CDBB2B9F1C3
:101AD000000F99D089F8083040F20653A9F8063073
:101AE00094F84622484602210BF094FA18F0010FB0
:101AF0008DD0D1E794F84622022148460BF08AFAAD
:101B000094F9472294F84712D4F84832002A86DA2A
:101B100096E726463046BDE8F0871221EDE700BF84
:101B2000F4AC070800E100E0FCEC00E00038024003
:101B30002DE9F047038A8489A4B21C4082B045D0C5
:101B4000814688464FF0004501F14C0701F134060B
:101B5000B4FA84F325FA03F2D24391B2A9F8101033
:101B600014401B3BB8F1000F5DD0042B2CD8DFE8EC
:101B700003F050463B300300D8F80C30D9F82CA0C5
:101B800033B19B6823B11FFA8AF108F1040098472A
:101B9000D8F8243033B19B6823B11FFA8AF108F1D9
:101BA0001C009847D8F83C302BB19B681BB11FFA3A
:101BB0008AF130469847D8F854302BB19B681BB156
:101BC0001FFA8AF138469847002CC1D102B0BDE80F
:101BD000F087D8F80C30D9F834105B6808F10400AD
:101BE0009847002CB4D1F1E7D8F82430D9F8381050
:101BF0005B6808F11C009847002CA9D1E6E7D8F8EB
:101C00003C30D9F83C105B6830469847002C9FD197
:101C1000DCE7D8F85430D9F840105B68384698476C
:101C2000002C95D1D2E7042B07D8DFE803F0031985
:101C3000140F0A00D9F840300193019B002C87D182
:101C4000C4E7D9F82C300193019BF7E7D9F8343079
:101C50000193019BF2E7D9F838300193019BEDE73E
:101C6000D9F83C300193019BE8E700BF70B5254CE3
:101C700094F86C2D012A034603D0022A09D00020D3
:101C800070BD214ED6F880548DB984F86C5D00206B
:101C900070BD002540F20112C0E95455C0E9565507
:101CA000A0F8442100F5A2716FF098FCEDE7402DFB
:101CB00022D823D0D4F8741D144AC3F858510A44CA
:101CC000C3E954220022C3F85C2140F2011203F55B
:101CD000A271A3F8442118466FF080FCD4F8743D3B
:101CE000D6F880242B44C3F30A03521BC4F8743D76
:101CF000C6F88024002070BD4025DBE7022284F86E
:101D00006C2DD7E7F01D0020E82E0020682B002066
:101D100001EB810138B500EBC1010E4DB1F88C1318
:101D200004462846FEF7D2FFE378C4F8A8534021C2
:101D30000022C4E9EC12012293422046A4F89C231D
:101D400004F5677108BFC4F8AC536FF047FC00207E
:101D500038BD00BF6C33002070B52B4CD4F8C434B0
:101D60000F2B04D05A1CC4F8C424002070BD274D8A
:101D700095F86C3D0022C4F8C424002BF5D1D5F8A9
:101D8000742DD5F8703D9A42EFD0D5F8742DD5F862
:101D9000703D9A422CD8D5F8706DD5F8743DF61A7E
:101DA000402EC4F8806428D9012385F86C3D402674
:101DB000D5F8742D164BC0F858611344C0E954335C
:101DC0000023C0F85C3140F20113A0F8443100F563
:101DD000A2716FF003FCD5F8743DD4F8802433442D
:101DE000C3F30A03921BC5F8743DC4F88024BCE712
:101DF000D5F8746DC6F50066D2E70CBF0223012347
:101E000085F86C3DD4E700BFE82E0020F01D0020CF
:101E1000682B002038B5224DD5F8D03495F8E8C4A9
:101E2000044623B195F8D4345CEA030331D001238E
:101E3000E06984F8463140F20112A4F844210268B6
:101E40001849002AA8BFC2F380739B0301EA12411C
:101E500043F020030B4363F31F42BCF1020F026007
:101E600000D038BDE278104BC4F8A8331F20002101
:101E7000C4E9EC01012A4FF00101A4F89C1308BF4A
:101E8000C4F8AC3304F567712046BDE838406FF004
:101E9000A5BB01216CF026FF95F8E8C4C7E700BF99
:101EA000E82E0020DFBFFFFFB033002070B590F8B0
:101EB000CF2590F8D13590F8CE5590F8D0C590F850
:101EC000CC1590F8CD6505EB02250CEB032C90F8B2
:101ED000D32590F8D23503EB0223012284B080F899
:101EE000112101F01F029BB2ADB21FFA8CFC012A36
:101EF00004468DF80810ADF80A50ADF80CC0ADF8E6
:101F00000E30C0F840318DF809600AD0022A57D04F
:101F1000002A3CD001F080016CF0E4FE002004B007
:101F200070BD90F81231032B2BD15FFA8CFCBCF101
:101F3000010F26D8D0F8E43502A99B689847BDF870
:101F40000E30002BEAD1C4E94A33C4E94C330421F2
:101F50004FF4807284F81111A4F81C2104F58E71DD
:101F600020466FF0CDFA636DC44A1A61E278012A07
:101F7000D4D104F2CC545C614FF0802219681A600D
:101F8000CCE720466CF076FE002004B070BD092E30
:101F9000F7D801A252F826F0432000085321000888
:101FA000831F00088D210008831F0008BB21000843
:101FB00067200008831F0008D120000801210008C5
:101FC00001F0600120295FFA8CF334D0012E00F07B
:101FD0006181032E00F09581002E9FD190F812218F
:101FE000022A00F01B81032ACBD11CF0800F40F0A5
:101FF000A48103EB830300EBC30393F87633002B38
:1020000000F0A6819E4B0122C3F8F8249D4A0223CA
:10201000C4E94E334FF48070002184F81131A4F8E4
:102020001C01C4E94C31C4E94A2204F58E712046F2
:102030006FF066FA72E7D0F8E43502A99B6898471A
:102040006CE790F81231023B012B9AD88C4BD0F8F8
:1020500018210021C3F8F01412B10222C3F8F024B1
:10206000894A0223D4E72E0A022EADF8063000F08A
:10207000CD81032E00F09181012E82D1D0F8EC3574
:1020800080781B680DF106019847BDF80630002BDB
:102090003FF444AFBDF80E20002A3FF43FAF934217
:1020A00028BF13464FF480720221A4F81C2100229D
:1020B000C4E94A0084F81111C4E94E33C4E94C3232
:1020C00004F58E712046ADF806306FF019FA25E759
:1020D000012B7FF456AF90F81221022A00F04981BB
:1020E000032A7FF44EAF4FF4807100F5887202200E
:1020F000A4F81C11C4E94E3384F81101002190E7C3
:10210000EDB25F4E012D86F8E9543FF63AAF90F8F4
:102110001231022B00F02181032B7FF432AF002D0E
:1021200000F07F8190F81011012910D0D0F8E4352B
:102130005B68984796F8E914D4F8E43584F81011F0
:102140001B6820469847D4F8E8359B6898470023D9
:10215000F9E690F81231023B012B3FF612AF012D48
:102160007FF4DCAED0F8E43500259B68C0F8185148
:1021700002A9984704224FF48073C4E94A55C4E980
:102180004C5584F81121A4F81C31E7E6012D00F02C
:10219000CC80022D7FF4C2AE5FFA8CF3002B7FF46B
:1021A000BDAE02694FEA1C23023B5268032B00F2CA
:1021B0005681DFE803F05B426B5F5CEA03037FF468
:1021C000E0AE90F81221032A3FF4DBAE016905F07E
:1021D0007F0680F8146108681A4665F30A12024304
:1021E0000A604FF480720421C4E94A33C4E94C33D5
:1021F00084F81111A4F81C2104F58E7120466FF0AB
:102200007FF9636D1D4A1A61E278012A0DD0002E14
:1022100000F01281022384F812317FE65A063FF45F
:102220007DAE19466CF05EFD78E604F2CC525A6140
:102230004FF0802219681A60E9E7032363F306125E
:1022400001210F4D84F816110421002384F8111187
:102250004FF48071A4F81C11C4E94A33C4E94C332B
:1022600004F58E712046C5F8F4247AE6022363F360
:102270000612E5E7052363F30612E1E7180008609C
:10228000E82E0020E0330020D8330020042363F33D
:102290000612D5E790F81221022ABFD0032A7FF454
:1022A00070AE002D7FF43AAE13F07F023FF44FAFD3
:1022B0001CF0800F40F0C48003EB830100EBC101F0
:1022C00081F8742381F8765381F87553282101FB36
:1022D000030300EB820293F87713506D03688A1EA4
:1022E000012A6FF35553D4F8E4258CBFC3F3007172
:1022F000012161F31C739268036002A92046904794
:1023000025E790F81221022A88D0032A7FF439AEFB
:1023100025B9590602D019466CF0E4FCD4F8E4352E
:1023200002A99B682046984711E7D0F8E43502A936
:102330009B68C0F81851984709E703F07F0303EB47
:10234000830300EBC30393F81E31002B7FF45AAED6
:10235000454B0022C3F8F82458E6002D3FF40AAF9D
:1023600001210322D0F8E43580F8101180F8122101
:10237000E6E63E4984F811214FF480700022C4E95A
:102380004A11A4F81C01C4E94E33C4E94C3204F5E7
:102390008E7120466FF0B4F8C0E5EDB2052D3FF622
:1023A000F0ADDFE805F02B231B130B03D0F8EC3561
:1023B00080789B690DF10601984766E6D0F8EC3508
:1023C00080785B690DF1060198475EE6D0F8EC3540
:1023D00080781B690DF10601984756E6D0F8EC3578
:1023E0008078DB680DF1060198474EE6D0F8EC35B1
:1023F00080789B680DF10601984746E6D0F8EC35E9
:1024000080785B680DF1060198473EE6D0F8E43528
:1024100080789B6A0DF1060198474670C4F8F00574
:1024200033E60222D0F8E43580F8122180F810510A
:102430005B68294698479DE6012384F812316DE5D3
:10244000282303FB020181F81C2100EB820281F8A2
:102450001E5181F81D61906991F81F113EE701231B
:1024600063F30612ECE600BFE82E0020D433002010
:1024700010B5044629B990F81121032A0DD0002087
:1024800010BDD0F8E4359B69002BF8D090F81221EC
:10249000032AF4D19847002010BDD0F890230B46B2
:1024A000D0F87C138A4213D9C078521A0128C4F894
:1024B000902336D08A4228BF0A4692B2C4E9E2236A
:1024C00004F55D71A4F8743320466FF019F8D6E76F
:1024D000D0F8E4351B691BB190F81221032A1ED0F5
:1024E00000234FF480720421C4E94A33C4E94C3319
:1024F00084F81111A4F81C2104F58E7120466EF0A9
:10250000FFFF636D104A1A61E278012AB7D104F225
:10251000CC545C614FF0802219681A60AFE798478D
:10252000DEE78A42D4F88003A4F8743328BF0A4651
:10253000084492B2C4E9E22304F55D71C4F8800353
:10254000C4F88403C0E700BF1800086038B504462B
:1025500049B990F81131022B11D094F81631012BA2
:1025600040D0002038BDD0F8E4355B69002BF8D0AE
:1025700090F81221032AF4D19847002038BDD0F8F2
:102580003831D0F82421934236D9C178012908BFC7
:10259000D0F82811A3EB020318BFD0F82821C0F807
:1025A000383108BF52189BB24FF480710025C0E942
:1025B0004C35A0F81C11C0E94A2200F58E716EF06E
:1025C0009FFFE378C4F88053012BC4E9E255A4F8D7
:1025D000745308BFC4F8845304F55D7120466EF04F
:1025E0008FFFBAE72A4B2269D3F8F4145160002315
:1025F00084F81631002038BDD0F83C31B3FBF2F539
:1026000002FB1535ADB99A4213D8D0F84021934258
:102610000FD24FF48073A0F81C31C0E94A55C0E9CD
:102620004C5500F58E716EF06BFFE378C4F84051A5
:10263000C8E7D4F8E435DB681BB194F81221032A0B
:1026400023D0E2780023012A4FF0050108BFC4F827
:102650008433C4E9E23384F81111C4F88033A4F858
:10266000743304F55D7120466EF04AFF636D094ACC
:102670001A61E278012A7FF470AF04F2CC525A61F9
:102680004FF0802219681A6067E720469847D8E71C
:10269000E82E002018000860F8B50B7813F06006EB
:1026A0000D46044620D0202E25D1CE884EB31B06E1
:1026B00049D5384F687832463946FEF7C3FAEB8879
:1026C0000222002684F811214FF48072C4E94E33AF
:1026D000C4E94A77C4E94C36A4F81C2104F58E718C
:1026E00020466EF00DFF0AE04B780A2B17D00B2B1B
:1026F0000ED0062B03D120466CF0BCFA02263046E1
:10270000F8BD022248781144FEF79CFA3046F8BD25
:102710008B78002B3AD1204BC3F8FC64EFE7022200
:1027200080F811214FF48072A0F81C211B4A01236C
:10273000C0E94E33C0E94A22C0E94C3600F58E713B
:102740006EF0DEFEDBE7164B164A4978116003F6A1
:10275000A4020321C0E9E46680F81111C0F888637F
:10276000C0F88023C078C3F8A06801284FF00003A8
:10277000C4F88C33A4F8743304F55D7108BFC4F851
:10278000842320466EF0BCFE0026B8E76CF072FA97
:10279000B5E700BF94260020E82E0020E433002097
:1027A000F01D002000000020002310B5194604464B
:1027B00040226EF035FE80212046002340226EF03C
:1027C0002FFED4F8E835A078012284F812215B6846
:1027D0009847002010BD00BF10B5022304464022D8
:1027E00081216EF01DFE20460223402201216EF061
:1027F00017FE20460323082282216EF011FE0E4BA5
:102800000222A3F84C20FEF709FAE2780B4BC4F839
:10281000A83340200021C4E9EC01012A4FF0010156
:10282000A4F89C13204604F5677108BFC4F8AC33C4
:102830006EF0D4FE002010BD000000206C3300209C
:1028400070B5812182B00446314E6EF0B7FD012192
:1028500020466EF0B3FD0025022340228121204650
:1028600086F8185A6EF0DCFD012102234022204632
:102870006EF0D6FD274B86F8185AD3F8002583F85A
:10288000E8541268284690470095009BE16843F0A1
:1028900010030093009B0B610A691F4B009203E039
:1028A0000A690092013B02D0009AD006F8D40023B6
:1028B0000193019B43F020030193019A164B0120E1
:1028C00060F38A120192019A0A610A69019203E097
:1028D0000A690192013B02D0019A9206F8D4E2788B
:1028E0000E4BC4F8A83300211F20C4E9EC01012AD3
:1028F0004FF00101A4F89C1304F5677105D0204640
:102900006EF06CFE002002B070BDC4F8AC33F6E788
:10291000F01D0020E82E0020400D0300B033002001
:102920002DE9F843394F8046894615461C4697F8ED
:10293000E01904290CD0082907D1D7F8D839434524
:1029400006D0FEF7F5F90228F1D00120BDE8F883A2
:10295000012387F8C4393B6397F89030C7F8CC4916
:102960000622022B2A4CC7F8C089C7F8C859C7F8F5
:10297000BC9987F8E02918BF4FEA48280A2640F298
:10298000FF554FF48B63A5630121C4F8088018201C
:10299000E360FDF7C3FC03464FF0000C40F27742C2
:1029A00001213720A56393B9012148466CF0C2FB91
:1029B000174B184959624FF400729A62DA6A002183
:1029C00042F09102DA620846B962BDE8F883A56375
:1029D000C4F808C0E260FDF7A1FC721EA5630028E0
:1029E000E2D012F0FF06CCD13E63FEF7D5FDD7F85A
:1029F000C84944B10120D7F8CC39D7F8C0193246BC
:102A0000A0470320E1E70320DFE700BFF01D00201F
:102A1000002C014000E1F5052DE9F04F3F4E9946AD
:102A200096F8E03983B0042B80460191924609D094
:102A3000082B03D0002003B0BDE8F08FFEF778F933
:102A40000228F7D196F890300122022BF26263D06F
:102A50004FEA482B324C019800216CF06BFB4FF48D
:102A60000072304B6362A262E36A40F2FF5743F0A8
:102A70009303E362A763A2604FF48A62E2600121DC
:102A80001020FDF74BFC0A25A76340F25142A763D3
:102A90000121C4F808B01120E260FDF73FFC0246B6
:102AA0004FF0000E40F2774301213720A763AAB907
:102AB0000023B362D6F8143A0199C6F8BC1905226E
:102AC0000120C6F8C089C6F8C8A9C6F8CC9986F80E
:102AD000E029C6F8D03903B0BDE8F08FA763C4F889
:102AE00008E0E360FDF71AFC013DA7630028DFD092
:102AF00015F0FF05C9D1F562B062FEF74DFDD6F8BD
:102B0000C849002C96D02846D6F8CC39D6F8C0193A
:102B10002A46A04728468EE7C3469BE7F01D0020C3
:102B2000002C014000E1F5051049114BD1F8882037
:102B300042F4700210B4C1F888201A680D4C0020CD
:102B400042F001021A6098601A6822F0847222F43E
:102B500080321A605C601A68074C22F480221A6086
:102B6000D8608C605DF8044B704700BF00ED00E05A
:102B7000003802401030002400000008704700BFF9
:102B80002DE9F84346697EB9D0F80080C8F30D09F5
:102B900004460F46B9F1000F26D03F68FDF7D8FE76
:102BA000092804D06FF001063046BDE8F8834A4D8D
:102BB0002B6923F440732B612B6943F400732B6161
:102BC0002B6943F001032B61C8F80070FDF7C0FECC
:102BD0002B69092823F001032B61E3D12368043317
:102BE00023603046BDE8F8833C4B98452AD303F573
:102BF0008043984524D303F58043984554D3384BFC
:102C0000984554D903F58033984553D903F50033DB
:102C1000984552D903F50033984551D903F500334F
:102C200098453ED903F5003398454CD903F58023E8
:102C300098454BD9B8F1016F4BD305200DF072FFC9
:102C40004FF00809FDF784FE092804D04FF0FF3645
:102C50003046BDE8F883204D2B6923F440732B6187
:102C60002B6943F400732B612B6923F0F8032B616C
:102C70002B6943EA090343F002032B612B6943F4F8
:102C800080332B61FDF764FE2B6923F002032B6177
:102C90002B69092823F0F8032B61D7D1D4F80080E1
:102CA0007BE74FF03809CDE74FF01009CAE74FF046
:102CB0001809C7E74FF02009C4E74FF02809C1E71A
:102CC0004FF03009BEE74FF04009BBE74FF048092D
:102CD000B8E74FF05809B5E7003C02400040000853
:102CE000FFFF00080148FDF795BA00BFD80000209B
:102CF0000148FDF78FBA00BF240300200148FDF70B
:102D000089BA00BF700500200148FDF783BA00BFF3
:102D1000BC070020704700BFF0B5254B026825496D
:102D200083B00646002401E051F834309A4209D0BD
:102D300001340E2CF8D100211F4A052005F076FD44
:102D4000002113E01D4F07EB8407D7F8045585B128
:102D5000717901EB410305EBC30300221820C3E99D
:102D6000032200FB01559E601A75291D084603B019
:102D7000F0BD07216C2005F04BFE0146C7F80405A5
:102D800070B129466C2275F089FF0A4BD7F80455BB
:102D900003EBC404C5E90045ED616D63ED64D7E75D
:102DA0000190074A052005F041FD0199DEE700BFCB
:102DB000000001404CAD0708DC4E0808E82E00205A
:102DC000044F0808704700BF30B40C4C0022234663
:102DD00004E001320C2A03F114030CD093F804C070
:102DE0008445F6D1DD68294201D10029F1D11420B2
:102DF00000FB024000E0002030BC7047040A0020C5
:102E000038B5D0E9004307EE902A1B68354A2068A0
:102E10000139934204688DB216D002F58062934264
:102E200012D002F5705293420ED002F580629342A6
:102E30000AD002F58062934206D02B4BD3F8F43AC5
:102E40005B0807EE103A04E0274B03F6F42393EDFA
:102E5000007ADFED266AB8EE477AF8EE677A87EEF9
:102E6000270A30EE260A70F06FFF1E4A23880138C9
:102E7000944280B29BB212D002F5806294420ED08E
:102E8000B4F1804F0BD0A2F58032944207D002F506
:102E90008062944203D002F58062944202D123F012
:102EA00070039BB2124A944212D002F5806294429F
:102EB0000ED023F4407302F56C429BB294422380FF
:102EC000E56220850AD1002323860123A38238BD31
:102ED0002380E56220850123A38238BD054B9C42F7
:102EE000F1D0F8E700000140000000200AD7233CA1
:102EF000001000400004014070B54068837903F081
:102F0000020213F0040300F0C9804FF0000E1346D4
:102F100004247246754690F805C0BCF1030F30D802
:102F2000DFE80CF08E5F30020368188C20F48050CC
:102F30000004000C1884188C9C8820F400500004B5
:102F40002A43000C40EA0232988B6C4D20F4E64094
:102F50000004000CAB42A4B240F4C04000F0B080CA
:102F600005F58065AB4200F0AB809C8098831964C6
:102F70001A849A8B22F400621204120C42F400624A
:102F80009A8370BD2A4305685C4E288C20F48070BB
:102F90000004000C2884288CB5F804C020F40070CC
:102FA0000004000C40EA0222A88B20F07300000409
:102FB000000CB5421FFA8CFC40F0600073D006F59F
:102FC0008066B5426FD0A5F804C0A883E9632A845F
:102FD000AB8B23F008031B041B0C43F00803AB83EB
:102FE00070BD2A430568454E288C20F0100000046F
:102FF000000C2884288CB5F804C020F020000004C0
:10300000000C40EA0212288B20F4E6400004000C79
:10301000B5421FFA8CFC40F4C04061D006F58066D2
:10302000B5425DD0A5F804C02883A9632A842B8B00
:1030300023F400631B041B0C43F400632B8370BD5B
:1030400000682E4E2A43058C25F001052D042D0C19
:103050000584058CB0F804C025F002052D042D0C64
:103060002A43058B25F073052D042D0CB0421FFA61
:103070008CFC45F0600528D006F58066B04224D06F
:10308000A0F804C0058341630284038B23F0080386
:103090001B041B0C43F00803038370BD4FF4807EB8
:1030A0001C46012537E722F4006242EA032222F49B
:1030B00080622CF4405C42EA04224CEA0E1C82E757
:1030C00024F4804444EA8E144FE74FF6F37616401A
:1030D0002CF4407C46EA03024EEA0C0C2243CFE774
:1030E00022F0800242EA031222F040022CF4406CEB
:1030F00042EA04124CEA8E0C94E700BF0000014043
:1031000042685379032B0FD8DFE803F00B08050260
:1031100010684030704710683C3070471068383095
:10312000704710683430704700207047024B0348E6
:10313000D3F80415FEF7FCBCE82E00200000014087
:1031400010B5064C0648D4F80415FEF7F1FCD4F887
:1031500024150448BDE81040FEF7EABCE82E002024
:10316000000001400040014010B5064C0648D4F86C
:103170000415FEF7DDFCD4F828150448BDE810401E
:10318000FEF7D6BCE82E00200000014000440140BC
:1031900010B5064C0648D4F80415FEF7C9FCD4F85F
:1031A0002C150448BDE81040FEF7C2BCE82E0020F4
:1031B0000000014000480140034B4FF08040D3F82D
:1031C0000815FEF7B5BC00BFE82E0020024B0348EF
:1031D000D3F80C15FEF7ACBCE82E0020000400402C
:1031E000024B0348D3F81015FEF7A2BCE82E0020CE
:1031F00000080040024B0348D3F81415FEF798BCB2
:10320000E82E0020000C0040024B0348D3F82015A4
:10321000FEF78EBCE82E00200004014010B5064CDD
:103220000648D4F82015FEF783FCD4F8301504487E
:10323000BDE81040FEF77CBCE82E002000040140F1
:103240000018004010B5064C0648D4F82015FEF7CB
:103250006FFCD4F834150448BDE81040FEF768BC94
:10326000E82E002000040140001C004010B5064C70
:103270000648D4F82015FEF75BFCD4F8381504484E
:10328000BDE81040FEF754BCE82E002000040140C9
:10329000002000400348D0F8043B13B100F6F820AA
:1032A00018477047000000200348D0F8243B13B1B2
:1032B00000F6183018477047000000200348D0F887
:1032C000443B13B100F63830184770470000002027
:1032D0000348D0F8643B13B100F6583018477047E4
:1032E000000000200348D0F8843B13B100F678308A
:1032F00018477047000000200348D0F8A43B13B1E2
:1033000000F6983018477047000000200348D0F8B6
:10331000C43B13B100F6B8301847704700000020D6
:103320000348D0F8E43B13B100F6D8301847704793
:10333000000000200348D0F8043C13B100F6F83038
:1033400018477047000000200348D0F8243C13B110
:1033500000F6184018477047000000200348D0F8D6
:10336000443C13B100F63840184770470000002075
:103370000348D0F8643C13B100F658401847704732
:10338000000000200348D0F8843C13B100F67840D8
:1033900018477047000000200348D0F8A43C13B140
:1033A00000F6984018477047000000200348D0F806
:1033B000C43C13B100F6B840184770470000002025
:1033C0000348D0F8E43C13B100F6D84018477047E2
:1033D0000000002030B44568154CA542154D2C6BFB
:1033E0000CBF44F4001444F480042C6390F914C01E
:1033F000C160BCF1000F836111DB0F49120101EBC9
:103400000C03D2B283F800234FEA5C1001230CF0C6
:103410001F0C03FA0CF330BC41F820307047074B07
:103420000CF00F0C12016344D2B21A7630BC704714
:10343000006002400038024000E100E0FCEC00E0E7
:103440002DE9F84FDFF814B300210BF6F8204FEA0E
:10345000411C50F80C30C3F30132C3F3032382F054
:10346000020283F0030352EA03040AD00131102957
:10347000EDD1A74E0023C6F8103A86F8E039BDE832
:10348000F88F6044A24E037FC6F8100A002BF1D1DA
:10349000DC44A04BDCF8007B9F4202D048339F42C3
:1034A000E8D19D4A536A43F4006353620DF0DEFA9B
:1034B000804689460DF0DAFAB0EB080361EB0901AA
:1034C000B3F57A7F71F10003F4D3934A536A23F47E
:1034D000006353620DF0CAFA804689460DF0C6FAC1
:1034E000B0EB080361EB0901B3F57A7F71F10003DA
:1034F000F4D3DFF824928948D9F8443043F40063C8
:10350000C9F84430D9F8303043F48003C9F830307A
:10351000D9F8303043F00C03C9F830304FF00D0AC1
:103520004FF000080C220E21A6F802AD86F8048D9B
:1035300009F070FD7A48A6F80EAD0C220E2186F82F
:10354000108D09F067FD7748A6F81AAD0C220E2100
:1035500086F81C8D09F05EFD7348A6F826AD0C2296
:103560000E2186F8288D09F055FD7048A6F832AD79
:103570000C220E2186F8348D09F04CFD0C226C488B
:10358000A6F862AD0E2186F8648D09F043FD694B03
:10359000302283F831234FF400325A60D9F83030AA
:1035A00043F48003C9F83030634BC3F83C75594B82
:1035B0009F425CD061496248C1F8A080614BC1F86C
:1035C000A8004FF474176048CF60C1F8A00007202E
:1035D000C1F8B4005D4F42461846194605E0013275
:1035E000102A01F1200100F08F808D68BD42F6D1D4
:1035F0000BEB42115201D1F8FC7A55498F4274D03D
:10360000454F396B41F4800139630BEB02054F499B
:103610000D22A5F8142B9A688A4225D00134102C6B
:1036200003F12003F7D100204A4900230122FFF7CC
:10363000D1FED6F80C3A4BB119689A880B691A4238
:1036400004D1002386F8E039BDE8F88FFDF7E6FDE8
:103650000028F6D1D6F8142AC6F8D029012386F816
:10366000E03986F8D4090AE700EB4410DCE7344976
:10367000C3F80080DFF8CCC099604FF07460324925
:1036800043F8500C19600721583B4246D966604602
:10369000634604E00132102A03F1200334D0996814
:1036A000B942F7D10BEB42135201D3F8FC1A284B65
:1036B000994223D018490B6B43F480030B630BEB47
:1036C00002050D23134AA5F8143BDCF80830934299
:1036D00011D00134102C0CF1200CF6D100201E4921
:1036E00000230122FFF776FEA3E70B4F396B41F46D
:1036F0000011396389E700EB4410F0E706490B6BD2
:1037000043F400130B63DAE700235B68FFDE00BFBE
:10371000F01D00205864024000380240EC2A0020CE
:10372000F82A0020042B0020102B00201C2B002046
:103730004C2B002000E100E0E82E00200064024055
:10374000802C0140F80A00206054A308A0640240C5
:1037500000600240650800089D0700080000002086
:1037600070B52D4C636BD9051ED54FF4807340F2B4
:10377000FF56A363A663E36B284D23F4414323F074
:103780003A03E3636B6B9A071FD4012200236A623A
:10379000AB62214A40F2FF539363D36B23F441435E
:1037A00023F03A03D36370BD636B980703D51B4BBB
:1037B00002229A62EDE7636B190721D4636B9A06C4
:1037C00022D5164B06229A62E3E7154BD3F83C2527
:1037D000136823F001031360E36A002223F0080357
:1037E000E3622A636B6BDB07CFD540F24C43A663E1
:1037F0000121A2600C20E360FCF790FDA663C4E702
:10380000064B04229A62C4E7636BDB06C1D5034B07
:1038100005229A62BDE700BF002C0140F01D002088
:10382000E82E002002683649002310B422F001027D
:10383000212488420260036043608360C3600361A7
:10384000446138D02F4B98422ED02F4B98423CD019
:103850002E4B984240D02E4B984232D02D4B98425E
:1038600041D02D4B984246D02C4B984217D02C4B30
:1038700098423CD02B4B984216D02B4B984224D0E8
:103880002A4B984228D02A4B98421AD0294B98426A
:1038900029D0294B98422ED0284B984208D14FF07E
:1038A0003D5243F8AC2C03E04FF4746243F8202CF3
:1038B0005DF8044B7047224B5DF8044B3D229A6043
:1038C0007047204A43F8642CF2E74FF474125DF815
:1038D000044B43F8382C70474FF074625DF8044B8A
:1038E00043F8502C7047184A43F87C2CE0E73D22FF
:1038F00043F8082CDCE7154A43F8942CD8E700BFBE
:10390000106002402860024040600240586002405F
:103910007060024088600240A0600240B8600240CF
:10392000106402402864024040640240586402402F
:103930007064024088640240A0640240B86402409F
:10394000006002403D000020400F002000003D20AC
:1039500000222DE9F04713460D684FF0010E0326B3
:1039600004E00133102B02F1020239D00EFA03FCFD
:103970003CEA0504F5D1076806FA02F427EA0407D1
:1039800007600F79D0F800A007FA02F9013F49EA71
:103990000A09012FA046C0F800906FEA040411D86C
:1039A00087683C4084604C79876894403C438460DD
:1039B000446824EA0C0444608C7947689C40A4B2B3
:1039C0003C434460C46824EA0804C460CC79C768F6
:1039D000944001333C43102BC46002F10202C5D174
:1039E000BDE8F0872DE9F0412348244F244E254CB3
:1039F00082B03822002175F051F9002557F82510C2
:103A00003246002301E054F8332091422ED0013396
:103A10000E2BF8D1002005356BF014FC3C2DEDD1B8
:103A2000DFF85880184F08F1F0054FF0007698F84D
:103A3000040009F0EBF808F11408044688B10368A3
:103A400003F13F4303F57E0307EB932393F8C8008C
:103A50006BF0F8FBA3880196206800936946FFF796
:103A600077FFA845E3D102B0BDE8F081064A02EB3A
:103A7000C30393F85C00CEE7EC330020040A002077
:103A8000000001404CAD0708F4AC0708224A9368D7
:103A900003F00C03042B10B421D0082B22D01F4BB1
:103AA00003601D4C1E4AA168C1F30311114491F833
:103AB000F81CCB404360A168C1F38221114491F806
:103AC000F81C23FA01F18160A1685DF8044BC1F391
:103AD00042310A4492F8F82CD340C3607047114B2E
:103AE0000360DEE75368516813F4800F01F03F0173
:103AF000536814BF0B4A094AB2FBF1F1064A5268F7
:103B0000C2F30142C3F38813013201FB03F35200F5
:103B1000B3FBF2F30360C4E7003802400024F40072
:103B20000000002000127A0070B5446B8668A389FB
:103B300023F400531B041B0CA381827905464079B2
:103B400012F0040F14BF4FF4805C4FF0000C11030F
:103B500010F0010F4FEA02220CBF0023042302F4ED
:103B60008062800748BF43F0080342EA0C02134317
:103B7000228A92B201F4005122F440520A43228276
:103B8000A28922F4B05222F00C021204120C1A4341
:103B9000A281A38A23F440731B041B0C84B0A3826C
:103BA0006846FFF773FF244B9C4205D003F5806302
:103BB0009C4201D0029A00E0039AA3891F491B048A
:103BC00002EB82024CBF7300B30002EB8202B2FB35
:103BD000F3F3A1FB0302A08952096426000406FB4B
:103BE00012334FEA02121FD41B013233A1FB03131D
:103BF000C3F3431313439BB22381AB796A6B13F076
:103C0000080F938A0AD09BB243F0080393829389EA
:103C10009BB243F40053938104B070BD23F00803BA
:103C20001B041B0C9382F2E7DB003233A1FB03136E
:103C3000C3F342131343DEE7001001401F85EB512D
:103C40002DE9F8431D462E4B9DF820609DF82490E9
:103C50009842884617463BD02A4B984240D02A4B80
:103C6000984245D0294B984221D14B4632462946AD
:103C70000520FDF797FE04460023C4E90B87C4E93D
:103C80000733C4E909336671A56084F806902046BD
:103C9000FFF74AFFF107626B12D4B3070BD4938985
:103CA0009BB243F4005393812046BDE8F88300247F
:103CB0002046BDE8F883D36843F08003D360EEE785
:103CC0004FF6DF731380D36843F02003D360E4E73B
:103CD0004B46324629460020FDF764FE0446CBE7FA
:103CE0004B46324629460120FDF75CFE0446C3E7F9
:103CF0004B46324629460320FDF754FE0446BBE7F7
:103D00000010014000440040004C004000140140FD
:103D1000816009E7417107E72DE9F043DFF814827C
:103D200008EBC00985B00546C70099F80C0D08F0EE
:103D30006DFF044699F80D0D08F068FF064699F8E6
:103D40000E0D6BF07FFA6B1CDBB2002C00F0AD8027
:103D500040F60C122372E280002E00F0C380337212
:103D600040F60C232046F38004223A2109F052F950
:103D7000042230463A2109F04DF908EB0703624A64
:103D8000D3F8084D944200F09880604B9C4200F0BC
:103D90009E805F4B9C4200F0AB80474497F80F2D0C
:103DA000022A5CD0032A7ED05A4B5B4E012A18BFF0
:103DB0001E46A7886846FFF769FE27F03F07029B6B
:103DC000564AB3FBF6F63F04A2FB03233F0C47EA37
:103DD0009347A780228822F001021204120C22804D
:103DE000B2B2C6F30B069B0C002E59D04FF496715D
:103DF00001FB03F34A49A1FB03139B0901339BB267
:103E000042F400422384A2832388464A9BB243F0B3
:103E100001032380238823F4816323F002031B041E
:103E20001B0C4FF4804143F480632380218123885D
:103E300023F080031B041B0C238023889BB202EB1E
:103E4000451243F0010323800121002382F84055ED
:103E500082F8411582F8423505B0BDE8F083A688A6
:103E60006846FFF713FE26F03F06029A2B4B3604F6
:103E7000A3FB0213360C46EA9346A680218821F064
:103E800001010904090C21809B0C27490133920987
:103E90002384A1FB02329209042A38BF0422B2E72C
:103EA00042F00102A2E7214E83E7002E3FF465AF06
:103EB000337240F60C23F3805AE71D4B1A6A42F422
:103EC00000121A621A6A22F400121A6265E703F5F8
:103ED000F0331A6A42F480021A621A6A22F48002EB
:103EE0001A625AE7042220463A2109F093F844E77F
:103EF00003F5EE331A6A42F400021A621A6A22F4D7
:103F000000021A6249E700BF005400400058004018
:103F1000005C0040804F1200009F240083DE1B43A2
:103F2000D34D6210E82E0020632D3E05C027090006
:103F300000380240000000202DE9F047954D90F92F
:103F400000108046807805EBC1060138CC0090B0A7
:103F5000D6F8081D14282ED8DFE810F053012601EA
:103F6000150057006100A200AA00CB01BD017D0031
:103F7000870045020D02E001C500D5003000380081
:103F8000AA019C015B01888A0C8B81B2824841EABC
:103F9000044130EA010100F02681D8E90210521AEA
:103FA00042F2107163EB00038A4273F1000302D303
:103FB000152388F8023010B0BDE8F08798F8130098
:103FC0000882C8E90223122088F80200888A0C8B34
:103FD00080B240EA0440714C34EA000000F0B68040
:103FE00000200E900F9001200F910E900E99002945
:103FF00000F01E820F9914310F910F99096849053D
:10400000CBD5142388F80230D5E798F8110000F0DA
:10401000FE000882C8E90223052088F80200888A89
:104020000C8B80B240EA04405D4C34EA000000F0A2
:10403000A48000200090019001200191009000993F
:10404000002900F001820199143101910199096858
:104050004F05D6D4A1E798F8110040F0010008827E
:10406000C8E902230B2088F80200888A0C8B80B2F2
:1040700040EA04404B4C34EA00006FD0002004902A
:1040800005900120059104900499002900F0D68143
:10409000059914310591059909684D05B1D47CE75E
:1040A00098F813000882C8E90223072088F8020064
:1040B000888A0C8B80B240EA0440384C34EA000015
:1040C0005FD000200290039001200391029002999A
:1040D000002900F0C58103991431039103990968FF
:1040E0004E058ED459E7088820F480600004000C47
:1040F000088098F8110000F0FE000882C8E9022349
:10410000102088F80200888A0C8B80B240EA0440B4
:10411000234C34EA000012D000200C900D900120B6
:104120000D910C900C99002900F094810D99143197
:104130000D910D99096848053FF563AF2DE798F893
:104140001330FF2B06D198F810301BB1132388F8D9
:10415000023030E7112388F802302CE7D8F8140039
:10416000012800F09381022800F049820E20098B7B
:1041700088F80200C8E902231DE7062388F8023008
:1041800019E7D8F81400002800F07081082388F897
:10419000023010E700000020010003008400070047
:1041A0008200070002000300088820F40060000479
:1041B000000C0880088880B240F48060088008887D
:1041C00080B240F480700880032088F80200888A5A
:1041D0000C8B81B2AB4841EA0441C8E9022330EAC2
:1041E00001037FF4E8AE98F81230002B40F0D38141
:1041F00098F81330FF2B00F04682042388F8023031
:10420000D9E6098889053FF5C8AE002388F8023051
:10421000D1E62C4494F80C0D08F0F8FC064694F80E
:104220000D0D08F0F3FC984AB2F8A03501339BB2AB
:104230008246A2F8A03516B13368B2881A83BAF163
:10424000000F04D0DAF80030BAF804201A831121E4
:10425000304605F0FFFC1121504605F0FBFC4FF005
:10426000090965272EB13368B28819690A4240F0FE
:104270002881013F00F022810CF0F8FB04460D4636
:104280000CF0F4FB001B61EB0501052871F1000344
:10429000F6D3E7E7088880B240F4007008804FF654
:1042A000FF3088820121C8E9022388F8021082E6E3
:1042B000D8F81400002800F07281D8F8184014F8DB
:1042C000016B0E8201381225C8E90504C8E90223F2
:1042D00088F802506FE6888A0C8B81B2694841EAFF
:1042E000044130EA01017FF458AE0A2388F8023015
:1042F00061E6088880B240F480700880092088F860
:104300000200888A0C8B81B25E4841EA0441C8E908
:10431000022330EA01037FF44EAEE6E700240125D4
:104320000A940B940B910A950A98002800F04A8190
:104330000B9814300B900B98006846077FF52DAE54
:10434000D8F81400032800F07281022800F2468198
:10435000088820F480600004000C0880088880B27F
:1043600040F400700880098A88F81C40C8E90223DC
:1043700088F802501FE60020012408900990099156
:1043800008940898002800F01781099814300990C3
:104390000998006847077FF500AEEFF311851020FC
:1043A00080F31288088880B240F400700880D8F842
:1043B00018000E8A471CC8F81870EDB2067085F315
:1043C00011880D8AD8F818106FF001004E1CC8F83B
:1043D00018600D70C8E90223C8F8140088F81C4062
:1043E00088F80240E7E50020069007900120079139
:1043F0000690069C002C00F0EB80079C1434079478
:10440000079C246864067FF5C8AD0C8AD8F818109C
:104410004D1CC8F818500C70D8F8141088F81C00FF
:104420000139C8E90223C8F8141088F80200C2E56F
:104430000F9918310F910F990968AEE50599183158
:10444000059105990968A8E501991831019101992B
:104450000968A2E50D9918310D910D9909689CE53F
:104460000399183103910399096896E5088880B289
:1044700040F4007008800121C8E9022388F8021086
:1044800099E500BF01000300E82E0020088820F411
:1044900080600004000C0880EFF31184102080F38A
:1044A0001288088B088880B240F40070E4B208805B
:1044B00084F311880C2188F802105BE616B133688A
:1044C000B2885A830CF0D2FA04460D460CF0CEFAAC
:1044D000031B61EB0501052B71F10003F6D316B147
:1044E0003368B2881A830CF0C1FA04460D460CF00A
:1044F000BDFA031B61EB0501052B71F10003F6D337
:10450000B9F101097FF4ADAE16B13368B2885A83B0
:104510000CF0ACFA04460D460CF0A8FA031B61EB54
:104520000501052B71F10003F6D3BAF1000F04D099
:10453000DAF80030BAF804205A830CF097FA0446EF
:104540000D460CF093FA031B61EB0501052B71F18D
:104550000003F6D316B13368B2881A830CF086FADA
:1045600004460D460CF082FA031B61EB0502052B95
:1045700072F10003F6D3BAF1000F04D0DAF800307C
:10458000BAF804201A8398F90000441C3FF43DAEA9
:10459000FFF7C2FB39E60F2388F802300BE50888E5
:1045A00080B240F4007008800121C8E9022388F835
:1045B0001C1088F80210FEE4099918310991099934
:1045C0000968EAE40B9918310B910B990968E4E446
:1045D00007991831079107990968DEE4D8F818009F
:1045E000098A441CC8F818400170D8F81410C8F89B
:1045F00008200139C8F81410C8F80C30DBE408882A
:1046000080B240F400600880EFF31184102080F342
:104610001288088B088820F480600004000CE4B243
:10462000088084F311880D2188F80210A2E508881B
:1046300020F480600004000C0880EFF31184102047
:1046400080F31288D8F818000D8A461CC8F8186044
:104650000570088880B240F40070E4B2088084F3EA
:104660001188D8F81800098A441CC8F8184001704D
:10467000D8F814100C200239C8E90223C8F8141025
:1046800088F8020097E498F81030002B3FF4B5AD9D
:104690002BE600BF38B5184D9DF814E005EB40142B
:1046A0004FEA401C94F8410500B938BD84F8532501
:1046B000C4F8543501220023490005F5A86584F8A3
:1046C000522584F85C35049A84F850E5022384F876
:1046D0005115C4F8582584F8423565440CF0C6F9E4
:1046E00002460B462846FFF727FC94F84235002B7C
:1046F000F4D194F85C0538BDE82E002038B5184D8B
:104700009DF814E005EB40144FEA401C94F8410575
:1047100000B938BD490084F85325C4F8543584F8ED
:1047200051150023049984F850E5022205F5A86587
:1047300084F85235C4F8581584F85C3584F842255D
:1047400065440CF093F902460B462846FFF7F4FB4C
:1047500094F84235002BF4D194F85C0538BD00BFC5
:10476000E82E0020F0B587B00023824A0093019321
:10477000136843F48033136003E0009BB3F5A04F4C
:1047800009D0136803F400330193009B01330093B5
:10479000019B002BF1D0774B1B6813F4003318BF3B
:1047A00001230193019B012B01D000BFFDE7714B59
:1047B00071491A6C714842F080521A640A6842F4D6
:1047C00040420A609A689A609A6842F400429A608D
:1047D0009A6842F4A0529A6058601A6842F0807257
:1047E0001A601A689201FCD5654A40F205711160A1
:1047F000996821F003019960996841F00201A2F5DE
:1048000080629960936803F00C03082BFAD19368D7
:1048100003F00C03042B00F08C80082B00F08E803A
:10482000584D594BC5F8F43A524BD5F8F41A9A68DA
:10483000564C5748C2F303122A44002692F8202D02
:10484000D140544AC5F8F41AE260534A596FA26045
:10485000596B524A21F080015963596F41F08071C0
:104860005967196B0A431A635A6B5A639A6B9A63B6
:104870001A6C4B490A431A64596C4A4A0A435A64EF
:1048800002A948F2FF7302934FF6FF770396FFF7F2
:104890005FF800F580600297FFF75AF800F5806036
:1048A0000297FFF755F800F58060FFF751F800F523
:1048B0008060FFF74DF800F58060FFF749F800F5DC
:1048C0008060FFF745F800F58060FFF741F800F5DC
:1048D0008060FFF73DF80846FFF7D8F8D4F8FC30C1
:1048E000029A3149314843F08073C4F8FC30304BB0
:1048F000C3F8B01F5E60196841F001011960D5F876
:10490000F43A4FF47A71B3FBF1F3013BB3F1807FDA
:104910002849B2FBF1F2C0F8A42508D24FF0E022FA
:10492000F0215361072384F823109661136107B0C7
:10493000F0BD144D204BC5F8F43A75E75368516843
:10494000104D13F4800F01F03F01536814BF1A4A51
:104950000D4AB2FBF1F1074A5268C2F30142C3F3B8
:104960008813013201FB03F35200B3FBF2F3C5F8E5
:10497000F43A59E7003802400070004008544007FC
:10498000003C0240000000200024F40000ED00E0A4
:10499000000002400003FA0500000008FF916700D4
:1049A000FFC9FE103357070055CEACC5E82E0020D6
:1049B000001000E040420F0000127A0082B0064B67
:1049C000002201920193019B03EB80000190019B67
:1049D000196002B0704700BF5028004010B51C207D
:1049E00008F014F91121044605F034F94CB123689C
:1049F000A2885A83C8200CF067F82368A2881A831B
:104A000010BDBDE81040C8200CF05EB8704700BF74
:104A1000704700BF704700BF10B5124C94F8B23514
:104A200023B9114B4FF480225A6110BD4FF0E022A0
:104A3000D2F8103D23F00603C2F8103DFEF774F8DB
:104A400094F8B235002BECD0D4F8B8359B68DB076E
:104A5000E7D5D4F8B426136823F0030161F3070304
:104A60001360DEE7E82E0020003C01402DE9F04F06
:104A7000B34CD4F8B4355A69D2078BB002D50BB019
:104A8000BDE8F08F5A699B6912EA0309F7D0C9F3B0
:104A9000074319F4002F009340F0E180009B590771
:104AA00043D419F0020F5FFA89F603D0D4F8B43575
:104AB00002225A61B9F1000FC0F2EE8119F4006FC1
:104AC000C9F3072540F04A81330708D59D4B9E481E
:104AD000D3F83C3D9847D4F8B43508225A61F7061C
:104AE00000F1C481EE0600F16F81A90600F1E880B3
:104AF000009BDA0609D5934B9348D3F84C3D984771
:104B0000D4F8B4354FF480125A61009B9B06B6D599
:104B10008C4B8D48D3F8503D9847D4F8B4354FF4BA
:104B200000125A610BB0BDE8F08FD4F8B825936934
:104B3000D26913401FFA83FABAF1000FB1D0DFF83F
:104B40001882CDF80C90A8F1180500271AF0010F73
:104B500078D0FEB2D4F8B82504EB86031069D3F8F8
:104B6000C015536B8968F340DB01DBB203430B4094
:104B700013F00109D9B240F0AB810A0740F1C881B6
:104B8000D8F8002008239360994619F0800F59D077
:104B9000D5E94CC0D5F82431D8F800E0ACEB0001E1
:104BA0008B42DEF8182028BF0B4692B20333B2EBDB
:104BB000930F47D9D4F8B82594F8AB95323604EB67
:104BC0008603CDE90178674698469446874237D9EF
:104BD000D5F82431391A994228BF194601F1030B3F
:104BE000D5F828314FEA9B0BB9F1000F10D18AB2EA
:104BF00003329210D8F8B0650AD04846013053F815
:104C0000047B37608242F9D1D5E94C70D5F8283160
:104C100008440B44B842C5F82831C5F83401DEF821
:104C200018300AD195F81C11012202FA01F1DCF8C2
:104C3000342022EA0102CCF834209BB29B45C5D334
:104C4000DDE901785FEA5A0A07F1010708F1040873
:104C500005F128057FF47AAFDDF80C9021E7D4F850
:104C6000B8359D69DB691D402D0C3FF417AF04F585
:104C7000B568DFF8D0B004F2FC560027C24608E061
:104C80006D0807F1010706F1040608F128083FF452
:104C900005AFEB07F4D5F9B204EB8103D4F8B825DE
:104CA000D3F8FC359B6852691340D807DAB200F19B
:104CB0003F81930740F16781336802229A60DFE702
:104CC000D4F8B835D4F8C0159A680868C2F3410220
:104CD000022A06BF032262F30A006FF30A0008608B
:104CE0005A6842F480725A6006A8FEF7CFFED4F8E4
:104CF000B425D4F8B815D368079D6FF38D23D3601E
:104D000088681249C0F34100014491F8D01003298A
:104D100000F05F810E490F480126294484F8AA65F6
:104D200081424FF04006A4F8AC6500F2AC810E2140
:104D300061F38D234FF40051D3605161D8E600BF79
:104D4000E82E00200000002090340020F4AC07087A
:104D5000401E1BFF3F420F00A834002000238DF8A7
:104D6000133094F8BA368DF81330B64BB648D3F8F2
:104D7000443D9847D4F8B835D4F8B425986894F8E9
:104D8000B2354FF400615161002B3FF49DAEC20774
:104D90007FF59AAE94F8BD36012B7FF495AE9DF861
:104DA0001330032B7FF490AED4F8B436A7491A68B9
:104DB00042F001021A601A6842F003021A600B699D
:104DC00043F006030B617FE6D4F8B865D4F8B41558
:104DD0007368002723F0010373600597059B43F078
:104DE00020030593059B67F38A130593059B0B61CD
:104DF0000B690593BC46964B03E00A690592013B9B
:104E000002D0059A9006F8D494F8A92552B1914B96
:104E100003EB820EFF2253F8040F8260D86B7345B8
:104E20008260F8D10B2363F3070763F3070C4FF09D
:104E3000FF33B3614FF00113F3617761C6F810C01F
:104E4000336885486FF30A13336094F8AB25D4F8C0
:104E5000FC35012A186100F0B5804FF480534B6196
:104E6000784B7948D3F8403D98473EE6D4F8B435BE
:104E70009A6922F010029A611A6AC2F3434002282A
:104E800002F00F0100F0B080062800F087809A69D8
:104E900042F010029A6125E694F8B2353BB1D4F89D
:104EA000B426136823F0030161F307031360D4F8F9
:104EB000B825644B6448D3F8481D536823F00103B8
:104EC00053608847D4F8B4354FF000425A61F5E595
:104ED000516BD8F800005B4B4FF0010C0CFA07FC4B
:104EE00021EA0C0151630122D3F8343D826031463E
:104EF0005548984794F8AB35012B00F0B18019F074
:104F0000020F3FF442AED8F8003002229A6099E6D0
:104F1000CB0604D5D8F8003010229A6092E64806F5
:104F200058BF8946EBD5D8F8003040229A6089E610
:104F300094F8AB25336801208242986007D11A6942
:104F4000D8F87C33C2F312029B1AC8F88C33DBF812
:104F5000303D5046984794F8AB35012B7FF490AE26
:104F6000002F7FF48DAE94F8B936052B7FF488AE10
:104F7000D4F8FC35384A1A61384A5A611A684FF039
:104F800080221A607CE610077FF57AAEDBF8383DA8
:104F900050469847336808229A6071E601EB810118
:104FA00004EBC101D4F87866D1F83409C2F30A12CF
:104FB00002443068C4F8740B3068C4F8780BC1F848
:104FC000342964E7254A5A611A684FF080221A6032
:104FD00043E7002184F8AA154FF40071A4F8AC153A
:104FE000092161F38D23A5E647F6F07010423FF4E6
:104FF0004EAFC2F30A1201EB810004EBC00002F1D4
:10500000030C5FEAAC0CD0F82869D4F878E64FEAD4
:10501000810818BF002006D00130DEF8007046F885
:10502000047B8445F8D1414404EBC101D1F828093F
:105030001044C1F82809D1F834090244C1F83429D0
:1050400025E700BF000000209034002000ED00E0C4
:10505000400D0300A4340020180008605C3A0020D2
:10506000002F7FF44CAF94F8B936042B7FF447AF90
:10507000D4F8FC352B4A1A612B4A5A611A684FF052
:1050800080221A603BE72948A5F57401A1F510516B
:10509000814203D80D2161F38D234BE62449254835
:1050A0002944814203D20C2161F38D2342E6224838
:1050B000A5F18C71A1F54341814203D80B2161F325
:1050C0008D2337E61D491E482944814203D20A2117
:1050D00061F38D232EE61B491B482944814203D2EC
:1050E000092161F38D2325E61848A5F1B771A1F5D3
:1050F0005851814203D2082161F38D231AE61449E5
:1051000014482944814203D2072161F38D2311E61B
:10511000114912482944814234BF0621052161F317
:105120008D2307E6180008605C3A0020DFC81000F5
:105130002013FBFE20D61300FF69180000D3CEFE1B
:1051400040771B00C05BB3FEC091210040AC27003C
:10515000C01D6AFE40E13300803C36FEE09C410009
:105160000378022B12D00E4943680269D1F8180265
:1051700010B41840D1F81042D1F80C12931E400A16
:1051800004FB030008445DF8044B7047044B42687D
:10519000D3E9800100EB410000EB5220704700BFD3
:1051A000BC5A00202DE9F84F12F0020E01D0002861
:1051B0003CD08A4DD5F80872002F43D14FF0FF3C08
:1051C000874CE146E046E24600262768B84200F0F8
:1051D000D98094F80EB0BBF1000F4ED0BBF1010F97
:1051E00016D1804F06F5817B07EB0B1B9BF807B0B0
:1051F0001BF0010F0CD11BF07E0F09D15FEADB170A
:1052000040F0B480D4F808B0D34501D2DA46B146B4
:105210000136082E04F11004D7D1BCF1FF3F38D17C
:10522000B8F1FF3F30D06F4CC44633E06B4D95F87A
:10523000B431A5F58054E3B10123637002263046F2
:10524000BDE8F88FD5E9834606FB0744A042B5D3F5
:1052500095F8B43113B9012385F8B431614B0122BB
:1052600000265A703046BDE8F88F95F8B431002B0F
:10527000E2D1012385F8B431DEE7B4460136082EC9
:1052800004F11004A1D1C8E7B9F1FF3F18BFCC4623
:1052900074D0544CD5F8986004EB0C1841F21809FE
:1052A000013648F8090041F21C090CF5817748F8ED
:1052B00009604FEA0718C5F8986044F8086004EBE5
:1052C00007164FF00008C6F8048004EB0716B679FD
:1052D000042ECAD8DFE806F0031952192F0012F085
:1052E000010868D104EB0710D61090F80790032B43
:1052F00066F3C71980F807905BD94FF6FF708342B9
:1053000028BF034604EB07108380BEF1000F12D0C4
:10531000D5F89830D5F89C0001330130C5F89830A5
:10532000C5F89C0004EB0C1041F21C05435104EB42
:10533000071304209871500705D504EB0710C379B3
:1053400043F00103C371D30608D504EB0714E379D6
:10535000C3F34502013262F34603E371224B012697
:1053600003EB4C230B603046BDE8F88FB0460136A6
:10537000082E04F110047FF428AF4EE700263046D3
:10538000BDE8F88F174C06F5817704EB071C4FEA50
:1053900007189CF806C0BCF1000F01D1B44679E7AC
:1053A000B446D5F89860013644F80860C5F89860AE
:1053B0008BE74346A6E70D4BD3F8683D002BDDD0C5
:1053C00009495D680A4A01EB4C210023A8470028DF
:1053D000D4D004EB07140223A37130E7BC5A002099
:1053E000D45A0020BC4A0020D44A0020F01D0020DE
:1053F000E50D000870B5104E3378022B0F4B0BBF34
:10540000020AC0F3D412C4B200F07F04D3F8000241
:1054100082B010440D460023032201A9FFF7C2FE0B
:10542000012807D13378022B019B0CBF23F81450BD
:1054300043F8245002B070BDBC4A0020BC5A002082
:105440002DE9F04FDFF82C8198F80060032E85B02D
:105450000C46154643D001288CBF00220122022EA3
:105460000B68019269D14FEA1329DFB24FF4807AB9
:105470000138012820D84FF0010B9D4217D93C4E2E
:10548000D6F878211AB1D6F89411994258D0D6F8A6
:10549000000200234844092203A9FFF783FE0128E4
:1054A0002CD0022817D020B123689D42E8D825606F
:1054B000032005B0BDE8F08FF7B12D4B93F8B42170
:1054C00012B9012283F8B4210123022088F80130A7
:1054D00005B0BDE8F08F022005B0BDE8F08F0128CF
:1054E0008CBF0023012301930B684FF0800AC3F3A4
:1054F000D41903F07F07BBE7D346BEE798F8002036
:105500000399DDF804C0022A14D0032AE3D151F82C
:10551000273023F07043B3FA83F35B0963455F449C
:10552000236821D05B4457452360ECD309F101097E
:105530000027BAE731F81730EDE74FF4807AD6E765
:10554000D6F81012013A02EB41224902B2FBF1F205
:105550001344B3FBFBF20BFB12320AB15B449B1A00
:105560009D4223608CD8A2E7AB42A2D39FE700BF45
:10557000BC5A0020BC4A00202DE9F04FDFF86CB186
:105580009BF800C0BCF1020F894683B009688246CF
:10559000174640F08C800BF58053CEB2D3F8005202
:1055A000A6EB010805EB112590444FF48073984455
:1055B000B94208F1FF38B8FBF3F84CD2A844BCF16B
:1055C000030F07EB06040CBF80224FF48072641AAD
:1055D0009442A8EB050328BF144666B994422CBF39
:1055E0000A220B2201A92846FFF7DCFD012809D079
:1055F00003B0BDE8F08F0B2201A92846FFF7D2FDCA
:105600000128F5D19BF800C0D9F80010BCF1020FB9
:1056100001F1010323D0B44210D9019906F180426F
:10562000013A01EB8202043901EB840142F8043FA4
:10563000914203F10103F9D1D9F80010A61B3144BE
:10564000BAF1010FC9F8001021D08F4205F1010510
:105650004FF00006B3D8012003B0BDE8F08FB4428C
:10566000ECD9019806F10042013A00EB42020238FF
:1056700000EB440022F8023F904203F10103F9D10C
:10568000A61B3144BAF1010FC9F80010DDD1B942AF
:10569000DBD1BCF1020F1DD004F18044019B013C21
:1056A0004FF0FF3243F82420D9F80010CDE70BF576
:1056B000805301F07F06D3F80032BCF1030FC1F331
:1056C000D415A6EB01081D44904414BF4FF4807319
:1056D00080236CE704F10044019B013C4FF6FF720C
:1056E000504623F8142003B0BDE8F08FBC4A0020D8
:1056F00030B50446C06983B010B9012003B030BD95
:105700000D460023032201A9FFF74CFD0128F5D126
:10571000B4F92030002B0ADA144B93F8B4210AB9FB
:1057200083F8B401124B01225A700220E6E7019A75
:10573000012D4FEA431102EB431303D0022D11D187
:10574000E5255554A268DA612278032A04D10022A3
:105750001A775A779A77DA77626A5A83120C9A82A2
:1057600003B030BDE268DA61EEE700BFBC5A00204A
:10577000BC4A00202DE9F04190F83C30002982B06D
:10578000044614BF02210021042B7BD8DFE803F07C
:10579000030C3D486900FFF7ABFF012870D1626B35
:1057A000002A75D184F83C00404EDFF808814FF69E
:1057B000F77706F5805516E0BA424FD869F030FA0F
:1057C00001284FF000011DD1206BFFF713FE0128C7
:1057D00018D1019AD5F814122263531E8B4228BFA8
:1057E0000B46C5F814323278236B032A01A91846F8
:1057F0009AB2E1D1434531D869F012FA01284FF04D
:105800000001E1D002B0BDE8F081426B04F130014B
:105810000020FFF7B1FE012832D1032384F83C3089
:105820002348E16AD0F89431D0F81022C0F89411DE
:105830005B1A02FB03F3D0F8782102EB4322C0F895
:105840007821D0F87C2102EB4323C0F87C31002181
:1058500000F5B870FFF74CFF012811D1042384F83C
:105860003C3094F82830042B04BF002384F82830FF
:10587000A36B8BB120469847012002B0BDE8F081B0
:105880000228BFD194F82830042B09D00220B9E7B0
:10589000022384F83C30B9E7012002B0BDE8F08172
:1058A000002384F828300220ACE700BFBC4A002067
:1058B000BC5A0020F7FFFF0F38B590F8343004468B
:1058C000052B43D8DFE803F01E033C0F185E006B86
:1058D0004FF0FF31FFF78EFD012837D1E06AB8BBEA
:1058E000032384F8343000212046FFF701FF01280C
:1058F0002CD1042384F8343094F82830082B2BD092
:10590000012038BD204DD5F8082200F130010232C7
:105910000120FFF795FD012823D00238C0B20128ED
:1059200014D8052384F8343094F82830082B04BFA9
:10593000002384F82830012385F8B531022038BDD2
:10594000C06A216BFFF756FD0128C9D0002038BD81
:10595000022384F83430F4E7002384F8283001204F
:1059600038BDE368D5F81012D4E90B2003EB4123CE
:10597000C5F81402C4E9033002B96062012384F857
:105980003430A5E7004DCFE7BC5A002010B590F8A1
:1059900038300446032B4DD8DFE803F0022F38439C
:1059A0002B4AC068117802F580530329D3F81012EE
:1059B000D3F894210CBF4FF0800C4FF4807C01FB96
:1059C0000CF100EB4120C4E90302D3F87801A0EB0D
:1059D0004120C3F87801D3F87C01A0EB4121E06AB3
:1059E000C3F87C1102EB0C01C3F89411C4E90C213B
:1059F00048BB6262012384F8383016480021FFF763
:105A000077FE012811D1022384F83830626B04F14B
:105A100030010120FFF7B0FD012806D1032384F8EF
:105A2000383000212046FFF763FE431EDBB2012B16
:105A300001D910BD022094F82830062B04BF0023A2
:105A400084F8283010BDA2EB0C022263D2E700BF1D
:105A5000BC4A00202C5C00202DE9F0434368C3F3CE
:105A600008020A44B2F5007F83B004460D4605D211
:105A70002B446360012003B0BDE8F08390F91A2045
:105A8000501C0AD0444902F5817201EB0212D1790F
:105A90006FF30001D171FF22A27694F91B20511CF3
:105AA00016D03D4802F5817100EB011200EB0111A7
:105AB000D279C879C2F34502012A86BF02F1FF32CA
:105AC00002F03F020022FF2662F34600C871E6762C
:105AD00094F800C0BCF1020FCAD0DFF8C480D8F837
:105AE0001022B5EB422F4FEA422915DCD8F8187284
:105AF0001F407A42AA420FDCEA194A4510D22069B7
:105B00000028B7D0244A1278032A40D080B24FF63A
:105B1000F7729042ACD9ADE7002003B0BDE8F08346
:105B2000227E206912F0080626D0D8F89421411C64
:105B30008A4213D300D100214B44A5EB0905DB1B9E
:105B4000BCF1020F60613D44216163600846D7D11A
:105B5000D8F82022B3EB422F8AD38BE798F8B421F0
:105B600022B9012388F8B431636820690A4A012602
:105B7000567094F800C0DFE701A969F051F80128D8
:105B8000CAD10199636894F800C02069D4E7034A38
:105B900090427FF66DAF6DE7BC4A0020F7FFFF0F24
:105BA000BC5A00202DE9F04790F8384082B00546F5
:105BB000032C00F2AD80DFE804F00219730BFFF74D
:105BC0007BFE012810D002280AD1032385F8383043
:105BD0002B6C002085F82800002B71D098470224F8
:105BE000204602B0BDE8F08785F838002B78022BFC
:105BF00062D0484A6B68D2F8182203EA0208C8F358
:105C00004F282846FFF7ACFA424F0646A8EB00089B
:105C1000A7F5805901A9022200233046FFF7C2FAF6
:105C200008EB060401281FFA84FA4FF400724FF0C3
:105C300000010446D4D1019873F030F8EB694FF4B9
:105C40000071284613B16B68002B3DD0D7F8103295
:105C50005A1E924506F101060DD2FFF7FDFE0028FF
:105C6000D8D197F8B43113B9012387F8B43101239F
:105C700089F80130CEE7C3EBC353590201F5007137
:105C80002846FFF7E9FE40B997F8B43113B901236C
:105C900087F8B431204B01225A70022385F838303E
:105CA0002B6C002285F8282063B1284698470124F0
:105CB000204602B0BDE8F0876B68C3F34F28A0E729
:105CC00002248DE701248BE7019B4FF020324FF037
:105CD0002E0E4FF0100C1A605A6083F800E0C3F8E3
:105CE00007206C6A1A625A6283F80BC0C3F8272037
:105CF00083F820E083F821E0EA6B5C835A8724FA7A
:105D00000CF422FA0CF29C8283F82BC09A869DE751
:105D1000002465E7BC5A0020BC4A00202DE9F04170
:105D2000B1F904300F2B82B00E460446174635D029
:105D30002046FFF715FA94F91B80B8F1FF3F3ED0DB
:105D4000554B41F2180203EB08118A58904211D1C9
:105D5000183303EB4825B38801331BB205EB431519
:105D6000B38020463D60FFF7FBF93060012002B0B0
:105D7000BDE8F08103F5805292F8B41100296AD091
:105D800001225A702278022A69D02369002B50D14F
:105D9000002301203B6002B0BDE8F0814FF40071A8
:105DA000FFF75AFE002852D04FF6FF73B38020460B
:105DB000FFF7D6F994F91B80B8F1FF3FC0D12278E4
:105DC000022A54D02369002BDDD0334909780329F6
:105DD0000EBF32499BB24FF6F7718B4294BF00233E
:105DE0000123002BCFD138B92D4A92F8B431002BC2
:105DF0004ED0294B01225A700023112201A9FFF72E
:105E0000D1F9012842D1019D264BEB1A48BF03F27C
:105E1000FF13B3F5805F4FEA632230D3204A92F834
:105E2000B43113B9012382F8B4311B4B01225A70EB
:105E300027E0194A1278032A0EBF184A9BB24FF680
:105E4000F772934294BF00230123002BA0D10020BE
:105E500002B0BDE8F081012182F8B41190E7104A48
:105E60006368D2F82022B3EB422F91D2EFE70C4ABD
:105E70006368D2F82012B3EB412FB4D3F1E74FFAA5
:105E800082F884F81B80002D7FF465AF22787AE7D2
:105E9000012382F8B431ACE7BC4A0020F7FFFF0FC2
:105EA000BC5A0020D44A00202DE9F04790F8303049
:105EB00086B00446042B54D8DFE813F005000E002A
:105EC0005600F8004F00C44869F05AFA4FF6FF72C6
:105ED0000123228484F83030DFF8FC8204F11C05B1
:105EE00001AE04F13109324629464046FFF716FF5C
:105EF000012800F00281022833D1B84901F580550C
:105F000095F9D221531C0AD002F5817201EB0212DD
:105F1000D3796FF30003D371FF2385F8D23195F95C
:105F2000D3315F1C16D003F5817301EB031201EB33
:105F30000313D279D979C2F34502012A86BF02F14F
:105F4000FF3202F03F02002262F34601FF22D971C4
:105F500085F8D321042384F830300020E36A2070D0
:105F6000984706B0BDE8F0879D4D95F8E031002BCD
:105F7000F7D1994F04F11C0901AE4FF009083246E0
:105F800049463846FFF7CAFE012840F021810198B2
:105F9000002800F0FD800378E52B01D0002BEED126
:105FA000904A821A48BF02F2FF12B2F5805F4FEAB0
:105FB000622380F05C8189491B018B4A13449A7BE0
:105FC000042A0CD0D5F898200132C5F898205A60E0
:105FD00004229A73D5F89C300133C5F89C3095F9AA
:105FE000D2315E1C0AD003F5817301EB0313FF224B
:105FF00085F8D221DA796FF30002DA7195F9D3319D
:106000005A1C18D003F5817301EB031201EB031343
:10601000D279C2F34502012A4FF0FF0188BF02F195
:10602000FF3285F8D311D9798CBF02F03F020022EC
:1060300062F34601D9712022002172F02FFE019BEC
:10604000D4F83120D4F8351059601A60B4F83920EA
:1060500094F83B1099721A81019B627EDA7203A850
:1060600003F008F8002800F0E5809DF80E509DF838
:106070000F10BDF80C00019B9DF8102041EA45115E
:10608000A0F2BC7041EA40218DB219829DF8111036
:10609000D20242EA41129DF8121042EA510290B235
:1060A000DA8103221D83D88284F83020237E98066B
:1060B00008D5E0690023112202A9FFF773F801282F
:1060C0007FF44FAF204669F05BF92369002B00F0A5
:1060D0008D80237E03F0F70213F00403227640F054
:1060E0009380122A00F0B1800022E36A84F828200D
:1060F0002046984706B0BDE8F087019F002F00F0CA
:10610000C2803B78002B00F0BE8097F80BA01AF0FD
:10611000080F7FF4E8AE0B224946384672F058FD6E
:1061200000287FF4E0AE637E8AEA0303D90640F1DB
:10613000EB802A4901F5805595F9D2315A1C0AD0D5
:1061400003F5817301EB0313FF2285F8D221DA797D
:1061500060F30002DA7195F9D321571C3FF4FAAECF
:1061600002F5817201EB021301EB0211DB79CA79AE
:10617000C3F34503012B86BF03F1FF3303F03F0355
:10618000002363F34602FF23CA7185F8D331E1E6A9
:1061900095F8B831022B3FF4DDAE95F8E031002BD5
:1061A0007FF4D8AEC5E97D3385F8F03185F8EC3160
:1061B000D5F8CC31C5F8E431D5F8143285F8E08152
:1061C000C5F8E8313846FFF7EDFC01283FF4D7AEBB
:1061D00002283FF4BFAEC4E6745C0020BC4A002035
:1061E000BC5A0020D44A0020D45A0020237E19072C
:1061F0007FF57AAF664B93F89821002A7FF4B1AE11
:10620000072283F898216FE7A568E66A002384F8DF
:10621000283029462046FFF71FFC00286ED194F84D
:106220002830002B7FF49DAE0223C4E90B6584F86F
:10623000283096E6019B6FF07E01472219745A744C
:106240009873D87344F281752BE7626AE16AA1639F
:10625000042084F82800C4E90B22C4E9023384F83E
:106260003C3063636362204669F08AF879E695F80A
:10627000B43113B9012385F8B431464901234B7079
:106280006FF00F0399E6434901F5805595F9D23136
:106290005F1C0AD003F5817301EB0313DA796FF306
:1062A0000002DA71FF2385F8D23195F9D3315E1CF3
:1062B00016D003F5817301EB031201EB0313D279BE
:1062C000D979C2F34502012A86BF02F1FF3202F0FA
:1062D0003F02002262F34601FF22D97185F8D321E3
:1062E000237ED8067FF536AE2B4869F049F84FF685
:1062F000FF720223228484F8303036E6002E3FF409
:1063000030AE2046B0472CE6BA8A7B8B204D43EA5C
:1063100002436362D5F81022FB69A3605202B3FB0B
:10632000F2F102FB113109B113445B1AE36084F806
:1063300019A095F9D23117495E1C0AD003F5817373
:1063400001EB0313DA796FF30002DA71FF2385F8AA
:10635000D23195F9D321501C16D002F5817201EB90
:10636000021301EB0211DB79CA79C3F34503012B58
:1063700086BF03F1FF3303F03F03002363F34602BC
:10638000FF23CA7185F8D331032384F830308DE6BA
:10639000BC5A0020BC4A0020745C002010B5037871
:1063A00090F818C0023B012B044602D91CF0060FDE
:1063B0006AD11CF0200F44D194F91A30591C0AD02C
:1063C000384A03F5817302EB0313FF21DA796FF387
:1063D0000002DA71A17694F91B305A1C16D03149AB
:1063E00003F5817301EB031201EB0313D279D97921
:1063F000C2F34502012A86BF02F1FF3202F03F02DA
:10640000002262F34601FF22D971E2761CF0080FE8
:106410000ED0254B93F89821072A06D093F8B42183
:10642000002A3BD01F4A01215170002283F8982195
:10643000E26A0023237084F8283022B3BDE81040BC
:10644000104700231949E0691A018A58904206D082
:106450000133082BB0D01A018A589042F8D1114963
:1064600003F5817301EB0312D279C2F34502012ACD
:1064700012D9013A02F03F0201EB0313D97962F31A
:106480004601D97198E710BD0121FFF731F90128C4
:10649000F9D194F818C08CE70022EDE7012283F8C7
:1064A000B421BFE7BC4A0020BC5A0020D45A0020C7
:1064B0004FF0FF302DE9F041344A354D04460023BA
:1064C00004E00133082B02F1100216D011780429E0
:1064D000F7D103F5817105EB0111C979CF07F0D42C
:1064E000661C52F80A1C01D08142EAD21C460133D4
:1064F000082B084602F11002E8D1631C02D10120EA
:10650000BDE8F081224DDFF8988004F5817705EB36
:1065100007139988F9B91F4ED8F8683D06EB442156
:1065200023B3D3F80C801C4A41F2180305EB041482
:10653000E0580023C047C8B1022824D106F6E87607
:1065400005EB0715D6F89C300122013BC6F89C30BC
:10655000AA710020D4E7D8F8683D3BB19A6841F2AF
:10656000180005EB041318589047D4E70B4BD3F8E9
:106570009C2005EB07150320013A0121C3F89C205C
:10658000A87183F8A0100020BDE8F081E25A002035
:10659000BC4A0020D44A00205D0E0008BC5A0020EE
:1065A000F01D00202DE9F04F90F82830013B83B01A
:1065B0000446082B0BD8DFE803F0383C1E230529DE
:1065C0000A2E33000121FFF7D5F8012802D003B0CD
:1065D000BDE8F08F2378002284F82820002BF6D025
:1065E000D4E901138B4238BF0B46226CA360032110
:1065F00084F82810E262204603B0BDE8F04FCDE6F3
:10660000002103B0BDE8F04FFFF7B4B803B0BDE818
:10661000F04FFFF7BBB903B0BDE8F04FFFF74CB93F
:1066200003B0BDE8F04FFFF7BDBA03B0BDE8F04FCF
:106630003AE4534F4368D7F81852016BD7F8102249
:106640001D406818B0EB422F4FEA42269C46C0F02E
:10665000938094F800E0DFF82C91A7F5805A4FF66C
:10666000F778BEF1020F14D02069002857D1D4F872
:1066700004C0A368E26A634538BF63460021A36093
:1066800084F82810002AA2D0204603B0BDE8F04FBD
:106690001047D4F804C0D7F82022BCEB422FE8D230
:1066A0002069227E12072CD5D7F8942100F1010C25
:1066B000624522D297F8B42122B9012387F8B43178
:1066C0006368216B01228AF8012094F800E0891B9D
:1066D000294433445B1B8E42C4E904C063602163D8
:1066E0009C464FF00005BCD9BEF1020F3ED0206998
:1066F0000028BED0DFF890B01FE0E8D14FF0000CCA
:10670000E5E701A968F08CFA01287FF460AF206901
:10671000DDF804C094F800E06368216BD7E79AF8CD
:106720000020032AD3461AD082B2424594BF0022E9
:106730000122002AB5D0D4F804C09BF80030032B06
:106740000EBF104B80B24FF6F773984294BF0020F3
:10675000012000288DD18C44C4F804C089E7484545
:1067600094BF00220122002A9BD0E4E7D7F8202220
:10677000B3EB422FEFD37CE794F800E0B4E700BF1F
:10678000BC5A0020F7FFFF0FBC4A002010B5184C80
:1067900018484422002172F081FA237804F58054CD
:1067A0004FF6FF70D4F81C22A4F8D201022B4FF050
:1067B000030118BF03234FF0100C84F8D01104F527
:1067C000DC700021C4F8C82184F8B831C4F8DC2199
:1067D00084F8D1C1FFF740F938B994F8E03123B912
:1067E000C4E97933022284F8E021012010BD00BF02
:1067F000BC4A0020745C002070B51A4D1A4BC5F8D5
:106800009C3B1A4B85F8A81B002683F8186A05F6EE
:106810009C33C0E954330D230446C0F8583140F28C
:106820000113C0F85C6100F5A271A0F844316AF070
:10683000D5FEE378C4F8B4631F22C4F8B023012264
:1068400005F599659342C4F8A853A4F89C2308BFA2
:10685000C4F8AC5304F567712046BDE870406AF097
:10686000BDBE00BFE82E002055534253F01D00204E
:10687000F0B50B7813F0600683B00C46054633D0B4
:10688000202E2DD14A78FE2A6BD0FF2A63D14A8868
:10689000002A40F08B80CA88002A40F087801906C1
:1068A00000F184806148624B80F8182AC5F8B4234F
:1068B000EA78012183F8E814A5F89C1303F599639D
:1068C0001F21012AC5F8B013C5F8A83305F5677173
:1068D00008BFC5F8AC3328466AF080FE002600E009
:1068E0000026304603B0F0BD4B780A2B6AD00B2B44
:1068F00063D0012BF5D18B88D9B21B0676D40196D3
:10690000019BC06843F010030193019B036103697D
:106910000193484B03E002690192013B02D0019AC6
:10692000D206F8D42846424F6AF048FD0223217966
:10693000402228466AF074FD97F8E834022B6DD0A7
:1069400094F90420002ACCDA012BCAD00121284670
:10695000FFF752FFC5E768F08DF90226304603B015
:10696000F0BD4E8816BBCC88012C1FD118061DD552
:106970002F4FD7F800359B699847C0B287F8AC0B0A
:10698000A0B1022307F6AC3785F811314FF48073BC
:10699000C5E94E44C5E94A77C5E94C46A5F81C311E
:1069A00005F58E7128466AF0ABFD9AE7284668F037
:1069B00061F90226304603B0F0BD1D4B4A8883F8CA
:1069C000AD2B8EE7022280F811214FF48072A0F8DF
:1069D0001C21194A0123C0E94E33C0E94A22C0E90B
:1069E0004C3600F58E716AF08BFD7AE70096009BBD
:1069F000C06843F020030093009B61F38A13009367
:106A0000009B0361036900930A4B03E00269009253
:106A1000013B87D0009A9706F8D483E78121284666
:106A200068F060F9002387F8E8345AE7F01D002089
:106A3000E82E0020400D0300953A002010B50D4BC4
:106A400093F8183A022B07D0033B012B02D8002100
:106A5000FFF7D2FE002010BD074B93F8D514044673
:106A60006AF06EFE0028F5DA01212046FFF7C4FE29
:106A7000F0E700BFF01D0020E82E0020F8B5404EE2
:106A800096F8185A074655B1012D06D13D4B93F89B
:106A9000D5146AF055FE002832DB0020F8BD394CD1
:106AA000B0F8B433D4F8CC24C4F8A02B1F2BD4F8FE
:106AB000D024C4F8A42B08D1334BD4F8C8249A426C
:106AC00003D194F8D51401291FD994F8AE3B04EBF7
:106AD000C3020133DBB2042B4FF0050108BF0023D2
:106AE00082F8B01B4FF4005184F8AE3B38460223C5
:106AF000C2F8B41B84F8E834FBF78CF90020F8BD29
:106B000029463846FFF778FEC7E794F8D634013BAC
:106B10000F2BDAD86AF014FE002827DB96F8183A13
:106B2000013B022BB9D9B4F8D03B1BB3042286F841
:106B3000182A164AC7F85C51C7E95422D4F8D02461
:106B400084F8A85B934228BF1346D4F8A42BC7F857
:106B5000583140F20111A7F84411D31A07F5A27178
:106B60003846C4F8A43B6AF039FD96E73846FBF78F
:106B700051F992E719463846FFF73EFE8DE700BF10
:106B8000F01D0020E82E002055534243BC3A00205F
:106B900000207047704700BF704700BFD0ED007AFB
:106BA000D0ED036A30EE677AE6EE877AB0EE670AD8
:106BB000C0ED007A704700BFD0ED017AF5EE407A63
:106BC000F1EE10FA09D1DFED0E7A60EEA70AB7EE0A
:106BD000007AC7EE207AC0ED017A31EE277AD0ED47
:106BE000007A80ED021AC1EE076A30EE677AC0EDD6
:106BF000036AE6EE877AB0EE670AC0ED007A704766
:106C0000DB0FC94090ED017AD0ED036AD0ED027A36
:106C100030EE470AA6EE807A90ED000A80ED017A08
:106C200037EE676AE6EE867A37EEC07AC0ED027A12
:106C3000A6EE870A80ED000A704700BFD0ED056A16
:106C4000D0ED017A90ED007A90ED066AD0ED025A0F
:106C500090ED035A80ED050A66EEA77AC0ED066A4C
:106C6000E7EE007A90ED077AE5EE867A90ED086A15
:106C7000D0ED045A80ED087AE5EE477AE5EEC67A63
:106C8000B0EE670AC0ED077A704700BFD0ED057A15
:106C900090ED006A90ED037AD0ED025AE6EE007AAC
:106CA000F0EE406AB0EE670A90ED016AD0ED047A2A
:106CB00027EE407A67EEC07AA6EE267AE5EEA67A4F
:106CC00090ED066AC0ED067A36EE077A80ED057A19
:106CD000704700BF03685A1C02601970704700BFFC
:106CE00003685A1C02601970704700BF024B186895
:106CF00003681B68184700BFE05C002000797047FC
:106D00000079C0F34010704700794009704700BF18
:106D100090F83C20034602F0FF0012B1002283F8F5
:106D20003C2070474FF48053838170474FF40063D9
:106D3000838170474FF40063838170474FF4006391
:106D4000838170474FF40063838170474FF4006381
:106D5000838170474FF4006383817047074B10B401
:106D600003F11001002453F8042B824208BF43F8BA
:106D7000044C8B42F7D15DF8044B7047E45C002073
:106D800070B5374C638CA08AB4F92C50B4F92660E6
:106D9000B4F91AC0C01A238C00FB03F3B4F92A001B
:106DA00005EBE335C00290FBF5F000EBE330A0F516
:106DB0007A6EB4F9243020630EFB0EF52D1305FB1B
:106DC00006F605FB03F3B4F91C500EFB0CFC4FEA6E
:106DD000EC2C0EFB05FE1B14B4F918500CEBE62C42
:106DE00003EB6E330CEB850C0233B4F93450A66B15
:106DF000E48B9B1003F500430CFA05FC04FB03F342
:106E00000CF1020C4CF25034A6EBAC0C2C4104FB00
:106E10000CF4002C4FEAD333ABBF6400B4FBF3F3A4
:106E2000B4FBF3F35B0089B11C120E4D04FB04F4B8
:106E300040F6DE3606FB04F403FB05F5241404EBF0
:106E4000254404F6CF6403EB24130B602AB100EB56
:106E500080004000083000111060012070BD00BFAC
:106E6000E05C002043E3FFFF0120704701207047F2
:106E70002DE9F84F6E4DD5F83CC0B5F84000B5F996
:106E80004A90B5F846E0C0EB2C1303FB03F4B5F9C8
:106E90004430241303FB04F44000B5F94230C0EB46
:106EA000EC0003FB00F0A41304EBE024B5F9483038
:106EB000AC650F46A4F5FA31164683FB013281FB1F
:106EC000018C12034FEAE97B42EA13524FEA033A7C
:106ED00009FB0CF308FB0B3BA9FB0839D9441B0A3F
:106EE00043EA096313EB0A0342EB292202F500424D
:106EF000A3FB0E390EFB029E4FEAEE734FEA6E02C1
:106F000053EA6E0E4FF0000000F08580B5F9509006
:106F100009FB0CFEB5F94EC08CFB011C4FEAE97A67
:106F20004FEA4C4C08FB0AEE4CEAD13CA9FB08980E
:106F3000490411EB0901F04448EB0C0C4018E96DD1
:106F4000C1F58019B5F94C1009F0004E4FEAC97827
:106F5000B8EB00080CEBC1014EEA590E6EEB010EC6
:106F600018EB080C4EEB0E011CEB080C4EEB01016C
:106F70004FEA81194FEA8C1049EA9C691CEB000C1E
:106F800041EB0901890041EA9C714FEA8C0C1CEB32
:106F9000080C4EEB01014FEA8C00890010EB080051
:106FA00041EA9C714EEB01016CF05CF8B5F956209A
:106FB000B5F954E0B5F952504FEA6138430B43EA52
:106FC000C14302FB08FC4FEAE27903FB09C9A2FBBB
:106FD000032CCC4402FB08F803FB0C88A2FB032C17
:106FE000C444520E42EACC12121841EB6C6C4FEAC8
:106FF000EE730EFB01F103FB0011AEFB0030014408
:10700000DB0C43EA4133D0184CEBE141000A40EA83
:10701000016000EB05100FB1000A386026B104EBE7
:1070200084048034241234600120BDE8F88F00BF4E
:10703000E05C002031B10A4BD3ED1E7AFDEEE77A19
:10704000C1ED007A52B1064B9FED067AD3ED1F7A5F
:1070500067EE877AFDEEE77AC2ED007A012070478D
:10706000E05C00200000C8422DE9F04F634D85B080
:10707000B5F88E30D5F88000B5F88C8001911B02F0
:10708000B5F88810B5F88A60B5F89040C01A67EB7B
:1070900007074FEA014EA8FB001CB5F8863008FB35
:1070A00007CCC90941EA4C6111EB0E0193464FEA46
:1070B000C332A6FB003E06FB07EE4FEA132343EA6A
:1070C0000E634FEAEC1C4CF1000C9B18A4FB00264D
:1070D00004FB07644FEAD25242EA44224FEA2E2EC2
:1070E0004FEAE4544EF1000E12F5FA6944F100063D
:1070F000B9F5FA6F029476F10004039631DA029C36
:10710000A2FB02A602FB04F806EB48044FEA84083F
:107110004FEA8A0616EB0A0648EA9A7844EB080812
:107120004FEA560A4AEAC87AB608354CB1EB0A016A
:1071300046EA88766CEB680C9B1B039E6EEBA80EF0
:10714000A1454FF0FF3476EB040427DB00FB07F783
:10715000A0FB000202EB4707C00F40EA4700B9EB73
:107160000009019C8CB1D5F89400A0FB033200FB10
:107170000E2E5B0D43EACE235B1A4FEA6E5E6EEB7A
:107180000C0CDB0B43EA4C432360BBF1000F01D036
:10719000CBF80090012005B0BDE8F08F40F6AC566A
:1071A000029C921944F1000402FB04F4A2FB028247
:1071B00002EB4404E6004FEAC802B8EB020246EADA
:1071C000587664EB060651184CEB060C18EB0806D3
:1071D00044EB040A16EB080644EB0A0A4FEA8A0A53
:1071E0004AEA967AB600B6EB08026AEB0404520843
:1071F00042EAC4729B1A6EEB640EA7E7E05C0020C3
:1072000024FAFFFF0120704710B4114B114C1B688A
:10721000D4F898001B1AFA2B0FD811B1D4F8A0306B
:107220000B6032B1D4F8A430136001205DF8044B38
:10723000704701205DF8044B7047074A136800202F
:1072400023F0040384F89C0013605DF8044B70473E
:1072500004280020E05C002000000010064B002203
:107260000021C3F8A820C3F8AC20C3F8B020C3F8AD
:10727000B4100120704700BFE05C0020104B114AA1
:107280001B68D2F8B4105B1AFA2B16D8D2ED2A6A12
:1072900092ED2B7AD2ED2C7AFDEEE66ABDEEC77A3E
:1072A00016EE903AFDEEE77AC38617EE103A0387A2
:1072B00017EE903A4387012070470020704700BFC7
:1072C00004280020E05C0020024BD3F8B8305B6853
:1072D000184700BFE05C0020024BD3F8B8300830FC
:1072E0009B681847E05C0020012070470120704730
:1072F00038B51446002944D0344B9FED356AD3EDA0
:107300002F7AB3F9D42093ED310AB8EEE77AD3EDB2
:10731000367AC7EE066A0D4604EE902AB3F9D020FD
:10732000F8EEE77A05EE902AB3F9D22087EE864A86
:10733000F8EEE44A05EE102AF8EEE55AB3F9CE204D
:10734000D3ED327AB3F9CC30E6EEA45A06EE102A29
:10735000B8EEE77AB8EEC55AB8EEC66AA6EEA57AD8
:10736000A6EE856A07EE903AB8EEC00AF8EEE77A24
:10737000A6EE870AE6EE867AA4EE270A6CF0E4FC15
:1073800028600CB3114BDFED125A93ED367AB3F946
:10739000C220B3F9C0309FED0F0AB8EEC76A07EEFE
:1073A000902A86EE257A06EE903AF8EEE77AF8EE25
:1073B000E66A67EE277AB6EE006AE6EE867A27EE90
:1073C000800A6CF0C1FC2060012038BDE05C002028
:1073D0000000F04A0000C8422DE9F0410446D0E91F
:1073E0000030134483421DD88E188E4217D00D46AC
:1073F00004F10C08002701E0AE4210D023695A1CAA
:107400002261234415F8010B1873042AF4D1414674
:107410002046FBF7B5FBAE42C4E90470EED16069CB
:10742000BDE8F0814FF0FF30FAE700BF70B50446C9
:10743000234894F9103003EB8303154650F82300DA
:10744000A3689A0782B00CD501906AF0C3FC01983A
:1074500029466AF0BFFCA3689B0717D5012002B03C
:1074600070BD636913B11A689B885383154B164A24
:107470001B6856684FEAC30C144BA3FB0C3C4FEA45
:107480009C1C53689B1B9C45FBD2DDE70D4B0E49B2
:107490001A680E4B4FF4FA7000FB02F2A3FB0232A3
:1074A000486892094B681B1A9A42FBD26369002B09
:1074B000D4D01A689B881383012002B070BD00BF2E
:1074C000600D00208C340020001000E0D34D6210CD
:1074D00010B504682379012B84B010D0022B0BD196
:1074E000A368DB074FF0F0024CBFFF217F2120464D
:1074F00004B0BDE8104099E7002004B010BDA268B8
:10750000617C94F9100002F0010201920DF10F026A
:107510000092F024FF228DF80F40FDF7BBF804B075
:1075200010BD00BF10B504682379CA4341EA0211B7
:10753000012B84B0CAB20ED0022B09D1A368DB079D
:107540004CBFD2215221204604B0BDE810406DE767
:10755000002004B010BD8DF80F20A268617C94F962
:10756000100002F001020DF10F04CDE90042D22219
:10757000FDF790F804B010BD10B504682379012B15
:1075800084B010D0022B0BD1A368DB074FF0B402FC
:107590004CBFFF217F21204604B0BDE8104045E7E5
:1075A000002004B010BDA268617C94F9100002F0C4
:1075B000010201920DF10F020092B424FF228DF816
:1075C0000F40FDF767F804B010BD00BF10B50468A8
:1075D0002379012B84B00FD0022B0AD1A368DB07DB
:1075E0000A4620464CBFA521252104B0BDE8104025
:1075F0001CE7002004B010BDA26894F910008DF8BB
:107600000F1002F00102617C0DF10F04CDE9004280
:10761000A522FDF73FF804B010BD00BF10B5046807
:107620002379012B84B010D0022B0BD1A368DB0788
:107630004FF096024CBFFF217F21204604B0BDE8E9
:107640001040F3E6002004B010BDA268617C94F9FC
:10765000100002F0010201920DF10F020092962437
:10766000FF228DF80F40FDF715F804B010BD00BFE4
:1076700010B504682379012B84B00FD0022B0AD1F6
:10768000A368DB070A4620464CBF8721072104B0C8
:10769000BDE81040CAE6002004B010BDA26894F90D
:1076A00010008DF80F1002F00102617C0DF10F0443
:1076B000CDE900428722FCF7EDFF04B010BD00BF0A
:1076C00010B504682379C901012B84B0CAB20AD06D
:1076D000022B05D17821204604B0BDE81040A5E674
:1076E000002004B010BD8DF80F20A268617C94F9D1
:1076F000100002F001020DF10F04CDE900427822E2
:10770000FCF7C8FF04B010BD10B504682379012B45
:1077100084B010D0022B0BD1A368DB074FF05502C9
:107720004CBFA5212521204604B0BDE810407DE6D0
:10773000002004B010BDA268617C94F9100002F032
:10774000010201920DF10F0200925524A5228DF83D
:107750000F40FCF79FFF04B010BD00BF10B50468D8
:107760002379012B84B010D0022B0BD1A368DB0747
:107770004FF02E024CBFF4217421204604B0BDE826
:10778000104053E6002004B010BDA268617C94F95B
:10779000100002F0010201920DF10F0200922E245E
:1077A000F4228DF80F40FCF775FF04B010BD00BF48
:1077B00010B5154B04689A8E237992013432012B4F
:1077C00084B0D2B20ED0022B09D1A368DB074CBF24
:1077D000F4217421204604B0BDE8104026E60020C4
:1077E00004B010BD8DF80F20A268617C94F91000E0
:1077F00002F001020DF10F04CDE90042F422FCF782
:1078000049FF04B010BD00BFE05C002010B5046863
:107810002379012B84B00ED0022B09D1A368DB079A
:107820004FF031024CBFF42174212046FFF7FEFDDA
:10783000012004B010BDA268617C94F9100002F030
:10784000010201920DF10F0200923124F4228DF811
:107850000F40FCF71FFF012004B010BD10B50468F5
:107860002379012B84B00BD0022B06D101225821A1
:10787000204604B0BDE81040D8E5002004B010BD9B
:10788000A26894F91000617C8DF80F3002F00102BB
:1078900001920DF10F0200925822FCF7FBFE04B09A
:1078A00010BD00BF10B504682379012B84B00BD044
:1078B000022B06D101224821204604B0BDE8104029
:1078C000B4E5002004B010BDA26894F91000617CFA
:1078D0008DF80F3002F0010201920DF10F020092BB
:1078E0004822FCF7D7FE04B010BD00BF10B50468F5
:1078F0002379012B84B00BD0022B06D11A46082124
:10790000204604B0BDE8104090E5002004B010BD52
:10791000A268617C94F9100002F0010201920DF15D
:107920000F020092022408228DF80F40FCF7B2FEED
:1079300004B010BD10B504682379012B84B00BD0BE
:10794000022B06D101220821204604B0BDE81040D8
:107950006CE5002004B010BDA26894F91000617CB1
:107960008DF80F3002F0010201920DF10F0200922A
:107970000822FCF78FFE04B010BD00BF2DE9F041D6
:107980000C4E356873691D4011D0DFF82C8001273B
:10799000B5FA85F4C4F11F0408EB840307FA04F474
:1079A000D3F8DC0003689847A5437461F0D1BDE8C3
:1079B000F08100BF003C0140E05C00202DE9F04177
:1079C000684CD4F81C0190B028B1674A0321FBF73A
:1079D00017FAD4F81C01654D0021FBF78DFAD4F895
:1079E0001C61D6F80480D8F8103000211F0B4FEA34
:1079F000132E4B0105EB4110EA5887EA123C8EEA40
:107A000012220CF0030C02F00F025CEA020401F1F6
:107A1000010106D01029ECD10020F06010B0BDE8C3
:107A2000F081017FD8F80020F06019B1204610B035
:107A3000BDE8F081B2F844104D4F6FEA41416FEA62
:107A4000514189B2A2F84410118889B241F08001F5
:107A5000118098F80610B2F820C011F0040F98F8C1
:107A6000051017F801E014BF0421012101FA0EF1FD
:107A700089B21FFA8CFC2CEA010CA2F820C0B2F8E3
:107A800020C01FFA8CFC41EA0C011184118889B2D4
:107A900041F0010111804168364A914236490A6B32
:107AA0001D440CBF42F4001242F480024FF0070C58
:107AB0000A6333463149A5F81CC00322FBF78AFC50
:107AC000F3689868FBF7AEFEF3689868036823F0E4
:107AD00001030360FBF7A6FE002371680693CDE95E
:107AE0000C33CDE90E330A934B79032B06D8DFE82C
:107AF00003F035312D020A6802F140040B7CF16875
:107B000007EB83071E4B88687A680192CDE9024330
:107B10004FF400330B9340F62B4140224FF4804347
:107B20000591049209934FF480624FF4805301A9A8
:107B30000792089367F05AFBF3689A68136801206C
:107B400043F01003136010B0BDE8F0810A6802F141
:107B50003C04D3E70A6802F13804CFE70A6802F16F
:107B60003404CBE7E05C0020009F2400F80A0020EA
:107B7000E8AD07080060024000380240A10200089A
:107B8000A475002010B5114CD4F81C0128B1104A7E
:107B90006421FBF735F9D4F81C010021FBF7ACF99F
:107BA000D4F81C315B681A68B2F844306FEA43437A
:107BB0006FEA53439BB2A2F84430138801219BB271
:107BC0000B43138084F8201110BD00BFE05C00203F
:107BD000009F240010B54FEA511E024400EB8E0CAA
:107BE000624529D901F01F014FF0FF3404FA01F377
:107BF00050F82E100B4093FAA3F3B3FA83F3DBB2E1
:107C0000202B16D10CF104018A4202D817E08A42D7
:107C100012D98C460431DCF8003093FAA3F3B3FA9E
:107C200083F3DBB2202BF2D0ACEB000003EBC000FF
:107C300010BD03EB4E1010BD4FF0FF3010BD2046BD
:107C400010BD00BF30B503694268474D83B00BB922
:107C5000002A63D0D0ED067AC46A013377EE807AC9
:107C60000361631C012BC0ED067AC36246D0D0EDE0
:107C7000075A90ED097A296807EE903A30EE656A66
:107C8000F8EEE76A8A1AC6EE267A81688A4277EEAB
:107C9000A57A30EE670AC0ED087AA6EE007AC0ED4C
:107CA000077A80ED0A7A80ED097A01D803B030BDF9
:107CB000012B4BDD07EE904AF8EEE77A87EE270AB4
:107CC000B5EEC00AF1EE10FA43DBB5EE400AF1EE74
:107CD00010FA41D4F1EEC07AF4EE677AF1EE10FAC0
:107CE00037D690ED057AB4EEE77AF1EE10FA18D5B2
:107CF000037B23B30323037003B030BD2B6881687B
:107D0000DFED1A7A80ED080A9A1A8A4280ED070A96
:107D1000C0ED097ACAD9B0EE670ADBE72A6842608B
:107D200098E7D0ED047AD0ED066AF8EE677A022380
:107D300086EEA77A037080ED067A03B030BD29681D
:107D40004160002203618261C362AFE79FED070AD1
:107D5000C0E7DFED067AC4E701906CF003F9019803
:107D6000F0EE407AB8E700BF0428002000000000D1
:107D700070B52DED028B044682B000F14805034634
:107D80000026B1EC017AD3ED067ADA6A77EE877ACB
:107D90000132012AC3ED067ADA626DD093ED075AFB
:107DA00093ED096A07EE902A77EE455AF8EEE77AE6
:107DB000C5EEA76A76EE857AF0EE466A37EE677A08
:107DC000C3ED087AE5EE876AC3ED077AC3ED0A6A68
:107DD000C3ED096A1833AB42D3D10369394E426807
:107DE0000133036133689B1A8268934240D99FED47
:107DF000368AE36A012B4DDD013B07EE903A94EDA4
:107E00000A7AF8EEE77A87EE270AB5EEC00AF1EEB5
:107E100010FA4DDBB5EE400AF1EE10FA4BD4F1EE5C
:107E2000C07AF4EE677AF1EE10FA41D690ED057A59
:107E3000B4EEE77AF1EE10FA24D41834AC42D8D17B
:107E4000D0ED047AD0ED066A90ED0C7AD0ED125A9E
:107E5000F8EE677A022386EEA76A0370C7EE276AF8
:107E600085EEA77A80ED066AC0ED0C6A80ED127A85
:107E700002B0BDEC028B70BD83ED087A83ED077A0A
:107E80005E62A7E7037B43B10323037002B0BDEC3E
:107E9000028B70BDB0EE480AC1E700223168416034
:107EA00003618261C362026343648264C365DFE786
:107EB000F0EE487ABAE701906CF054F80198F0EED1
:107EC000407AAEE70428002000000000F0EEC07AFF
:107ED000B0EEE07AB4EEE77AF1EE10FAD4BFB0EE8D
:107EE000676AB0EE476AB5EE406AF1EE10FA48D024
:107EF000B4EEE77AF1EE10FA54BFF0EE675AF0EE06
:107F0000475AC5EE866ADFED202ADFED203ADFED25
:107F1000204A9FED205A9FED203A9FED204A9FED89
:107F2000206AE6EEA23AA6EE834AE6EEA34AF7EE10
:107F3000005AA6EEA45AE6EE845AA6EE856AB1EE81
:107F4000466AC6EE256AB4EEE77AF1EE10FA48BF4B
:107F5000DFED147AF5EEC00A48BF77EEE66AF1EE7F
:107F600010FA48BFDFED107AB5EEC00A48BF77EED1
:107F7000E66AF1EE10FA48BFF1EE666AB0EE660A04
:107F80007047DFED0A6ADEE739094E3DE3B59EBE74
:107F900088FA16BE45FE7FBF99FB243F69A2163EB4
:107FA000A7DFA8B4DB0FC93FDB0F4940A7DFA83428
:107FB00091ED007AD0ED047AD0ED055A90ED064AA5
:107FC000D0ED074A90ED085A90ED096AD0ED0A6AA3
:107FD000E7EE077AF7EE003AC0ED047A91ED007A09
:107FE000D1ED017AE7EE275A90ED0B7AC0ED055AF4
:107FF000D1ED025A91ED003AD0ED0C7AA3EE254A6C
:1080000080ED064AD1ED005A74EEA54AC0ED074A4C
:10801000D1ED014AD1ED005AA4EEA55A80ED085ADF
:1080200091ED015AA5EE056A80ED096AD1ED015A7C
:1080300091ED026AE5EE866AC0ED0A6AD1ED016A49
:1080400037EE267A80ED0B7AD1ED026A91ED007A57
:10805000E6EE877AC0ED0C7A91ED026AD1ED016A05
:10806000D0ED0D7A90ED0E7A90ED0F4AD0ED104ADA
:1080700090ED115AD0ED135AE6EE267A75EEA35A1A
:10808000C0ED0D7AD1ED026AD0ED127A90ED006A62
:10809000A6EEA67AD0ED016A80ED0E7A91ED027A15
:1080A00034EE074A90ED027A80ED0F4A91ED004AD6
:1080B00074EE844AC0ED104AD1ED014A35EE245ADF
:1080C00080ED115A91ED025AC0ED135A77EE857A80
:1080D000C0ED127AD1ED017AD1ED005A91ED025A3C
:1080E00067EEA77AE5EEA57AE5EE057AA5EEA76A32
:1080F00080ED006A91ED016AE6EE276AC0ED016A43
:10810000D1ED026AA6EEA77A80ED027A90ED037AAD
:1081100077EE277AC0ED037A704700BF2DE9F04F64
:1081200089B0CDE9011200F11009834600F1300851
:10813000CE4607464E46054684460024CDF80C90B0
:108140006246284684B1D2ED007A01463B46894614
:10815000F3EC016A99ED007AE6EEC77A634501F126
:108160001001C2ED007AF2D10432724500F1040030
:10817000E8D1032C04F1010A30D062463046ABEB63
:1081800005099CB1D2ED047A009409EB000329465D
:108190000C46F3EC016A94ED007AE6EEC77A83426E
:1081A00001F11001C2ED047AF2D1009CD2ED046A13
:1081B00016ED047AC6EE877A1032424500F11000BF
:1081C000C2ED007ADDD10CF1140C08F1040804357D
:1081D00014360EF1100E10375446B1E7DDE90229CE
:1081E000002500230135059306930793042D52F8CB
:1081F000043B049305A80BF1140418D0F2EC017AA7
:1082000004A9C0ED007A4B46B1EC017AF3EC016AA7
:10821000E6EEC77AA342C0ED007AF5D10135042D10
:1082200009F1100900F1040004F11404E6D1019AE7
:1082300008AE76ED017A022510320BF14004022DD2
:108240002046A2F1040142ED017A20D02346F3EC4E
:10825000016AB2EC017AE6EEC77A9842C1ED007A83
:10826000F5D154ED016A87EEA67A6B1C81ED007A98
:1082700014D076ED017A013D0A46022DA4F11404D2
:10828000A0F11000A2F1040142ED017ADED154ED1B
:10829000016A87EEA67A02ED017AEAE709B0BDE845
:1082A000F08F00BF10B584B00C460246694610300E
:1082B000FFF734FFDDED007A9DED017ADDED026A16
:1082C000B6EE006A67EE867A27EE067A66EE866A72
:1082D000F4EE677AF1EE10FAC4ED007A84ED017ADB
:1082E000C4ED026A0DD6B4EE477AF1EE10FA13D659
:1082F000F4EE666AF1EE10FA78BF012016D604B0EB
:1083000010BD9FED106AF0EEE77AF4EE467AF1EEDA
:1083100010FAE8DD0020F2E7DFED0A7AB0EEC77A66
:10832000B4EE677AF1EE10FAE2DDF3E7DFED057AFD
:10833000F0EEE66AF4EE676AF1EE10FAD4BF0120BF
:108340000020DCE7FFFF7F7FDFED257AB4EEE70A50
:10835000F1EE10FA08DD9FED237A30EE470AB4EE15
:10836000E70AF1EE10FAF8DCDFED1F7AB4EEE70A67
:10837000F1EE10FA08D59FED1B7A30EE070AB4EE45
:10838000E70AF1EE10FAF8D4DFED187AB4EEE70A56
:10839000F1EE10FA18DD30EE670A37EEC00A60EE33
:1083A000007A9FED137A9FED136ADFED136AA7EE53
:1083B000876A9FED127AE7EE866A60EE275AA7EE8B
:1083C000A67AA5EE870A70479FED0D7AB4EEC70A2C
:1083D000F1EE10FA44BF30EE270A37EE400ADEE72E
:1083E000DB0F4940DB0FC940DB0F49C0DB0FC93F42
:1083F0009A7C2E36FAAF4FB93587083CA4AA2ABE1C
:10840000DB0FC9BF10B53E4CB4FBF2F4A1420DD353
:1084100000234FF07E52026043608360C3600361BB
:108420000023836143610362C36110BD07EE902A9C
:10843000B8EE677ADFED337A27EE277AB7EE006A77
:10844000C6EE076A07EE901A9FED2F7AF8EE677A6C
:10845000B0EE405A67EE877AC7EEA64AFDEEE47AA0
:1084600017EE902A2032402A47D8B0EE640AFFF770
:108470006BFFB0EE404A9FED250A34EE800AFDEE18
:10848000C07A17EE902A2032402A31D8FFF75CFFDD
:10849000F8EE006A60EE266A012B24D0F7EE007A2F
:1084A00037EEC00AF6EE005A60EE255A35EE055A50
:1084B000B7EE007A84EE056A76EE077A37EE467AF2
:1084C00080EE275A85EEA76AC6EEA75AC7EE276A3E
:1084D00080ED006A80ED015A80ED026AC0ED035A1A
:1084E000C0ED046A9CE7B0EE660AF7EE005ADDE7DD
:1084F000DFED076A9FED070ACEE79FED064ABAE770
:1085000020A10700BD378635DB0FC940DB0FC93F0F
:108510000000008000000000DFED077A30EE270A3F
:10852000FDEEC07A17EE903A2033402B00D80BE7CF
:108530009FED020A704700BFDB0FC93F000000003B
:1085400091ED005A9FED520A35EE000A08B5FDEE96
:10855000C07A17EE903A2033402B7DD8FFF7F4FE17
:10856000FDEEC57AB0EE403A17EE903A2033402B3C
:108570007BD8B0EE450AFFF7E7FEB0EE405AF1EEC9
:10858000402A91ED014A9FED420A34EE000AFDEEC9
:10859000C07A17EE903A2033402B74D8FFF7D4FE00
:1085A000F0EE404AB1EE402AFDEEC47A17EE903A62
:1085B0002033402B64D8B0EE440AFFF7C5FEB0EE7E
:1085C000404AD1ED021A9FED320A31EE800AFDEEEB
:1085D000C07A17EE903A2033402B4ED8FFF7B4FE06
:1085E000F0EE403AFDEEE17A17EE903A2033402B60
:1085F00040D8B0EE610AFFF7A7FE63EE836A20EE73
:10860000037A63EE857A20EE055AF0EE475AB0EE13
:10861000666AE7EE845AA5EE446AE7EE047AA6EEAF
:10862000C45A63EEA43A62EEA42A22EE000A64EE73
:10863000834AC0ED003A80ED010A80ED024AC0EDA8
:10864000035A80ED046AC0ED052A80ED065AC0ED9C
:10865000077AC0ED084A08BDFDEEC57A9FED0D3AD8
:1086600017EE903A2033402B83D9DFED0B2A9FED94
:10867000095A86E79FED070ABFE7DFED063AB1E743
:108680009FED044A9DE79FED042ADFED024A8BE748
:10869000DB0FC93F00000000000000802DE9F04F13
:1086A00083B005469DF830400D9E0192002C14BF0A
:1086B0004FF030094FF020091C1E88464ADB16F89F
:1086C000010B014600286CD0002C65D04FF0000A49
:1086D000324601E0002C34D012F8013B2746013C21
:1086E000002BF7D1BAF1000F3CD1023F002C65D02E
:1086F000BA4645450AF1FF3A4946284601D2019B50
:108700009847BAF1FF3FF4D10D9A107823463C1BED
:1087100001469B4688B14FF0000A01339F1B454537
:1087200006EB070B284601D2019B984716F8011B60
:108730000029F4D1BAF1000F18D1584603B0BDE8B2
:10874000F08FBAF1000F31D0014683460028F4D0F3
:108750002346E2E716F8010B634258B31C464FF07C
:10876000010AB5E7014683460028D6D1002C04F162
:10877000FF36E2DD3446454506F1FF3649462846D8
:1087800001D2019B9847731CF5D10BF1010BA34457
:10879000584603B0BDE8F08F2346A2464FF0FF34A1
:1087A000BBE7671EA346002CA2D1C6E723464FF0C5
:1087B000FF34ADE7E64383463446DCE723463C46D8
:1087C000A6E700BF0FB430B583B006AB0A4C53F830
:1087D000042B0193D4E9CF0169F03EFB05462068E4
:1087E00003685B6998470028F9D0284603B0BDE8C4
:1087F000304004B0704700BFE05C00200EB410B5FC
:1088000083B005AB044653F8042B0749009301A835
:10881000019469F021FB019B00221A7003B0BDE8AE
:10882000104003B0704700BFE16C00080CB4F0B515
:108830003C4CD4F84433ADF5277D002B4CD094F854
:108840004C33994240D8384B384A1B68A2FB03127C
:1088500092094FF47A7101FB123306A83449FFF7ED
:10886000CDFF06AB03443349AC9A01930646ADAB4A
:1088700001A8009369F0F0FA019BD4F844530A214F
:108880000246581C01901970019B591C019100214E
:10889000197035B32B681B6A1BB128469847D4F86A
:1088A00044539DF8181049B10DF119042B6828465E
:1088B0001B68984714F8011B0029F7D10DF5277D97
:1088C000BDE8F04002B07047D4F85023012303FA0A
:1088D00000F01042B7D1F1E7D4F84833002BAED105
:1088E000ECE7D4F84873002FE8D0901926AB841C2D
:1088F000FD20CDE9045506A92246ADF81000184622
:108900006EF02EF802220346044402A93846CDE94F
:10891000023436F0F3FC0DF5277DBDE8F04002B0DF
:10892000704700BFE05C002004280020D34D621097
:108930002C4F0808D56C000830B54FF4004087B0C4
:1089400034F0FEFD58B14FF40041044634F022FEED
:10895000022806D1226848F201039A4224D007B0C7
:1089600030BD00234FF46121022294F904008DE808
:108970000E001A464FF4004134F016FE1C4BC3F8AB
:1089800044030028EBD01B4A1B4B1C4C1C481D49C0
:108990000091CDE90332CDE901041B4B1B4A0221B2
:1089A0000020FFF743FFDAE7114C00254FF40040A9
:1089B00084F8E85565F028F80028D0D0D4F854336E
:1089C00083420AD0D4F8303483420BD0D4F80C352B
:1089D00098420AD0C4F84853C1E704F55573C4F867
:1089E0004833D0E704F58663F9E704F20C53F6E761
:1089F000E05C0020504F08085C4F0808684F0808EA
:108A0000744F0808384E08084C4E0808384F0808BC
:108A100038B5184CD4F8EC55033005EB9003B3F59A
:108A2000007F18D804EB810120F00302D1F8F00D8B
:108A3000C4F8EC351044C3F5007304F5BE64C1F806
:108A4000F00D0D4A04EB85049B0004210020FFF784
:108A5000EDFE204638BD00210846084AFFF7E6FE35
:108A6000074AD2F89C30002443F00073C2F89C30CF
:108A7000204638BDE05C00207C4F0808A04F080865
:108A80000000001038B50568EB690446F3B198782A
:108A900000B938BDB3F90A2007EE902AF8EEE77A5C
:108AA0000120C4ED057AB3F90C2007EE902AF8EE08
:108AB000E77AF1EE677AC4ED047AB3F90E3007EE87
:108AC000903AF8EEE77AC4ED067A38BD0921142011
:108AD000FFF79EFF0346E861D9E700BF38B5056898
:108AE000EB690446E3B1987800B938BDB3F90420C6
:108AF00007EE902AF8EEE77A0120C4ED047AB3F984
:108B0000062007EE902AF8EEE77AC4ED057AB3F96D
:108B1000083007EE903AF8EEE77AC4ED067A38BDF1
:108B200009211420FFF774FF0346E861DBE700BF6B
:108B300038B50568EB690446E3B1987800B938BDEB
:108B40009A88D2BA07EE902AF8EEE77A0120C4EDAF
:108B5000047ADA88D2BA07EE902AF8EEE77AC4ED02
:108B6000057A1B89DBBA07EE903AF8EEE77AC4ED96
:108B7000067A38BD09211420FFF74AFF0346E86151
:108B8000DBE700BF38B50468E3690D467BB1987830
:108B900000B938BD5B89094ADBBA82FB0312DB17D7
:108BA000C3EB221303F26D132B80012038BD092182
:108BB0001420FFF72DFF0346E061E8E77978787825
:108BC0002DE9F041944603EB43031CF8068B86B075
:108BD000144602EB430315464FFA88F69CF80070E2
:108BE000A0EB070E821BBEF1000FB8BFCEF1000E46
:108BF000002AB8BF52429645B8BF65460CF1060C34
:108C0000B8BF7EB26345E9D1B0456F88A3F10602D3
:108C100006D0BE46A24216D014F8068FB045F8D151
:108C2000B4F80280CB1BA1EB080C002BB8BF5B4251
:108C3000BCF1000FB8BFCCF1000C6345BE46E9DDC6
:108C400047462546E5E76B7904932B7903932B7808
:108C5000064A0091CDE9013E032103460120FFF7BA
:108C6000E5FD284606B0BDE8F08100BFB04F08081A
:108C70004B1EDBB2062B98BF224A30B598BF02EBE1
:108C80004303214C98BF9D8E04F1580388BF4FF4D5
:108C90008075002808BF1C46A44620893CF8082B94
:108CA00087B04FFA82FE90B12A1AA5EB0E03002A74
:108CB000B8BF5242002BB8BF5B429A42BCBF4FFACA
:108CC00080FE64463CF8080F0028EDD122880F4B47
:108CD0000F4893F878CEA3790593A38804930D4B9E
:108CE000BCF1000F08BF0346A078CDE90015CDE91F
:108CF00002200321084A0120FFF798FD204607B013
:108D000030BD00BFE8AD070800150020E05C002082
:108D1000484E080804640808EC4F080803681A461F
:108D2000591C016012F8021B0260587841EA0020C9
:108D3000704700BF02681146531C036011F802CB54
:108D40000160D31C5178036093781B0443EA01232C
:108D5000111D0160D07843EA0C0343EA00607047BC
:108D600012B370B50446864604E0981B17D114EB85
:108D70000C0C15D01EF8013BA3F14100192811F885
:108D8000010BA0F1410598BF2033192DA2EB0E0C69
:108D900000F12006E9D91B1A04D10028E7D170BDE3
:108DA000604670BD184670BD1046704710B402880A
:108DB000C378184CA2F5FA6202F0030140F2B55CE8
:108DC0009208013B0CFB0233827801EB4101013A2E
:108DD00002EB810204EB42010279B1F8444041798F
:108DE000234403EB430302EBC30384790A4A00895B
:108DF000C3EB031301EB8303C3EB0313224402EB26
:108E0000830200214FF47A73C2FB03015DF8044B27
:108E1000704700BFE8AD070880436D382DE9F04189
:108E200017461E4605464FF47A72002338463146EF
:108E30006AF018F94449454A014482FB0143C817C6
:108E40000B44C0EB631382FB03021A44D817404C57
:108E5000C0EB621284FB02044FEAE27C3D48CCEB9B
:108E6000A40C80FB0C404FEAEC74C4EBE010C3EBA5
:108E70000314A1EB8401A971C2EB0211A3EB8103DE
:108E80006B710CEB4C03A2EBC30240F2B55303FB36
:108E900010CCBCF5896F2A714FEA800045DA40F2A8
:108EA000DA239C4548DCBCF5B77FB4BF0022012221
:108EB000294B02EB420103EBC1034FEA4208B3F82E
:108EC0005A3091B2254C08EB020E04EBCE04163456
:108ED0004FF00B0E01E034F8023D634520DDBEF19A
:108EE000010EF8D11C4B424403EBC2024FF0010EBD
:108EF000B2F8443085F802E000F5FA600CF1010C9C
:108F00000844ACEB030C288085F803C04FF47A7258
:108F10000023384631466AF0A5F82A81BDE8F08181
:108F20000EF1010E5FFA8EFEE4E7032140F2965344
:108F30000A464FF00608C5E7022140F229430A46D7
:108F40004FF00408BEE700BF80BC92C789888888BC
:108F5000ABAAAA2A73B06D16E8AD07082CAE0708B5
:108F600030B52E4D84468E460FCD8DB06C460FC465
:108F70000FCD0FC495E80F001CF0030F84E80F001D
:108F80000DD1274B274A03FB0CF3B2EBB30F43D3AE
:108F9000254AB2EB331F2CBF1D241C2400E01C24E7
:108FA0000CF1FF33002B40F26D12194602FB0CF25C
:108FB000B8BF0CF1020102EBA1021C491C4D019447
:108FC00081FB0301DB17A3EB61100244C3EBE11348
:108FD0001A44253285FB02301044D317C3EBA0009E
:108FE000C0EBC000ADF10403101A0DF1040C03EB4B
:108FF0008E0E01E05CF8044F031985FB0320C218B4
:10900000D817C0EBA200C0EBC000E645A3EB000000
:10901000F0D1201A0DB030BD1D24C1E78CAE070879
:10902000295C8FC2285C8F020AD7A3001F85EB51F1
:109030009324499208B50D4BD3F8802ED3F8843E83
:1090400052EA030C09D1002340F2011242808380CE
:10905000837103800381184608BD054909688A1891
:1090600043F10003FFF7DAFE012008BDE05C0020B9
:109070000428002030B5144DD5F8802ED5F8843E54
:1090800052EA030183B0044609D1002040F20113E3
:1090900020806380A080A071208103B030BD0B4987
:1090A00009688A1843F10003FFF7B8FEB5F8883E57
:1090B000ADF8063020460DF10602214665F0FAFCB7
:1090C000012003B030BD00BFE05C00200428002078
:1090D00088422DE9F0414FF001043DD301FB04F437
:1090E000B0FBF4FC8C45F9D23CB3002616E0BCF191
:1090F000090F274698462C4623DD002A14BF4FF05F
:10910000370E4FF0570EF444B94288F800C003F10F
:10911000010306F1010610D8B0FBF5FCB4FBF1F534
:1091200004FB1C00002EE2D1BCF1000FDFDCA142E9
:109130000AD90CF1300C03F801CB00221A70BDE8FB
:10914000F0814FF0300EDEE7B0FBF5FC2C4605FB5E
:109150001C00B5FBF1F5E7E78446C6E790422DE930
:10916000F0410B46044615460AD2B0FBF5F6134A09
:1091700005FB16441846135D00F8013BBDE8F0817D
:10918000B0FBF2F69642B6FBF2F706D20B4A05FBAD
:109190001767D15D03F8011BEAE7BA42B7FBF2F8A3
:1091A00007D9064A05FB187812F8081003F8011BC6
:1091B000EDE74046FFF7D2FF0346F2E738500808D4
:1091C000B5EEC00ADFED347AF1EE10FACCBF30EE26
:1091D000270A30EE670ADFED317A20EE270A70B5F4
:1091E000FDEEC07A86B017EE904A054684EAE47038
:1091F000002303A9A0EBE470CDE90033029366F0ED
:1092000045F8002CACBF20232D2303A88DF8003097
:1092100069F060F801286E4628D0022832D0032871
:109220001CD003A9304670F089FC304669F052F832
:109230000338C4B22246314628466DF091FB002324
:109240002B55284669F046F82E232B54013031194E
:10925000284470F08FFC284606B070BD302303A967
:1092600030468DF8013070F069FCDEE7302303A949
:1092700030468DF801308DF802308DF8033070F0F3
:109280005DFCD2E7302303A930468DF801308DF81C
:10929000023070F053FCC8E76F12033A00007A44C2
:1092A0000278202A034600F10100F9D0092AF7D0FC
:1092B0002D2A29D02B2A03BF5A78B7EE000A03467D
:1092C000B7EE000AA2F13001C8B20928DFED4C7AEE
:1092D00010D8F2EE046A07EE101AB8EEC77A13F847
:1092E000012FA7EEA67AA2F13001C8B20928F0EE4C
:1092F000477AF0D92E2A49D0197801F0DF014529A3
:1093000007D020EE270A70475A78BFEE000A0346BE
:10931000D8E710B459782D2962D02B2954D0A1F167
:109320003002092A03F1010355D80024002202EB80
:10933000820201EB420213F8011FA1F1300009285B
:10934000A2F13002F3D9B2F59A7F134628BF4FF449
:109350009A73072A50D9DFED2B6A1A46B7EE007AC6
:10936000083A072A27EE267AFAD803F007032BB12A
:10937000F2EE046A013B27EE267AFBD16CB3C7EE0E
:10938000877A5DF8044B20EE270A70475978A1F1DF
:109390003002D0B2092803F10103AED8F2EE046A1C
:1093A000F0EE665A07EE102AB8EEC77A13F8011FDE
:1093B00087EE266AA1F13002D0B2092866EEA56ACE
:1093C00077EE867AEED998E79978A1F13002092AEA
:1093D00003F10203A9D9B7EE007A67EE877AD0E7E6
:1093E0009978A1F13002092A03F1020388BFB7EE90
:1093F000007AC4D8012499E7B7EE007AB7E700BF36
:109400000000000020BCBE4C00B50378202B0146B4
:1094100000F10100F9D0092BF7D02D2B03BF4B78B9
:109420004FF0FF3E01464FF0010E0022A3F1300C39
:109430005FFA8CF3092B03D90EFB02F05DF804FBF5
:1094400002EB820211F8013F0CEB4202EEE700BF93
:10945000F0B5384D2B78082141F221008B4002E015
:10946000013993B209D013F4004F4FEA4302F7D009
:1094700080EA430301399BB2F5D1B5F80120002AF7
:1094800055D0DFF8C0C02C4EB4452DD2ACF1060C3F
:109490000CEB0204B44227D2052A41F2210022D962
:1094A000A44514D00CF1FF3C04F1FF3E1CF8011F51
:1094B000082283EA012313F4004F80EA43010ABF24
:1094C0005B008BB29BB2013AF5D1E645EED1228822
:1094D00062B1A11DB14206D2A118B142A44602D286
:1094E000052A0C46DCD800210846F0BDA71C2646FC
:1094F00041F2210016F8011B082283EA012313F42C
:10950000004F80EA43010ABF5B008BB29BB2013A75
:10951000F5D1B742EED16188084AC91AB1FA81F192
:10952000231D49095B1BA2F88C3E0846F0BD044F81
:10953000BC1EDCE700000E0800001008E05C002004
:1095400003000E0807000E082DE9F04F9B4B9C4AC4
:109550008FB09A1ACDE9013203230393984B0793F6
:10956000029B0993019B08930023CDE90A33CDE9BF
:109570000C33944A1369002BC0F2A181914B92499C
:10958000F322DA6000220C92019A01238A428DF8BC
:109590003430C0F08C810B937E238DF82830082264
:1095A0004FF4FC4341F2210103E05B00013A9BB21E
:1095B00006D01804F9D581EA4303013A9BB2F8D1E9
:1095C000824AADF81230824B934280F08E8103F1D3
:1095D000140801997A4B41F2210538F8120C38F839
:1095E000142CC0F30B06B41DADF81440C2F30B04E9
:1095F000120B8DF8182000270204ADF816408DF8E4
:1096000019705DD406338B4200F251810DF11409BB
:109610000DF11A0A4C4601E0A24513D00B9B14F839
:10962000011B03F138026A440133042B02F8101CB9
:109630000B93F1D10AA907A8F9F7A2FAA245CDE93F
:109640000B70EBD10C9B002BC0F23181BDF81240A6
:1096500019F8013B84EA0324082327044CBF85EA58
:1096600044046400013BA4B2F7D1CA45F0D158F8D4
:10967000101C324607A8FDF7AFFE0028C0F2178184
:1096800058F8102C91198A4210D0013A013912F879
:10969000013F84EA0324082320044CBF85EA4404E4
:1096A0006400013BA4B2F7D19142F0D1474BADF831
:1096B0001240984574D2DDE9073108F114088CE7AF
:1096C000B946CDF8008009F1010906335FFA89F93E
:1096D0008B428DF8199000F2EA800DF1140A0DF119
:1096E0001A0BD046002401E0C34513D00B9B18F899
:1096F000011B03F138026A440133042B02F8101CE9
:109700000B93F1D10AA907A8F9F73AFAC345CDE9B5
:109710000B40EBD10C9B002BC0F2C980BDF812406E
:109720001AF8013B84EA0324082322044CBF85EA8B
:1097300044046400013BA4B2F7D1D345F0D1009BAF
:1097400053F8102C02EB070A5146324607A8FDF7E2
:1097500043FE0028C0F2AB800AEB06018A4511D017
:109760000AF1FF32013912F8013F84EA0324082389
:1097700020044CBF85EA44046400013BA4B2F7D145
:109780008A42F0D1B9F1030FADF81240374402D04C
:10979000DDE9073197E7DDF800800C4B98458AD367
:1097A000DDE90731023300229942ADF814207ED35F
:1097B0000DF115040DF1160516460FE00000100816
:1097C00000000E08003C024001000E0834CE0808DC
:1097D000F8C80808A54213D014F8012B0B9B03F11D
:1097E000380169440133042B01F8102C0B93F1D19B
:1097F0000AA907A8F9F7C4F9A542CDE90B60EBD196
:109800000C9B002B53DBBDF81230082241F22101E2
:109810001C0454BF5B0081EA4303013A9BB2F7D1B9
:10982000082241F2210118044CBF81EA43035B0086
:10983000013A9BB2F7D1ADF81230079B0899023379
:109840008B4234D814460DF1120505AE01E0B54245
:1098500013D00B9B15F8011B03F138026A44013346
:10986000042B02F8101C0B93F1D10AA907A8F9F7F1
:1098700087F9B542CDE90B40EBD10C98002816DBF7
:109880000B9B13B3079A08991A448A420FD80AA966
:10989000C818C3F1040200216FF000FA0AA907A852
:1098A000F9F76EF9002398420C900B930DDA039BA5
:1098B000013B03937FF452AE052007F033F90F4BC1
:1098C000536003F18833536058E69DF834307BB918
:1098D0000028ECD10A4B1B787E2BEDD1FFF7B8FDA9
:1098E0000028E9D00FB0BDE8F08F0199044B59E78B
:1098F000044A136943F000431361E9E72301674514
:1099000000000E08003C024070B545880B46044636
:10991000C5F30B052A46002118466FF0BFF92169EF
:10992000084A9142034602D3074A914205D319B12E
:10993000BDE870401846084770BD2A46BDE8704033
:109940006DF00EB834CE0808EFD2080810B50379D0
:10995000012B84B08E460ED0022B09D18368DB0721
:1099600058BF01F07F0104B0BDE81040FDF75EBDB7
:10997000002004B010BD144682688DF80F4002F03C
:10998000010201920DF10F020092417C90F910004A
:109990007246FAF77FFE04B010BD00BFF8B578221A
:1099A000044600210068FFF7D1FF052707F05EF8A5
:1099B00005460E4607F05AF8431B61EB0602B3F565
:1099C0007A7F72F10003F5D3013FEFD120682022A6
:1099D0000121FFF7BBFF052707F048F805460E46B3
:1099E00007F044F8431B61EB0602B3F57A7F72F18E
:1099F0000003F5D3013FEFD120683A460221FFF77B
:109A0000A5FF642607F032F804460D4607F02EF84D
:109A1000031B61EB0502B3F57A7F72F10003F5D306
:109A2000013EEFD10120F8BDF8B5072204460A2116
:109A30000068FFF78BFF052707F018F805460E466C
:109A400007F014F8431B61EB0602B3F57A7F72F15D
:109A50000003F5D3013FEFD1206824224121FFF715
:109A600075FF052707F002F805460E4606F0FEFFD3
:109A7000431B61EB0602B3F57A7F72F10003F5D365
:109A8000013FEFD12068C0224221FFF75FFF05268A
:109A900006F0ECFF04460D4606F0E8FF031B61EB01
:109AA0000502B3F57A7F72F10003F5D3013EEFD1E1
:109AB0000120F8BD10B50446002221210068FFF7FF
:109AC00045FF2068FC222021FFF740FF206840224C
:109AD0002421FFF73BFF20680C222321FFF736FFEC
:109AE000206800222221FFF731FF012010BD00BFB6
:109AF000F8B50122074610210068FFF727FF00B9DB
:109B0000F8BD142606F0B2FF04460D4606F0AEFF7F
:109B1000031B61EB0502B3F57A7F72F10003F5D305
:109B2000013EEFD13868A022BDE8F84011210DE7D1
:109B300030B505682B79012B85B0044611D0022B76
:109B40000CD101220B212846FDF770FC30B12068B2
:109B50001D22092105B0BDE83040F7E6002005B020
:109B600030BDAA6895F91000697C8DF80F3002F0BD
:109B7000010201920DF10F0200920B22FAF78AFD09
:109B8000E4E700BF10B50446C06900B110BD09216B
:109B90001420FEF73DFFE06110BD00BF10B5174C6B
:109BA00004EB8000406830B300EB400004EB80031E
:109BB00093F991CEBCF1FF3F1ED093F8990ED0B12E
:109BC00004EB0C0293F8980E92F8E4EE8C23142127
:109BD00003FB0CFC00220CEB000304EB43030139F4
:109BE000B3F8E83E704412FA83F2F4D10448A0FBC3
:109BF0000230C0F30F1010BD002010BDE05C00204B
:109C0000CDCCCCCC30B5032083B00D461446FFF745
:109C1000C5FF01909DB107EE900A9FED0B7AF8EE1B
:109C2000677AF0EE006A67EE877AB8EE047AA7EEFC
:109C3000A67ADFED067A67EE277AC5ED007A0CB1D9
:109C4000034B236003B030BD6740533A00007A44B1
:109C50003313904328B30368124A30B503F13F43EE
:109C600003F57E039B0A054683B00C46D05C65F085
:109C7000E9FAA988009104F00303C4F381028DF886
:109C8000043028688DF80520C4F300136946C4F336
:109C900041148DF806308DF80740F9F759FE03B0EE
:109CA00030BD7047BCAD070870B5114B114CA342D5
:109CB00003D319E00C33A34216D293F805C08C45A8
:109CC000F8D193F804C0844501D00028F2D193F86C
:109CD00007E09645EED11D6895F804E0E645E9D128
:109CE0002E689E42E6D100E00025284670BD00BFE8
:109CF000F0D20808A0D408080379022B00D07047DE
:109D000010B590F91020204882B00831694403242E
:109D10004FF0000C02EB82024FF0010E8DF800C0F4
:109D20008DF801E08DF802308DF8034050F82220C4
:109D300011F8084C15498A4222D0A1F578418A428F
:109D400020D001F580618A4218D1118821F04001AC
:109D5000090403EB8303090C118000EB83001388D3
:109D6000C16823F0380331F824101B041B0C0B438B
:109D7000138013889BB243F04003138002B010BDE0
:109D80006346E2E77346E0E7600D002000300140E3
:109D9000F8B5074600210068FFF7AEFF3868B62225
:109DA0001421FFF7D3FD642606F060FE04460D463D
:109DB00006F05CFE031B61EB0502B3F57A7F72F1DE
:109DC0000003F5D3013EEFD1812210213868FFF75F
:109DD000BDFD06F04BFE04460D4606F047FE031B94
:109DE00061EB0502B3F57A7F72F10003F5D38022AF
:109DF00015213868FFF7AAFD06F038FE04460D4627
:109E000006F034FE031B61EB0502B3F57A7F72F1B5
:109E10000003F5D338680321BDE8F8406CE700BFC4
:109E2000F8B5044600210068FFF766FF2068B622F7
:109E30007E21FFF78BFD642706F018FE05460E46CF
:109E400006F014FE431B61EB0602B3F57A7F72F154
:109E50000003F5D3013FEFD13A4620687C21FFF79C
:109E600075FD642706F002FE05460E4606F0FEFD6F
:109E7000431B61EB0602B3F57A7F72F10003F5D361
:109E8000013FEFD1206804227D21FFF75FFD6427A9
:109E900006F0ECFD05460E4606F0E8FD431B61EBBF
:109EA0000602B3F57A7F72F10003F5D3013FEFD1DB
:109EB0008C2240212068FFF749FD06F0D7FD0546BA
:109EC0000E4606F0D3FD431B61EB0602B3F57A7F25
:109ED00072F10003F5D3022241212068FFF736FD1D
:109EE00006F0C4FD05460E4606F0C0FD431B61EBBF
:109EF0000602B3F57A7F72F10003F5D320680221E0
:109F0000FFF7FAFE4FF40063A381F8BD2DE9F0419D
:109F1000046884B00546B6227E212046FFF716FD70
:109F20004FF0640806F0A2FD06460F4606F09EFDBF
:109F3000831B61EB0701B3F57A7F71F10003F5D361
:109F4000B8F10108EED102212046FFF7D5FE636982
:109F500013B11A689B88538306F088FD06460F46A6
:109F600006F084FD831B61EB0702B3F57A7F72F183
:109F70000003F5D3636913B11A689B8813834FF00C
:109F80000A0806F073FD06460F4606F06FFD831BB8
:109F900061EB0701B3F57A7F71F10003F5D3B8F1F6
:109FA0000108EED142467C212046FFF7CFFC06F0A7
:109FB0005DFD06460F4606F059FD831B61EB070267
:109FC000B3F57A7F72F10003F5D3002259212046C0
:109FD000FFF7BCFC06F04AFD06460F4606F046FDBC
:109FE000831B61EB0702B3F57A7F72F10003F5D3AF
:109FF00094F91030A2688D4903EB83035E20920729
:10A000008DF80F0051F8230040F1E48001230DF199
:10A010000F020021019067F08DFE4FF4A473844A73
:10A020000198002167F086FEA3689B0740F1E58058
:10A030004FF00A0806F01AFD06460F4606F016FD18
:10A04000831B61EB0701B3F57A7F71F10003F5D350
:10A05000B8F10108EED1012259212046FFF776FC24
:10A0600006F004FD06460F4606F000FD831B61EB7B
:10A070000702B3F57A7F72F10003F5D38C224021F9
:10A080002046FFF763FC06F0F1FC06460F4606F09B
:10A09000EDFC831B61EB0702B3F57A7F72F10003DD
:10A0A000F5D3032241212046FFF750FC06F0DEFCE9
:10A0B00006460F4606F0DAFC831B61EB0702B3F598
:10A0C0007A7F72F10003F5D3AA6B5A4E95F83500EA
:10A0D000B6FBF2F2092391B2574AFEF771FD4388AD
:10A0E000B6FBF3F62E640279422142F0C00220460C
:10A0F000FFF72CFC06F0BAFC05460E4606F0B6FC4F
:10A10000431B61EB0602B3F57A7F72F10003F5D3CE
:10A11000082243212046FFF719FC06F0A7FC05465C
:10A120000E4606F0A3FC431B61EB0602B3F57A7FF3
:10A1300072F10003F5D3042258212046FFF706FCF4
:10A1400006F094FC05460E4606F090FC431B61EBBE
:10A150000602B3F57A7F72F10003F5D30A22532188
:10A160002046FFF7F3FB06F081FC05460E4606F09D
:10A170007DFC431B61EB0602B3F57A7F72F10003AD
:10A18000F5D300227C212046FFF7E0FB06F06EFCB1
:10A1900005460E4606F06AFC431B61EB0602B3F56A
:10A1A0007A7F72F10003F5D306227D212046FFF766
:10A1B000CDFB06F05BFC04460D4606F057FC031B86
:10A1C00061EB0502B3F57A7F72F10003F5D304B0B9
:10A1D000BDE8F081636913B11A689B885383174BFC
:10A1E00017491A68174B4E68D200A3FB0232920936
:10A1F0004B689B1B9A42FBD208E7104B10491A6828
:10A20000104B48684FF4FA7606FB02F2A3FB0232C9
:10A2100092094B681B1A9A42FBD26369002B3FF4E8
:10A2200007AF1A689B88138302E700BF600D002008
:10A23000BCAE070840420F0004B007088C34002071
:10A24000001000E0D34D62102DE9F041604A04682F
:10A25000816B604FB7FBF1F10646102389B290F88D
:10A260003500FEF7ADFC00214388B7FBF3F7054648
:10A2700037642046FFF740FD80226B212046FFF720
:10A2800065FB4FF0640806F0F1FB06460F4606F04A
:10A29000EDFB831B61EB0701B3F57A7F71F10003DE
:10A2A000F5D3B8F10108EED1032268212046FFF76B
:10A2B0004DFB4FF0640806F0D9FB06460F4606F04A
:10A2C000D5FB831B61EB0701B3F57A7F71F10003C6
:10A2D000F5D3B8F10108EED101226B212046FFF73A
:10A2E00035FB4FF00F0806F0C1FB06460F4606F09F
:10A2F000BDFB831B61EB0701B3F57A7F71F10003AE
:10A30000F5D3B8F10108EED118221B212046FFF742
:10A310001DFB4FF00F0806F0A9FB06460F4606F09E
:10A32000A5FB831B61EB0701B3F57A7F71F1000395
:10A33000F5D3B8F10108EED118221C212046FFF711
:10A3400005FB4FF00F0806F091FB06460F4606F09E
:10A350008DFB831B61EB0701B3F57A7F71F100037D
:10A36000F5D3B8F10108EED12A791A212046FFF77A
:10A37000EDFA4FF00F0806F079FB06460F4606F09F
:10A3800075FB831B61EB0701B3F57A7F71F1000365
:10A39000F5D3B8F10108EED16A7919212046FFF70B
:10A3A000D5FA642706F062FB05460E4606F05EFB12
:10A3B000431B61EB0602B3F57A7F72F10003F5D31C
:10A3C000013FEFD120460321BDE8F04194E400BFF6
:10A3D0003CB0070840420F002DE9F0416C4A046888
:10A3E000816B6C4FB7FBF1F10646102389B290F8F0
:10A3F0003500FEF7E5FB00214388B7FBF3F7054680
:10A4000037642046FFF778FC80226B212046FFF757
:10A410009DFA4FF0640806F029FB06460F4606F049
:10A4200025FB831B61EB0701B3F57A7F71F1000314
:10A43000F5D3B8F10108EED1072268212046FFF7D5
:10A4400085FA4FF0640806F011FB06460F4606F049
:10A450000DFB831B61EB0701B3F57A7F71F10003FC
:10A46000F5D3B8F10108EED142466B212046FFF743
:10A470006DFA4FF0640806F0F9FA06460F4606F04A
:10A48000F5FA831B61EB0701B3F57A7F71F10003E5
:10A49000F5D3B8F10108EED101226B212046FFF778
:10A4A00055FA4FF00F0806F0E1FA06460F4606F09F
:10A4B000DDFA831B61EB0701B3F57A7F71F10003CD
:10A4C000F5D3B8F10108EED118221B212046FFF781
:10A4D0003DFA4FF00F0806F0C9FA06460F4606F09F
:10A4E000C5FA831B61EB0701B3F57A7F71F10003B5
:10A4F000F5D3B8F10108EED118221C212046FFF750
:10A5000025FA4FF00F0806F0B1FA06460F4606F09E
:10A51000ADFA831B61EB0701B3F57A7F71F100039C
:10A52000F5D3B8F10108EED12A791A212046FFF7B8
:10A530000DFA4FF00F0806F099FA06460F4606F09E
:10A5400095FA831B61EB0701B3F57A7F71F1000384
:10A55000F5D3B8F10108EED16A7919212046FFF749
:10A56000F5F9642706F082FA05460E4606F07EFAF3
:10A57000431B61EB0602B3F57A7F72F10003F5D35A
:10A58000013FEFD120460321BDE8F041FFF7B4BB06
:10A590003CB0070840420F001EE700BFF0B504467C
:10A5A00083B000680021FFF7A7FB0C22252120685B
:10A5B000FFF7CCF90A2226212068FFF7C7F900220D
:10A5C00063212068FFF7C2F9206881222721FFF765
:10A5D000BDF9142706F04AFA05460E4606F046FA7B
:10A5E000431B61EB0602B3F57A7F72F10003F5D3EA
:10A5F000013FEFD10C2225212068FFF7A7F90A229D
:10A6000026212068FFF7A2F90F2263212068FFF7B7
:10A610009DF9206881222721FFF798F90A2706F083
:10A6200025FA05460E4606F021FA431B61EB0602A9
:10A63000B3F57A7F72F10003F5D3013FEFD1032325
:10A6400001AA1021204663F017FD0A2706F00EFA32
:10A6500005460E4606F00AFA431B61EB0602B3F507
:10A660007A7F72F10003F5D3013FEFD19DF804002A
:10A670009DF805109DF806202B4B803080318032EC
:10A68000A3F83801A3F83A11A3F83C2125210C22A4
:10A690002068FFF75BF926210A222068FFF756F9A8
:10A6A0003A4663212068FFF751F92068812227216B
:10A6B000FFF74CF90A2706F0D9F905460E4606F0D1
:10A6C000D5F9431B61EB0602B3F57A7F72F1000303
:10A6D000F5D3013FEFD10DF1030201230221204602
:10A6E00063F0CAFC01230DF103020921204663F047
:10A6F000C3FC20680C222521FFF728F920680A22D4
:10A700002621FFF723F9206812226321FFF71EF9A3
:10A71000812220682721FFF719F920680321FFF71C
:10A72000EBFA012003B0F0BDD86D0020F0B505466E
:10A7300090F91000244C00EB800085B054F8200004
:10A74000AC68A40710D5CDE90223019067F042FB65
:10A75000DDE902230198002167F0ECFAAB689B0762
:10A7600018D5012005B0F0BD6C6914B12668A48825
:10A770007483164C164E246877684FEAC40E154C45
:10A78000A4FB0E4E4FEA9E1E7468A4EB070CE64530
:10A79000FAD2D8E70D4B0E491A680E4B4FF4FA70F7
:10A7A00000FB02F2A3FB0232486892094B681B1AB5
:10A7B0009A42FBD26B69002BD3D01A689B88138313
:10A7C000012005B0F0BD00BF600D00208C340020DA
:10A7D000001000E0D34D621030B50579012D83B033
:10A7E0008E460DD0022D08D18468E40758BF41F091
:10A7F000800103B0BDE8304098E7002003B030BDD1
:10A8000014468268009402F00102417C90F9100025
:10A8100001927246F9F73EFF03B030BDF0B5054630
:10A82000164695F91020244802EB820283B050F8B6
:10A830002200AA6892070FD5CDE9000367F0CAFA93
:10A84000019B00980022314667F074FAAB689B07C1
:10A8500018D5012003B0F0BD6A6912B1146892885E
:10A860006283164A1468164A4FEAC40E154C57689C
:10A87000A4FB0E4E4FEA9E1E5468A4EB070CE6455F
:10A88000FAD2D9E70D4B0E491A680E4B4FF4FA7005
:10A8900000FB02F2A3FB0232486892094B681B1AC4
:10A8A0009A42FBD26B69002BD3D01A689B88138322
:10A8B000012003B0F0BD00BF600D00208C340020EB
:10A8C000001000E0D34D621030B50579012D83B042
:10A8D0008E460DD0022D08D18468E40758BF41F0A0
:10A8E000800103B0BDE8304098E7002003B030BDE0
:10A8F00014468268009402F00102417C90F9100035
:10A9000001927246F9F7FAFE03B030BD2DE9F0432B
:10A91000814A0568816B814CB4FBF1F185B0064634
:10A92000102389B290F83500FEF74AF900214388D8
:10A93000B4FBF3F4074634642846FFF7DDF98022C0
:10A940006B212846FFF702F84FF0960906F08EF8C3
:10A950000446884606F08AF8031B61EB0801B3F54C
:10A960007A7F71F10003F5D3B9F10109EED1032229
:10A9700068212846FEF7EAFF4FF0960906F076F8C0
:10A980000446884606F072F8031B61EB0801B3F534
:10A990007A7F71F10003F5D3B9F10109EED10322F9
:10A9A0006B212846FEF7D2FF06F060F80446884681
:10A9B00006F05CF8031B61EB08010F2B71F100033B
:10A9C000F6D310226A212846FEF7C0FF06F04EF8A3
:10A9D0000446884606F04AF8031B61EB08010F2B7A
:10A9E00071F10003F6D300226C212846FEF7AEFF7A
:10A9F00006F03CF80446884606F038F8031B61EB85
:10AA000008010F2B71F10003F6D37A79192128463A
:10AA1000FEF79CFF06F02AF80446884606F026F862
:10AA2000031B61EB08010F2B71F10003F6D3182211
:10AA30001B212846FEF78AFF06F018F804468846D0
:10AA400006F014F8031B61EB08010F2B71F10003F2
:10AA5000F6D318221C212846FEF778FF06F006F8E8
:10AA60000446884606F002F8031B61EB08010F2B31
:10AA700071F10003F6D33A791A212846FEF766FFF2
:10AA800005F0F4FF07460C4605F0F0FF8C4208BFC6
:10AA90008742F9D003212846FFF72EF930680623B4
:10AAA00002AA4321FFF710FF28B3BDF80810BDF834
:10AAB0000A30BDF80C20C9BA07EE901ADBBAD2BA38
:10AAC000F8EEE76A07EE102A07EE903AB8EEC77A7A
:10AAD000F8EEE77AC6ED076AC6ED087A86ED097AE0
:10AAE000FDEEE77ACDED017A9DF90430013305D012
:10AAF00005B0BDE8F083D6ED087AF1E7D6ED077A28
:10AB0000FDEEE77ACDED017A9DF904300133EFD106
:10AB1000062006F007F800BF3CB0070840420F00CF
:10AB200010B504460068037982B0022B0CBF4321A4
:10AB3000032106236A46FFF7C7FE68B1BDF800107F
:10AB4000BDF80220BDF8043049BA52BA5BBAE186BA
:10AB50006287238702B010BDE086A06302B010BDFB
:10AB60002DE9F047154D95F8413107468A4663B9FE
:10AB70000021386895F8423185F841115246492143
:10AB8000FFF7A2FE0120BDE8F08705F06FFFD5F8C2
:10AB90004841001BC0F5FA54002CE9DD05F066FFC2
:10ABA0004FEAE4790646884605F060FF831B61EBB7
:10ABB0000801A34271EB0903F6D3D9E7D86D002051
:10ABC000F0B5614C0546D4F85001C5F8360094F84C
:10ABD0004031B4F854216A87012B83B00AD0022B8C
:10ABE0002ED003B3002384F8403184F85631184640
:10ABF00003B0F0BD94F84131002B41D1694628469D
:10AC0000FFF7AEFF002851D09DF8003099074DD0D6
:10AC100007220321284664F0F3FC022294F85631FF
:10AC200084F84021E3E728460122022164F0E8FC91
:10AC300094F856310122184684F8402103B0F0BD43
:10AC400094F8413105F1360704F5A87623BB69462F
:10AC50002846FFF785FF9DF8062003460028C1D04F
:10AC60001207BFD4B4F83811BDF8002012FB01F26E
:10AC700036498A4222DBB2F5000F5EDB344A1EE021
:10AC800005F0F4FED4F84831C01AC0F5FA50002897
:10AC9000B4DD94F85631AAE705F0E8FED4F848315F
:10ACA000C01AC0F5FA500028D1DDF2E794F8563109
:10ACB0000022184684F8402103B0F0BD254AB4F8BC
:10ACC0003A11EA86BDF8022012FB01F21F498A42BE
:10ACD00005DBB2F5000F2ADB47F6FF7200E01D4AE4
:10ACE000B4F83C112A87BDF8042012FB01F2174981
:10ACF0008A4204DBB2F5000F12DB154A00E0154A68
:10AD0000D5F83600C4F850016A87BA88B2800021AD
:10AD10000122184684F8401184F8562103B0F0BD92
:10AD2000002AB8BFFF321212524212B2E8E7002ADC
:10AD3000B8BFFF3242F30F22D2E7002AB8BFFF327A
:10AD40001212524212B2BAE7D86D002001FF7FFF03
:10AD50000180FFFF0080FFFFF0B50668F56983B052
:10AD60000446002D65D000232B7004230DEB030255
:10AD70003046FF21FFF7A8FD10B9002003B0F0BD59
:10AD8000206804236A46FF21FFF79EFD0028F4D0C7
:10AD90009DF804108A09023A012AEED99DF805307F
:10ADA00003EB012343F6FF74C3F30D03A342E4D086
:10ADB000002BE2D09DF806109DF8072002EB01223F
:10ADC00040F2FF71B1EB521F4FEA6216D5D0002E50
:10ADD000D3D09DF800C09DF8012002EB0C22C2F3F5
:10ADE0000D02A242C9D0002AC7D09DF802709DF87A
:10ADF000034004EB0724B1EB541F4FEA6417BCD0A7
:10AE0000002FBAD0991A0029B8BF4942FF29B4DCF3
:10AE1000F11B0029B8BF4942FF29AEDC13445B1087
:10AE2000F2195210C5F805300123C5F801202B7026
:10AE3000A4E709211420FDF7EBFDF0610546266823
:10AE400091E700BF10B5044600680179012984B07C
:10AE500028D0022923D1836813F0010F08BF822173
:10AE6000062302AAFFF7DAFCB8B1BDF9083006EEF6
:10AE7000903ABDF90A3007EE103ABDF90C3007EEF2
:10AE8000903AF8EEE66AB8EEC77AF8EEE77AC4EDE3
:10AE9000076A84ED087AC4ED097A04B010BD002079
:10AEA00004B010BD8368417C90F9100003F00103E9
:10AEB000019302AB009302220623F9F71FFC00283E
:10AEC000D3D1EAE730B5044600680379012B85B099
:10AED00014D0022B0FD1826802AD12F0010F18BFFF
:10AEE00003212A4608BF8321FFF798FC18B19DF97A
:10AEF0000930002B10DB002005B030BD8368417C99
:10AF000090F9100003F0010302AD019300950223B4
:10AF10000322F9F7F3FBE9E7206807232A46122109
:10AF2000FFF7D2FC0028E6D09DF90A209DF80930F1
:10AF30009DF90C1043EA022313EB430248BF03328E
:10AF40009DF80B30921043EA012307EE902A13EB91
:10AF50004302F8EEE77A48BF03329DF90E109DF8E0
:10AF60000D30C4ED047A921007EE902A43EA0123D3
:10AF700013EB4303F8EEE77A48BF03339B10C4EDAD
:10AF8000057A07EE903AF8EEE77AC4ED067AB3E771
:10AF900070B50668F46982B00546002C3FD033795D
:10AFA000012B04F1040205D0022B2CD00020A0704C
:10AFB00002B070BDB368717C96F91000009203F086
:10AFC000010301930C231A46F9F798FBA07000289F
:10AFD000EED0B4F9043007EE903AF8EEE77AC5ED1A
:10AFE000077AB4F9063007EE903AF8EEE77AC5ED45
:10AFF000087AB4F9083007EE903AF8EEE77AC5ED32
:10B00000097A02B070BDB36813F0010F4FF00C0362
:10B01000304614BF19468C21FFF700FCD6E7092102
:10B020001420FDF7F5FCF06104462E68B7E700BF79
:10B0300070B50668F46982B00546002C3FD03379BC
:10B04000012B04F1030205D0022B2CD00020A070AC
:10B0500002B070BDB368717C96F91000009203F0E5
:10B06000010301930C220D23F9F748FBA07000287F
:10B07000EED0B4F90A3007EE903AF8EEE77AC5ED73
:10B08000077AB4F90C3007EE903AF8EEE77AC5ED9E
:10B09000087AB4F90E3007EE903AF8EEE77AC5ED8B
:10B0A000097A02B070BDB36813F0010F30464FF05B
:10B0B0000D0314BF0C218C21FFF7B0FBD6E709214B
:10B0C0001420FDF7A5FCF06104462E68B7E700BF29
:10B0D00010B500680379012B84B00C4618D0022B00
:10B0E00013D1836813F0010F14BF2221A22103237F
:10B0F00003AAFFF793FB30B1BDF90D3003EB8303D7
:10B100001B12E633238004B010BD002004B010BD34
:10B110008368417C90F9100003F00103019303ABB5
:10B12000009322220323F9F7E9FA0028E4D1EAE7A1
:10B1300010B5044600680379012B84B02DD0022B92
:10B1400028D1836813F0010F02AA4FF0060314BF41
:10B150001F219F21FFF762FBD0B1BDF80810BDF899
:10B160000A20BDF80C30C9BA07EE901AD2BAF8EE30
:10B17000E76A07EE902ADBBAB8EEE77A07EE903A74
:10B18000F8EEE77AC4ED046A84ED057AC4ED067A38
:10B1900004B010BD002004B010BD8368417C90F95C
:10B1A000100003F00103019302AB00931F2206235A
:10B1B000F9F7A4FAD0E700BF10B504460068037998
:10B1C000012B84B02DD0022B28D1836813F0010FFE
:10B1D00002AA4FF0060314BF2521A521FFF71EFB8D
:10B1E000D0B1BDF80810BDF80A20BDF80C30C9BABE
:10B1F00007EE901AD2BAF8EEE76A07EE902ADBBAA9
:10B20000B8EEE77A07EE903AF8EEE77AC4ED076A0F
:10B2100084ED087AC4ED097A04B010BD002004B0B2
:10B2200010BD8368417C90F9100003F00103019385
:10B2300002AB009325220623F9F760FAD0E700BF9E
:10B2400070B50668F46982B00546002C3FD03379AA
:10B25000012B04F1040205D0022B2CD00020A07099
:10B2600002B070BDB368717C96F91000009203F0D3
:10B27000010301933B220E23F9F740FAA070002846
:10B28000EED0A389DBBA07EE903AF8EEE77AC5ED87
:10B29000077AE389DBBA07EE903AF8EEE77AC5ED74
:10B2A000087A238ADBBA07EE903AF8EEE77AC5ED22
:10B2B000097A02B070BDB36813F0010F30464FF049
:10B2C0000E0314BF3B21BB21FFF7A8FAD6E70921E3
:10B2D0001420FDF79DFB0446F061B8E700B5006857
:10B2E0000379012B85B012D0022B0CD103AAF621D1
:10B2F000FFF794FA20B1BDF80C300C4A5BBA938288
:10B3000005B05DF804FB002005B05DF804FB836820
:10B31000417C90F9100003AA03F00103CDE900235A
:10B320000223F622F9F7EAF9E4E700BFE05C002027
:10B3300000B500680379012B85B01FD0022B19D10D
:10B34000032303AAF621FFF769FA80B19DF80D30B7
:10B350009DF80CC010499DF80E201B0243EA0C43D7
:10B360001343B1F93420C2F10802D3408B6305B016
:10B370005DF804FB002005B05DF804FB8368417CA8
:10B3800090F9100003AA03F00103CDE90023032381
:10B39000F622F9F7B3F9D8E7E05C002010B50068B1
:10B3A0000379012B84B02ED0022B23D1062302AACD
:10B3B000F721FFF733FAE8B19DF809209DF808401E
:10B3C0009DF80A109DF80C309DF80BC0120142EA5E
:10B3D000043242EA11121B019DF80D10114C43EA90
:10B3E0000C3343EA11131049E265C1E95623E363C4
:10B3F00004B010BD0C4A0B4BD2E956120020D9659F
:10B40000DA6304B010BD8368417C90F9100002AA91
:10B4100003F00103CDE900230623F722F9F76EF9C3
:10B42000C9E700BFE05C0020D86D002000B50068CF
:10B430000379012B85B01DD0022B0AD1836813F04C
:10B44000010F03AA4FF0030314BF00218021FFF76F
:10B45000E5F99DF80D309DF80C009DF80E100C4A92
:10B460001B0243EA00430B430120C2F8803005B0C1
:10B470005DF804FB8368417C90F9100003AA03F097
:10B480000103CDE9002303230022F9F737F9E0E7B0
:10B49000E05C002000B500680379012B85B01DD069
:10B4A000022B0AD1836813F0010F03AA4FF00303A4
:10B4B00014BF00218021FFF7B1F99DF80D309DF8F0
:10B4C0000C009DF80E100C4A1B0243EA00430B438C
:10B4D0000120C2F8943005B05DF804FB8368417C1C
:10B4E00090F9100003AA03F00103CDE90023032320
:10B4F0000022F9F703F9E0E7E05C002010B50068EE
:10B500000379012B84B029D0022B24D1836813F056
:10B51000010F4FF0030303AA14BF19468321FFF75D
:10B520007DF9B0B19DF80C309DF90C109DF80D20FF
:10B530009DF80EC01B04002943EA0223B8BF4FF058
:10B540007F410D4AA8BF002143EA0C030B43C2F818
:10B55000D83004B010BD002004B010BD8268417C1A
:10B5600090F9100002F00102032303ACCDE9004280
:10B570001A46F9F7C3F8D4E7E05C002000B500688C
:10B580000379012B85B02BD0022B25D1836813F0D2
:10B59000010F03AA4FF0030314BF00218021FFF71E
:10B5A0003DF9B0B19DF80C309DF90C109DF80D20BF
:10B5B0009DF80EC01B04002943EA0223B8BF4FF0D8
:10B5C0007F410E4AA8BF002143EA0C030B43C2F897
:10B5D000BC3005B05DF804FB002005B05DF804FB4D
:10B5E0008368417C90F9100003AA03F00103CDE9C0
:10B5F000002303230022F9F781F8D2E7E05C002062
:10B6000010B5044600230068E386A3630279012A8B
:10B6100084B022D0022A1DD1836813F0010F02AA40
:10B620004FF0060314BF03218321FFF7F7F878B129
:10B63000BDF90A30BDF80810BDF80C205B4201EBE3
:10B64000410103EB430302EB4202E1862387628759
:10B6500004B010BD184604B010BD8368417C90F959
:10B66000100003F00103019302AB009303220623B1
:10B67000F9F744F8DBE700BF00B500680379012B58
:10B6800085B00DD0022B07D1012303AAFF21FFF7BC
:10B69000C5F805B05DF804FB002005B05DF804FBBB
:10B6A0008268417C90F9100002F00102019203AA25
:10B6B0000092FF22F9F722F805B05DF804FB00BF05
:10B6C00070B50446244894F9103003EB8303154603
:10B6D00050F82300A3689A0782B00ED5019066F057
:10B6E00079FB012301980022294666F023FBA36819
:10B6F0009B0717D5012002B070BD636913B11A68AA
:10B700009B885383154B164A1B6856684FEAC30C37
:10B71000144BA3FB0C3C4FEA9C1C53689B1B9C45A1
:10B72000FBD2DBE70D4B0E491A680E4B4FF4FA7053
:10B7300000FB02F2A3FB0232486892094B681B1A15
:10B740009A42FBD26369002BD4D01A689B8813837A
:10B75000012002B070BD00BF600D00208C340020BD
:10B76000001000E0D34D621010B50379012B82B0B8
:10B770008E460DD0022B08D18368DB0758BF41F0FD
:10B78000800102B0BDE810409AE7002002B010BD71
:10B7900014468268009402F00102417C90F9100086
:10B7A00001927246F8F7AAFF02B010BD70B50568A5
:10B7B0002B79012B84B004460E4615D0022B10D1F4
:10B7C000AB68E122DB074CBF114661212846FBF73D
:10B7D0002DFE30B120683246FF2104B0BDE8704034
:10B7E000C2E7002004B070BDAA68697C95F910001A
:10B7F00002F001020DF10F0501920095E1228DF892
:10B800000F20F8F747FFE4E770B505682B79012BA7
:10B8100084B004460E4616D0022B11D1AB68DB076C
:10B820004FF0C3024CBFE12161212846FBF7FEFD2A
:10B8300030B120683246FF2104B0BDE8704093E784
:10B84000002004B070BDAA6895F91000697C02F070
:10B85000010201920DF10F020092C3228DF80F2018
:10B86000E122F8F717FFE3E770B505682B79012BA4
:10B8700084B004460E461AD0022B15D1AB68DB0704
:10B880004FF0F0024CBFE12161212846FBF7CEFDCD
:10B8900050B12246FF2152F8040BFFF765FF18B1A3
:10B8A0002379337004B070BD002004B070BDAA6865
:10B8B00095F91000697C02F0010201920DF10F026E
:10B8C0000092F0228DF80F20E122F8F7E3FEDFE787
:10B8D000F0B5044683B000680021FEF70DFA206839
:10B8E00015227E21FEF732F8642705F0BFF80546E1
:10B8F0000E4605F0BBF8431B61EB0602B3F57A7FF9
:10B9000072F10003F5D3013FEFD1206811227E21AF
:10B91000FEF71CF8052705F0A9F805460E4605F0C8
:10B92000A5F8431B61EB0602B3F57A7F72F10003C1
:10B93000F5D3013FEFD120680DF107020321FFF796
:10B9400013FF9DF8073003F03C03142B40F09A805E
:10B950000C2240212068FDF7F9FF05F087F8054625
:10B960000E4605F083F8431B61EB0602B3F57A7FC0
:10B9700072F10003F5D3454DA16B454AB5FBF1F1DA
:10B98000092389B294F83500FDF71AF94388B5FB0D
:10B99000F3F52564027920684221FDF7D7FF05F011
:10B9A00065F805460E4605F061F8431B61EB06029B
:10B9B000B3F57A7F72F10003F5D3082241212068A4
:10B9C000FDF7C4FF05F052F805460E4605F04EF8A7
:10B9D000431B61EB0602B3F57A7F72F10003F5D3E6
:10B9E000002243212068FDF7B1FF05F03FF805462E
:10B9F0000E4605F03BF8431B61EB0602B3F57A7F78
:10BA000072F10003F5D3102251212068FDF79EFF4B
:10BA100005F02CF805460E4605F028F8431B61EBAF
:10BA20000602B3F57A7F72F10003F5D30A2253219F
:10BA30002068FDF78BFF05F019F805460E4605F066
:10BA400015F8431B61EB0602B3F57A7F72F1000330
:10BA5000F5D3802256212068FDF778FF05F006F81F
:10BA600005460E4605F002F8431B61EB0602B3F5EE
:10BA70007A7F72F10003F5D320680321FEF73CF9C9
:10BA800003B0F0BD062005F04DF800BF40420F00A6
:10BA90009CB007082DE9F043A44A0468816BA44ECA
:10BAA000B6FBF1F183B005460F2389B290F835005B
:10BAB000FDF786F800214388B6FBF3F607462E64AF
:10BAC0002046FEF719F9002276212046FDF73EFFB9
:10BAD0000F224E212046FDF739FF4FF00F0904F0E9
:10BAE000C5FF0646884604F0C1FF831B61EB0801D1
:10BAF000B3F57A7F71F10003F5D3B9F10109EED105
:10BB00007A794F2102F00F022046FDF71FFF4FF018
:10BB10000F0904F0ABFF0646884604F0A7FF831B1D
:10BB200061EB0801B3F57A7F71F10003F5D3B9F148
:10BB30000109EED17A79502102F00F022046FDF77B
:10BB400005FF4FF00F0804F091FF06460F4604F082
:10BB50008DFF831B61EB0701B3F57A7F71F1000361
:10BB6000F5D3B8F10108EED1FF2252212046FDF7AE
:10BB7000EDFE4FF00F0804F079FF06460F4604F083
:10BB800075FF831B61EB0701B3F57A7F71F1000349
:10BB9000F5D3B8F10108EED195F83510072941D059
:10BBA000644E96F8780EFDF763F80546012276217B
:10BBB0002046FDF7CBFEAA780C212046FDF7C6FEF5
:10BBC0002A790D212046FDF7C1FEAA79AB88120122
:10BBD00042EA1322D2B20E212046FDF7B7FE4FF4FF
:10BBE000807196F8780EFDF743F80546022276211B
:10BBF0002046FDF7ABFEAA785200032102F0FE02B8
:10BC00002046FDF7A3FE2A7904212046FDF79EFE7B
:10BC1000AA79AB88120142EA1322D2B2052120464A
:10BC2000FDF794FE002276212046FDF78FFE0322C9
:10BC300014212046FDF78AFE0F2704F017FF054662
:10BC40000E4604F013FF431B61EB0602B3F57A7F47
:10BC500072F10003F5D3013FEFD13A46632120464C
:10BC6000FDF774FE642704F001FF05460E4604F05C
:10BC7000FDFE431B61EB0602B3F57A7F72F1000310
:10BC8000F5D3013FEFD1082265212046FDF75EFE86
:10BC90000DF1070264212046FFF766FD9DF807209D
:10BCA00022F0100242F06002642120468DF8072045
:10BCB000FDF74CFE0F2704F0D9FE05460E4604F0B2
:10BCC000D5FE431B61EB0602B3F57A7F72F10003E8
:10BCD000F5D3013FEFD10DF106024D212046FFF7CC
:10BCE00043FD9DF8062002F03F0242F040024D2144
:10BCF00020468DF80620FDF729FE0F2704F0B6FE3A
:10BD000005460E4604F0B2FE431B61EB0602B3F596
:10BD10007A7F72F10003F5D3013FEFD10321204672
:10BD2000FDF7EAFF03B0BDE8F08300BFD4B0070819
:10BD300040420F00E05C0020F0B583B015460DF1E5
:10BD400007021C4606460F46FFF70EFD9DF807202A
:10BD500005EA0203A34201D103B0F0BD22EA0502C5
:10BD600022433946304603B0BDE8F040FDF7EEBD52
:10BD7000F0B5044683B00D461746061D20680379CA
:10BD8000012B18D0022B13D18368DB0732464FF00A
:10BD9000FF015CBF3246FF21FFF792FC30B115B1C5
:10BDA0002379DB07EAD40FB123793B7003B0F0BDF0
:10BDB000002003B0F0BD8268417C90F9100002F0D1
:10BDC0000102CDE90062FF22F8F798FCE6E700BF28
:10BDD00030B5044683B0051D20680379012B14D0CB
:10BDE000022B0FD18368DB072A464FF0FF015CBFAF
:10BDF0002A46FF21FFF764FC10B12379DB07EBD45F
:10BE000003B030BD002003B030BD8268417C90F9A2
:10BE1000100002F00102CDE90052FF22F8F76EFC9B
:10BE2000EAE700BF30B50246044652F8040B037936
:10BE3000012B83B00ED0022B09D1FF21FFF740FC6C
:10BE400018B12079C04300F0010003B030BD0020DC
:10BE500003B030BD8568417C90F91000009205F078
:10BE600001050195FF22F8F749FCE9E730B5B42256
:10BE700083B00446FF210068FDF768FD10B900207B
:10BE800003B030BD20680379012B04F1040514D000
:10BE9000022BF4D18368DB072A464FF0FF015CBF19
:10BEA0002A46FF21FFF70CFC0028E8D02379DB07A6
:10BEB000E6D520680379012BEAD18268417C90F9AC
:10BEC000100002F00102CDE90052FF22F8F716FC43
:10BED000EAE700BF30B50A4683B00446A5210068F2
:10BEE000FDF734FD10B9002003B030BD20680379A0
:10BEF000012B04F1040514D0022BF4D18368DB0775
:10BF00002A464FF0FF015CBF2A46FF21FFF7D8FB0E
:10BF10000028E8D02379DB07E6D520680379012BD8
:10BF2000EAD18268417C90F9100002F00102CDE96B
:10BF30000052FF22F8F7E2FBEAE700BF70B582B0DB
:10BF4000CDE900230446FFF791FF10B9002002B0AD
:10BF500070BD20685522A521FDF7F8FC0028F5D01A
:10BF6000251D20682A46FF21FFF7FEFB0028EDD0A3
:10BF70002379DB07F5D40DF1FF350DF1070615F830
:10BF8000011F2046FFF7A6FF0028DFD0B542F6D1FB
:10BF9000DDE700BF002A37D0F0B5013A83B0044690
:10BFA0004E1E51FA82F7051D16F8012F2068A521B3
:10BFB000FDF7CCFC90B9002003B0F0BD8268417C55
:10BFC00090F9100002F00102CDE90052FF22F8F7CB
:10BFD00095FB0028EFD02379DB0710D52068037983
:10BFE000012BEBD0022BE6D18368DB072A464FF00A
:10BFF000FF015CBF2A46FF21FFF762FBE9E7B7427A
:10C00000D2D1012003B0F0BD0120704770B5962257
:10C0100082B004460E460068FF21FDF797FC10B978
:10C02000002002B070BD251D20680379012B1FD0B0
:10C03000022BF5D18368DB072A464FF0FF015CBF76
:10C040002A46FF21FFF73CFB0028E9D02379DB07D4
:10C05000EAD4E12220681146FDF778FC0028DFD001
:10C0600020683246FF2102B0BDE87040FFF77CBB7C
:10C070008268417C90F9100002F00102CDE9005283
:10C08000FF22F8F73BFBDFE7002A46D0F0B5013A84
:10C090004F1C83B004460E4657FA82F7051D2068F0
:10C0A0009622FF21FDF752FC90B9002003B0F0BDAD
:10C0B0008268417C90F9100002F00102CDE9005243
:10C0C000FF22F8F71BFB0028EFD02379DB0710D500
:10C0D00020680379012BEBD0022BE6D18368DB07C4
:10C0E0002A464FF0FF015CBF2A46FF21FFF7E8FA1E
:10C0F000E9E7E12220681146FDF728FC0028D4D0AA
:10C1000020683246FF21FFF72FFB0028CDD00136F3
:10C11000BE42C4D1012003B0F0BD0120704700BF72
:10C1200070B505460B460446164655F8040B82B01A
:10C1300087211A46FDF70AFC20680379012B18D0E5
:10C14000022B13D18368DB072A464FF0FF015CBF47
:10C150002A46FF21FFF7B4FA30B12379DA07EBD48E
:10C1600016B1C3F34013337002B070BD002002B0AB
:10C1700070BD8268417C90F9100002F00102CDE9A7
:10C180000052FF22F8F7BAFAE6E700BF70B578214F
:10C1900082B00446164600680022FDF7D7FB10B9AE
:10C1A000002002B070BD251D20680379012B14D03A
:10C1B000022BF5D18368DB072A464FF0FF015CBFF5
:10C1C0002A46FF21FFF77CFA0028E9D02379DA0715
:10C1D000EAD45B09337002B070BD8268417C90F98B
:10C1E000100002F00102CDE90052FF22F8F786FAB2
:10C1F000EAE700BF30B5CC2283B00446A521006831
:10C20000FDF7A4FB10B9002003B030BD206803790E
:10C21000012B04F1040514D0022BF4D18368DB0751
:10C220002A464FF0FF015CBF2A46FF21FFF748FA7C
:10C230000028E8D02379DB07E6D520680379012BB5
:10C24000EAD18268417C90F9100002F00102CDE948
:10C250000052FF22F8F752FAEAE700BF30B5B422E5
:10C2600083B00446FF210068FDF770FB10B9002081
:10C2700003B030BD251D20680379012B22D0022B8D
:10C28000F5D18368DB072A464FF0FF015CBF2A46E1
:10C29000FF21FFF715FA0028E9D02379DA07EAD45D
:10C2A000CC212046FFF716FE0028E0D002E02379DB
:10C2B000DB07DDD520682A46FF21FFF755FA002865
:10C2C000F5D1D4E78268417C90F9100002F00102B8
:10C2D000CDE90052FF22F8F711FADCE72DE9F04F23
:10C2E00089B00446CDE90623002004F1040B049034
:10C2F000029103905D462046049FFFF7B7FD069B21
:10C30000FE0003EBC70B20B90AE0237913F0010A02
:10C310000CD020682A46FF21FFF726FA0028F4D126
:10C32000079B049A1A7009B0BDE8F08F9B07F7D5F8
:10C33000F0212046FFF7CEFD0028F1D0069B083EF5
:10C34000334401270593D0463E46029B002B4AD03A
:10C35000082E48D806F1FF3943FA09F909F0010916
:10C3600020684FEAC9127821FDF7F0FA0028D7D0EB
:10C3700020680379012B47D0022B43D18368DB0768
:10C380002A464FF0FF015CBF2A46FF21FFF798F9CC
:10C390000028C5D0237913F00102E9D103F0600130
:10C3A00060294FEAD31C51D0029919B1082E01D847
:10C3B000E145B5D1BCF1000F3AD01BF808303B4342
:10C3C0000BF808307F00013617F0FF07F6B2BCD13A
:10C3D00008F101085FFA88F8B8F1080F36D0029B1F
:10C3E0000127002BB4D1049BD3B1039BB34217D9CF
:10C3F000059B13F808301F4214BF4FF001094FF09E
:10C400000009ADE700208BE78268417C90F91000BD
:10C4100002F00102CDE90052FF22F8F76FF9B7E709
:10C42000039BA3EB0609B9FA89F94FEA591997E773
:10C430001BF8081021EA07010BF80810990941EAD6
:10C44000531313F0010F08BFB246BBE7402E06D8C6
:10C45000079B049A1B7893423FF64DAF60E79BF829
:10C4600007C00BF1FF370BF1060B17F8011F08236C
:10C4700082EA010616F0010F4FEA520218BF82F05D
:10C480008C0203F1FF3318BFD2B213F0FF034FEA5F
:10C490005101EDD1BB45E8D19445D9D1049B01337D
:10C4A000DBB20493BAF1000F3FF43AAFCDF80CA021
:10C4B000CEE700BF30B505682B79012B85B0044667
:10C4C00000F09280022B08D1AB68DB0702AA4CBFB8
:10C4D000082188212846FFF7F3F89DF8083013F06B
:10C4E000100302D1184605B030BD2068062302AA09
:10C4F0000021FEF7E9F90028F5D09DF809209DF804
:10C5000008109DF80A309FED3F6A120202EB0142CB
:10C510001344140248BF03F17F4307EE903AF8EE4C
:10C52000E77A9DF80C109DF80B409DF80D20364BD6
:10C53000C7EE866A090201EB04410A44090248BFBA
:10C5400002F17F4207EE902AB3F9742007EE102A19
:10C55000B3F97020F8EEE77A05EE102A87EE864AE6
:10C56000B3F96C20B8EEC77AB8EEC55AD3ED1A7A93
:10C57000A6EE875AF8EEE75A04EE902AE6EE855AC0
:10C58000B3F97220D3ED197A03EE902AF8EEE77A28
:10C59000B3F96E20E6EEA57A06EE102AB3F9622012
:10C5A000F8EEE44AF8EEE33A07EE102AB8EEC66A6F
:10C5B000B3F96020A6EEA36AE4EE247A05EE902A91
:10C5C000B8EEC77A66EE846AF8EEE55A27EE047A8A
:10C5D000B6EE005AA5EE857AE6EE867A83ED1F7AEE
:10C5E000C3ED1E7A05B030BDAA68697C95F91000CC
:10C5F00002F00102019202AA00920822F8F77EF8E6
:10C600006BE700BF00007848E05C002030B50568AB
:10C610002B7987B00022012B04468DF80F2035D0EE
:10C62000022B12D1AB68DB070DF10F024CBF2721A3
:10C63000A7212846FFF744F828B19DF80F3013F0E2
:10C64000080305D1184607B030BD104607B030BD0D
:10C650002068062304AA2821FEF736F920B3BDF985
:10C660001030BDF91220002BB8BF03339B10E386B6
:10C67000BDF91430002AB8BF0332002BB8BF033312
:10C6800092109B102287638707B030BDAA68697C2F
:10C6900095F9100002F0010201920DF10F020092D3
:10C6A0002722F8F72BF8C7E7E086A06307B030BD74
:10C6B00030B5054600240068EC86AC630379012B95
:10C6C00087B02AD0022B0ED18368DB070DF10F0251
:10C6D0004CBF21468021FEF7F3FF28B19DF80F40A3
:10C6E00014F0080402D1204607B030BD28680623A4
:10C6F00004AA0121FEF7E8F80028F5D0BDF81430AF
:10C70000BDF81010BDF812205BBA49BA52BA5B42AC
:10C71000E9862A876B8707B030BD22468468417C52
:10C7200090F9100004F0010401940DF10F0400943D
:10C73000F7F7E4FFD1E700BF30B5044600202568D5
:10C74000E086A0632B79012B87B027D0022B10D174
:10C75000AB68DB070DF10F024CBF0621862128468E
:10C76000FEF7AEFF28B19DF80F3013F0040302D19D
:10C77000184607B030BD2068062304AA0021FEF742
:10C78000A3F80028F5D0BDF81010BDF81220BDF8B0
:10C790001430E1862287638707B030BDAA68697CC0
:10C7A00095F9100002F0010201920DF10F020092C2
:10C7B0000622F7F7A3FFD5E710B50368DA6B82B05E
:10C7C000044612B1904740B123685B6B1BB1214610
:10C7D00001A8984718B9FF23E38202B010BDBDF845
:10C7E0000630013B9BB2F7E7F0B585B0044618462A
:10C7F0000D461646039365F06DFD28442768A07327
:10C80000E673204600240094039B7C693246294647
:10C81000A04705B0F0BD00BF38B504468B68016085
:10C820000D46984700230B4A226123752B6B13B1E9
:10C83000204698472075084B93F860311BB1237D43
:10C8400023F0010323750023E3822046BDE838402E
:10C85000B2E700BF0001FF00D86D002010B5154BF6
:10C86000D3F8644184B024B12379012B10D0022B7A
:10C8700002D0002004B010BDA16811F001010246F1
:10C8800018BF8021204604B0BDE81040FAF7CEBDA5
:10C89000A268617C8DF80F0002F0010294F910008B
:10C8A0000DF10F04CDE900428022F7F7F3FE04B04A
:10C8B00010BD00BFD86D00202DE9F041264ED6F8FE
:10C8C000645184B09DB1B02280212846FDF73EF826
:10C8D000402280212846FDF739F800228021284691
:10C8E000FDF734F8102280212846FDF72FF84FF489
:10C8F00080644FF000080DF10F0795B12B79012BE3
:10C9000015D0022B0DD1AB6813F001034FF00002DC
:10C910004FF04001284602BF1A4640212846FAF748
:10C9200085FD013CA4B29CB1D6F86451E5E7AA6844
:10C9300095F91000697C8DF80F8002F00102013C2E
:10C94000CDE90072A4B24022F7F7A4FE002CEBD18F
:10C9500004B0BDE8F08100BFD86D00200B4B10B5CE
:10C96000D3F864418CB15038C2B280212046FCF724
:10C97000EDFF002280212046FCF7E8FF2046102230
:10C98000BDE810408021FCF7E1BF10BDD86D00204C
:10C99000F0B5204C204F203800EB8000661DD7F802
:10C9A000645185B004440644E5B12B792278012B0B
:10C9B0001DD0022B0AD1AB6813F0010F4FF04001DC
:10C9C000284604BF40212846FAF730FD0134B4421E
:10C9D000EAD155B100224021284605B0BDE8F0401B
:10C9E000FCF7B4BF0134B442F0D105B0F0BD8DF80E
:10C9F0000F20AA6895F91000697C02F001020192EB
:10CA00000DF10F0200924022F7F744FED7F864516F
:10CA1000DCE700BF30B10708D86D00202DE9F041F8
:10CA2000734ED6F8645184B0002D00F09680D42265
:10CA300080212846FCF78AFF802211462846FCF711
:10CA400085FFA82280212846FCF780FF3F22802115
:10CA50002846FCF77BFFD32280212846FCF776FF8F
:10CA6000002280212846FCF771FF402280212846C1
:10CA7000FCF76CFF8D2280212846FCF767FF14220B
:10CA800080212846FCF762FFA12280212846FCF77E
:10CA90005DFFC82280212846FCF758FFDA2280215A
:10CAA0002846FCF753FF122280212846FCF74EFF50
:10CAB000812280212846FCF749FFCF228021284689
:10CAC000FCF744FFD92280212846FCF73FFFF122E2
:10CAD00080212846FCF73AFFDB2280212846FCF71C
:10CAE00035FF402280212846FCF730FFA422802118
:10CAF0002846FCF72BFFA62280212846FCF726FFBC
:10CB0000AF2280212846FCF721FFA622802128465B
:10CB1000FCF71CFFAE2280212846FCF717FF2022DD
:10CB200080212846FCF712FF002280212846FCF7CE
:10CB30000DFFB02280212846FCF708FF402280210B
:10CB40002846FCF703FF002280212846FCF7FEFE62
:10CB5000102280212846FCF7F9FE4FF480644FF044
:10CB600000080DF10F0755B32B79012B2FD0022BA5
:10CB70000DD1AB6813F001034FF000024FF04001FC
:10CB8000284602BF1A4640212846FAF74FFC013CCE
:10CB9000A4B2002CE7D175B1812280212846FCF790
:10CBA000D5FEC82280212846FCF7D0FEAF22802186
:10CBB0002846FCF7CBFE012004B0BDE8F081013C23
:10CBC000A4B2002CE3D1012004B0BDE8F081AA6832
:10CBD00095F91000697C8DF80F8002F00102CDE913
:10CBE00000724022F7F756FDD6F86451CFE700BF38
:10CBF000D86D0020FAF7C2BEFAF7C0BEFAF7BEBE83
:10CC0000FAF7BCBEFAF7BABEFAF7B8BE10B5040917
:10CC1000013C032C18D80E4A32F8141000F00F0310
:10CC200041FA03F212F0010210D0012098400138BD
:10CC300008406DF0E3FE074B074A1B5D184400EB0C
:10CC4000400002EB800010BD002010BD104610BD5A
:10CC5000DCAD0708D8AD07080C2900202DE9F04FFE
:10CC6000542204460021BF4893B06CF017F8BE4A26
:10CC7000611EE01C144611F8013F5D1E052D88BFA2
:10CC80000023884244F8043BF5D102F11003114619
:10CC900051F8040B012800F07D819942F8D111462A
:10CCA00051F8040B022800F053819942F8D1114643
:10CCB00051F8040B032800F077819942F8D152F81B
:10CCC000041B042900F03A819A42F8D10520FAF7B2
:10CCD00045F80620FAF742F8A24DDFF8A892DFF8EF
:10CCE000A8821A2600272C7B002C40D02046FFF774
:10CCF0008DFF95F90DA08346E0B103689B498BF841
:10CD0000076003F13F4303F57E039B0A0522C85CDD
:10CD10008BF8062000238BF8083062F093FA944ACF
:10CD2000BBF804300492DBF80000039303A9F6F784
:10CD30000FFE2C7B0023302201E019F833209442AF
:10CD40002ED00133102BF8D100200AEB4A0A08EB51
:10CD5000CA030122D3F86C1828618C180720C3F885
:10CD60006C482975A8756A7583F8682817440136D8
:10CD7000F6B2202E05F10C05B5D177B17D4CDFF868
:10CD80000CA2DFF80C920025237C7BB90135032D22
:10CD900004F118040AF58C7AF6D113B0BDE8F08FCF
:10CDA000754A02EBC303D3F8F005CEE7607962F071
:10CDB00049FA207962F046FAA068F6F733FD236855
:10CDC000A068CDF814A04C3304936369142202FBCD
:10CDD00003F307930023CDE90E33CDE91033069317
:10CDE0000893E36803934FF480624FF40063CDE946
:10CDF00009234FF400514FF48073CDE90B134FF426
:10CE0000003303A90D9362F0F1F9A2685B4913683E
:10CE100043F001031360D9F8043023F4733323F48F
:10CE2000477323F0030343F44033C9F80430226806
:10CE300063695068012B20F0407020F48070D4BFEB
:10CE40000026012640EA062050609068014041F02B
:10CE500002019160D16A013B21F47001DBB241EA29
:10CE60000353D3623F4B012103F148074FFA85F882
:10CE700002E00C33BB422ED0587D0028F9D093F944
:10CE80000D004045F5D1187C9E7D01F1010C09286B
:10CE90005FFA8CFC30D800EB400E06FA0EF6D2F8A2
:10CEA00010B00196072606FA0EFE019E2BEA0E0E22
:10CEB00046EA0E061661062930D8013901EB8101D8
:10CEC0001F2688408E406146D2F834C02CEA060600
:10CED00030435063CDE7936843F4007393609368E5
:10CEE00043F480739360936843F001039360936805
:10CEF00043F08043936049E7A0F10A0E0EEB4E0E1B
:10CF00004FF0070B06FA0EF60BFA0EFED2F80CB035
:10CF10002BEA0E0E46EA0E06D660CCE70C294DD859
:10CF2000073901EB81011F2688408E406146D2F807
:10CF300030C02CEA0606304310639AE7104B93F892
:10CF4000E42E3021013283F8C01E83F8E42EBDE6C2
:10CF50000B4991F8E40E3524013081F8A84E81F890
:10CF6000E40EA4E6706B0020E45C0020BCAD070872
:10CF700003000100B8150020E8AD0708FDF7FFC069
:10CF8000E05C0020D4B30708600D0020C86B0020CF
:10CF900000230140104991F8E40E3424013081F857
:10CFA0009C4E81F8E40E7AE60B4991F8E40E2024B9
:10CFB000013081F8B44E81F8E40E80E60D3901EBC2
:10CFC00081011F2688408E406146D2F82CC02CEA91
:10CFD00006063043D0624CE7E05C002010B50368E1
:10CFE0001A79022A044603D000232371236010BD5E
:10CFF000987AFFF70BFE0028F6D040F61A6100225F
:10D00000C18002722021FCF725FE002323712360DA
:10D0100010BD00BF70B506461C48336803F13F439E
:10D0200003F57E039B0A82B0C05C0C46154662F095
:10D0300009F9B2880092B2FA82F304F003028DF883
:10D040000420C4F3810230688DF80520C3F11F036A
:10D05000C4F3001264098DF80740C3F3CC0400EB5D
:10D06000840403F007038DF806209B00226A0F2634
:10D070009D4006FA03F322EA03032362226A154362
:10D0800069462562F6F764FC02B070BDBCAD0708C6
:10D090002DE9F04FA84CA94DAC4283B050D21E46AA
:10D0A00002E00C34AC424BD294F805C08C45F8D168
:10D0B00094F804C0844501D00028F2D194F807C048
:10D0C0009445EED12568002D3BD000236B60AB600A
:10D0D000EB602B616B61AB61EB612C6022792A7193
:10D0E000A779AF60217AE960012A33D0022A27D1DB
:10D0F000E07AFFF78BFD94F90980A861A07A85F8A2
:10D100001080FFF783FD6861F8B18D4C08EB880A49
:10D110004FEA880954F82A3004EB8A0AABB19AF82E
:10D12000123003B30E2200238671C27103720921EB
:10D13000FCF790FD6B6923B11A689B88138300E0AC
:10D140000025284603B0BDE8F08F2846FFF746FFCC
:10D150000025F6E7E07AFFF759FD627AA37A6B744F
:10D16000A8612A74EDE79AF8080062F06BF89AF863
:10D1700008104A09012301F01F01023A8B40032ADB
:10D1800008D8DFE802F0A7ADA1026E494A6922EA99
:10D1900003034B6109EB080304EB830308F1010A65
:10D1A0005879FFF733FD5FFA8AFA014620B140F65D
:10D1B0000A3380F808A0C38009EB080304EB83035B
:10D1C0000091D879FFF722FD0099034620B140F67F
:10D1D0000A5280F808A0C28009EB080204EB820220
:10D1E000CDE900139079FFF711FDDDE900138346C7
:10D1F00020B140F60A4280F808A0C28009EB08027C
:10D2000004EB820217F0040A527A6FD039B1084653
:10D210004A2101930092FFF7FDFEDDE900232BB1C7
:10D2200018462A210092FFF7F5FE009ABBF1000F85
:10D2300003D058460A21FFF7EDFE09EB080B04EB7B
:10D240008B0B9BF80470002F6BD109EB08033E4A4F
:10D2500054F82330934200F099803C4A934200F006
:10D26000AB803B4A934200F09C803A4A934200F0E4
:10D270008280394A934273D0384A934200F0A780A3
:10D280001A88BAF1000F02F441510CBF03220022A8
:10D290000A4342F445721A809A8B22F40062120407
:10D2A000120C9A8307221A821A8892B242F0400224
:10D2B0001A806FBBC844686904EB88040123A37417
:10D2C00000283FF434AF2DE71E490A6922EA030320
:10D2D0000B615FE71B494A6A22EA03034B6259E785
:10D2E00018490A6A22EA03030B6253E739B1084678
:10D2F0000A2101930092FFF78DFEDDE90023002B48
:10D3000094D018460A210092FFF784FE009A8DE718
:10D310003846FFF77BFC0028CCD0036882881A834C
:10D32000C8E73846FFF772FC00288ED09BF809202A
:10D330000921FFF76FFE88E7F0D20808A0D408089B
:10D34000600D0020003802400030014000380040ED
:10D35000003C0040003401400050014000540140B6
:10D3600002F56842516A41F480115162516A21F418
:10D370008011516284E702F58232516A41F4005112
:10D380005162516A21F40051516279E702F5843209
:10D39000516A41F480515162516A21F480515162C5
:10D3A0006EE702F5FE32116A41F400411162116A22
:10D3B00021F40041116263E702F50032116A41F481
:10D3C00080411162116A21F48041116258E702F52F
:10D3D0006442516A41F400115162516A21F4001112
:10D3E00051624DE72DE9F043002383B01A46362100
:10D3F0000120FFF74DFEDFF87C900746C9F8680171
:10D4000060B34FF00508962603F030FB04460D4646
:10D4100003F02CFB031B61EB0501B3F57A7F71F17F
:10D420000003F5D3013EEFD10DF107023146384636
:10D43000FEF79AF9044668B9B8F10108E3D199F802
:10D440006C31D9F868010C2B04BF0223C9F8703184
:10D45000FFF7C4FD204603B0BDE8F08399F86C31B6
:10D460000C2B01D00446F5E70123C9F870310446BE
:10D47000F0E700BFD86D0020074B53F8203021B1F2
:10D480004BB11A689B8853837047002BFCD01A68F5
:10D490009B88138370477047CCAD07081D4B70B550
:10D4A000D3F81C4174B193F8203105465BB1626832
:10D4B0005379032B2BD8DFE803F0212427021368CC
:10D4C00040331D6070BDE068666881680A6822F0BC
:10D4D00001020A603168104A767932F816608A894A
:10D4E00092B222EA06028A8123740A8892B242F03A
:10D4F00001020A800377FAF745FBD8E71368343353
:10D50000DFE713683833DCE713683C33D9E70023DF
:10D510001B60FFDEE05C0020F4AC0708254BD3F86D
:10D520001C219AB193F8201181B110B5224C94F8C6
:10D53000901103290BD0022911D0002283F8202159
:10D54000FAF73CFA08B984F8910110BD70475268A7
:10D550005379032B2AD8DFE803F023201D185268E3
:10D560005379032B1FD8DFE803F00D0A0702136875
:10D57000403300221A6010BD13683C33F9E713688A
:10D580003833F6E713683433F3E713684033642223
:10D590001A6010BD13683C33F9E713683833F6E7B7
:10D5A00013683433F3E700231B60FFDE00231B60A6
:10D5B000FFDE00BFE05C0020D86D00202DE9F04FB9
:10D5C000BA4BBB4C93F8949193F8958193F896716C
:10D5D000DFF8ECA283B0002603F5CC7501964FF07E
:10D5E000010EAB78E978C3F1FF039BB2002B40F04A
:10D5F00091800B460F468C460A4688468946012193
:10D600000191100240EA0340172240EA0C0006EBA9
:10D61000020CACEB02030EFA02F12A3301429BB278
:10D6200014BF02210121013A44F82310531CF0D108
:10D63000A04B04351836AB42B6B2D2D19B4A4FF458
:10D640004063A2F898338023A2F89A33019B2BB150
:10D6500082F8949182F8958182F89671934B93F8B1
:10D660009131002B53D09449D1F81C31002B4ED06E
:10D67000EFF31180102282F31288DC685E68A568DF
:10D680002A6822F001022A6035688C4A767932F8DD
:10D690001660AA8992B222EA0602AA812269656806
:10D6A0001F2A40F2E080203A202404FA02F2EA60C5
:10D6B000C2B282F31188DA68D1F81C01926840F690
:10D6C0002B44546011680124214311601C740368C9
:10D6D0001A7DA24204BF02221A7593F82C100CBFC7
:10D6E0004FF400720022012904D1022183F82C108A
:10D6F00042F4806293F84410012900F0B98093F855
:10D700005C10012900F0BD80002A40F0BF8003B00A
:10D71000BDE8F08FB5F800C0C3F1FF03AAFB0CB061
:10D7200001FB03F340091B120A46052800F2B980E9
:10D73000DFE800F0886C53361C03AAFB0C077F0956
:10D74000C7EB0717ACEB8707BFB2C81AC7F13C0796
:10D7500000FB07F7AAFB07075FFA83F808EB5717E8
:10D760008946FFB20121BC4601914AE7AAFB0C029F
:10D770005209C2EB0212ACEB820292B2A1EB030996
:10D7800002FB09F9AAFB09295FFA83F808EB59198A
:10D790008C465FFA89F90F4601214A46019130E72C
:10D7A000AAFB0C025209C2EB0212ACEB82081FFA70
:10D7B00088F8CA1AC8F13C0802FB08F8AAFB082836
:10D7C0005FFA83F909EB58188C465FFA88F80F4620
:10D7D00001211A460191434613E7AAFB0C025209A4
:10D7E000C2EB0212ACEB820292B2CF1A02FB07F735
:10D7F000AAFB07275FFA83F909EB57171A46FFB20E
:10D800000B4688460121BC460191FAE6AAFB0C02B0
:10D810005209C2EB0212ACEB82091FFA89F9CA1A4B
:10D82000C9F13C0902FB09F9AAFB0929DFB207EBA0
:10D8300059195FFA89F99C4688460B4601214A46E8
:10D840000191DEE6A1EB03080CFB08F8DFB2AAFBAE
:10D85000080807EB58185FFA88F89C4601230193E3
:10D8600089464346CDE6202404FA02F2AA601FE767
:10D87000022183F8441093F85C10012942F40062FD
:10D8800004D1022183F85C1042F4805243681B6883
:10D8900000215962998989B20A439A8103B0BDE88F
:10D8A000F08F43464A46BC46ABE600BFD86D002029
:10D8B000A475002070710020E05C0020F4AC070823
:10D8C00089888888F8B500212120F5F77DFA10B302
:10D8D0000446F5F721FA264F0546C7F81C01D0B1DA
:10D8E0002120FFF793F9234EC6F89C0340B140F284
:10D8F0001522C28000220272227A4A21FFF78AFB97
:10D9000096F89031022B2AD0032B20D0FAF756F844
:10D9100010B986F89101F8BD174843F2AC02002116
:10D920006BF0BCF996F89031012B03D1134BFF2219
:10D93000C3F8A82097F82031012286F89121002B06
:10D94000E9D12B7C002BE6D1BDE8F84036E6FAF7AA
:10D9500019F92846F5F7D4FB64230360F8BDFAF7FC
:10D9600011F92846F5F7CCFB00230360F8BD00BF92
:10D97000E05C0020D86D0020A4750020A4A5002044
:10D980002DE9F04FA24FA7B000210A260C4607F55B
:10D9900068754FF0050B01968DE097F8A4375E0689
:10D9A00019D404F1020E43F04003BEF18C0F87F846
:10D9B000A43700F2E18004F1010C98340DEB040A65
:10D9C0000CF198040DEB040C74464FF0040E0AF8A9
:10D9D0008CEC0CF88C3C04F1020CBCF18C0F42F086
:10D9E000020E00F2C98004F198036B4403F88BEC3B
:10D9F00004F1040EBEF18C0F03F88CBC00F2BC8065
:10DA000004F19A060DEB060C4FF0060A0CF88CACEC
:10DA100004EB0A0C4FEA8909BCF18C0F5FFA89F616
:10DA200003F8891C00F2A88004F19C0EEE444FF02C
:10DA300007090EF88C9C04F1080EBEF18C0F03F858
:10DA4000876C00F299800CF198060DEB060C0CF82F
:10DA50008CBC03F8852C04F10A028C2A00F28C801D
:10DA600004F1A0060DEB060E0EF88CAC03F8831C37
:10DA700004F10C018C297FD804F1A20204F1A30364
:10DA80006A446B4402F88C9C0C4603F88C8C410968
:10DA900000F01F0C55F82120012303FA0CF322EAB1
:10DAA000030345F82130019B013B01936CD0411CDD
:10DAB000B1F5F07F68D23C222846FAF78BF80028AF
:10DAC0005DDB07EB4003C0F30722B3F8DC335E07EE
:10DAD000C1B25FFA83F94FEA13283FF55EAF97F8BA
:10DAE000A4C71CF0400F03D10CF0380ECE451BD05C
:10DAF0002CF0780C4CEA030304F1020EDBB2BEF109
:10DB00008C0F87F8A43737D804F1010C98340DEB4B
:10DB100004090CF198040DEB040C74464FF0040E4C
:10DB200009F88CEC0CF88C3CA31C8C2B24D804F149
:10DB300098060DEB060C0CF88B2C221D8C2A0CF889
:10DB40008CBC19D804F19A036B444FF0060E03F80D
:10DB50008CEC0CF8891C04EB0E018C290CD804F118
:10DB60009C0204F19D036A446B44072402F88C4C28
:10DB70000C4603F88C8C8AE76FF0004487E7204658
:10DB800014B927B0BDE8F08FD7F89C57214995F913
:10DB90001030AA6803EB8303920751F8230023D5C2
:10DBA000234603AA002164F0C5F8AB689B0703D5A0
:10DBB000012027B0BDE8F08F174B18491A68184BA1
:10DBC0004FF4FA7000FB02F2A3FB0232486892099C
:10DBD0004B681B1A9A42FBD26B69002BE8D01A687B
:10DBE0009B8813830120CCE76B6913B11A689B886B
:10DBF0005383094B09491A68094B4E68D200A3FBAD
:10DC0000023292094B689B1B9A42FBD2C8E700BFC5
:10DC1000D86D0020600D00208C340020001000E042
:10DC2000D34D6210F0B52A4CD4F89C0783B010B1E4
:10DC300094F8A2370BB103B0F0BD0DF107028421B7
:10DC4000012384F8A237FDF78FFD94F8A427D4F8B8
:10DC50009C0742F004020421FBF778FED4F89C07ED
:10DC60000DF107028421FDF77FFD9DF8073013F0C9
:10DC70000406F3D1174D84F8A43731463C222846D8
:10DC80006BF00CF804F29A77314604F2DA3C012684
:10DC90003CF8023F1A0A22F0200203F0040301F0CC
:10DCA0001F0013434FEA511E06FA00F001F1010173
:10DCB00004D055F82E30184345F82E00BC45E7D166
:10DCC000FFF75EFE0028FBD184F8A20703B0F0BD89
:10DCD000D86D00207871002070B5414DD5F89C4773
:10DCE00082B094B395F8A037012B42D0022B2ED1ED
:10DCF000082294F910303B4885F8A32703EB8303EF
:10DD0000042150F823008DF8052000238DF80430FD
:10DD1000A3688DF806109A078DF8071042D50423E2
:10DD20000DEB0302002164F005F8A3689B0722D5E0
:10DD30002D483C22FF216AF0B1FF95F8A13723B9A5
:10DD4000FFF770FF012385F8A13702B070BD0DF118
:10DD50000302A0212046FDF707FD9DF8033003F0E4
:10DD60000503012B37D0002B2FD1D5F89C47082273
:10DD7000BFE74822BDE71D4B1D491A681D4B486887
:10DD80004FF4FA7606FB02F2A3FB023292094B68CB
:10DD90001B1A9A42FBD26369002BC9D01A689B8870
:10DDA0001383C5E7636913B11A689B8853830F4BCC
:10DDB0000F491A680F4B4E68D200A3FB023292093A
:10DDC0004B689B1B9A42FBD2A9E70B4A126840F2B0
:10DDD000DC539A42B9D9D5F89C47482289E700BF5D
:10DDE000D86D0020600D0020787100208C34002058
:10DDF000001000E0D34D621004280020F0B54A4B1B
:10DE00008BB04FF4005103F5707223F8021F9A4251
:10DE1000FBD1464E464C356804F2A377323502E01A
:10DE200033689D4250D9D4F89C073A468021FDF7CB
:10DE30009BFC0028F4D1102203463E4E01250AE047
:10DE40000EF8242C0132D2B2202A034601F8245CB9
:10DE50000CF1040C12D0981C03F1280703F12901DE
:10DE600022280DEB070E69449C46E9D90132D2B253
:10DE70006FF00043202AB4461846ECD1BCF1220FC3
:10DE80004FD800F128020DEB020003F12802012116
:10DE90006A4400F8241C4C21023302F8231CD4F8F5
:10DEA0009C47254894F91020A16802EB820250F8A3
:10DEB00022008A0722D501AA002163F03BFFA36854
:10DEC0009B0704D50BB0F0BD10220023B5E71B4B18
:10DED0001B491A6848684FF4FA7303FB02F24FF4C7
:10DEE0007A73B2FBF3F24B681B1A9A42FBD2636956
:10DEF000002BE7D01A689B881383E3E7626912B1AD
:10DF0000116892884A830D4A0D4D11686E68C900E8
:10DF10004FF47A72B1FBF2F16A68921B9142FBD224
:10DF2000C9E76FF00043BAE7B2710020042800206F
:10DF3000D86D002001000080600D00208C3400208E
:10DF4000001000E02DE9F041334D95F8A23782B082
:10DF500004460E46002BFDD195F8A327D5F89C0763
:10DF6000194602F0F702012385F8A23785F8A327A6
:10DF7000FBF7ECFCE2B207460921D5F89C07FBF75A
:10DF8000E5FCB4F5807F3FD0D5F89C07DFF88C80A6
:10DF900050220821FBF7DAFCD5F89C070DF10702A7
:10DFA000A021FDF7E1FB48B9D8F8D830B8F8DC205B
:10DFB00059690A4214BF5A831A83EDE79DF8074056
:10DFC00014F02004F0D1E2B20A21D5F89C07FBF747
:10DFD000BDFC3219D5F89C07C0210134FDF7C4FB04
:10DFE000362CF0D157B995F8A327D5F89C0702F045
:10DFF000F702394685F8A327FBF7A8FC002385F82C
:10E00000A23702B0BDE8F081D5F89C0740220A2172
:10E01000FBF79CFCB8E700BFD86D00200C2900205E
:10E020002DE9F04F5F4E96F8A247C3B005460F4664
:10E03000002CFDD196F8A327D6F89C0702F0F70232
:10E040000123214686F8A32786F8A237FBF77EFC3A
:10E05000FF2D4FF009038DF8055088BFAD0801AAC8
:10E0600088BF05F0C008137098BFA04602234FF088
:10E07000000C4FF00A0B0DF1050A4FF00B0914E0EC
:10E08000B4F5827F02F803B00AF8031017F80C30D9
:10E0900017D80CF1010CBCF1360F02F8059000F115
:10E0A000060002F80E30234614D09D1C48EA0C01ED
:10E0B000B5F5827F03F104041846C9B203F1030EDB
:10E0C000DED90CF1010C6FF00044BCF1360F36487C
:10E0D0002346EAD1B0F5827F61D8082111550DF1B0
:10E0E0000501A020C8540233D6F89C472F4894F964
:10E0F000101001EB810150F82100A168890722D599
:10E10000002163F017FEA3689B0731D5284CD6F891
:10E110009C070DF10302A021FDF726FB48B9D4F8B6
:10E12000D830B4F8DC2059690A4214BF5A831A83E4
:10E13000EDE79DF8033013F02003F0D186F8A23705
:10E1400043B0BDE8F08F616911B10D6889886983BA
:10E150001849194F0D681949D7F804C0ED00A1FB03
:10E160000515AD097968A1EB0C018D42FAD2C7E71C
:10E17000104B11491A68114B48684FF4FA7505FBAA
:10E1800002F2A3FB023292094B681B1A9A42FBD29D
:10E190006369002BBAD01A689B881383B6E76FF0C7
:10E1A0000043A1E7D86D002001000080600D002031
:10E1B0000C2900208C340020001000E0D34D6210A8
:10E1C000002ABCBF80185242002B30B53BDB5D18E3
:10E1D0000028B7BF121A841814460020A4F11D0CA1
:10E1E0000029BCBF2B460021BCF1000FC8BFA2EB29
:10E1F0000C04A5F10F02C8BF2418002AC4BF9B1A43
:10E200005D1884421EDBC1F1010C114AAC44C1EB24
:10E210000113CCEB0C1C00EB430301344FEA4C0C14
:10E2200002EB43024FF0200E8D42A8BF002304DB17
:10E2300022F813E01E339C45FAD10130A04202F1CE
:10E240000202F1D130BD5C180D465B422146BFE7AA
:10E25000B47100201B4B1C48196C1C4A10B441F0CF
:10E2600080510124196404625321FF24CA2054629E
:10E27000506251625B6FDB0085B013D400231449F8
:10E2800002930291029A134804320292029A136096
:10E2900003930391039B0393039B186005B05DF800
:10E2A000044B70470A4B002201920193019B01939A
:10E2B000019A084B12689A42E0D105B05DF8044B10
:10E2C000704700BF0038024000000E4200280040A6
:10E2D0005028004076614E69012070470120704748
:10E2E0000120704731B10C4BD3ED007AF8EEE77A9C
:10E2F000C1ED007A72B1084BDFED086A5B68A3F5E7
:10E30000D543333B07EE903AF8EEE77A87EEA67AEC
:10E3100082ED007A704700BF50A600200000C8427E
:10E320000120704701207047704700BF034B03EB8B
:10E33000800083680BB19B681960704750A600206D
:10E34000044B03EB80039B680BB19B68196023F0BF
:10E3500017BF00BF50A60020044B03EBC00040F2E3
:10E36000FF739942A8BF194681807047485E00201C
:10E370000C4A13787BB10C4B93F8481059B193F8C1
:10E38000491059B150680022FA2883F84920A8BFE3
:10E390004FF0FF3070476FF0010070476FF00200E0
:10E3A000704700BF0016002050A600200B4B93F8CA
:10E3B0004A2082B193F84B2052B109498868002263
:10E3C000B0F5967F83F84B20A8BF4FF0FF30704721
:10E3D0006FF0020070476FF00100704750A60020F8
:10E3E00000160020014BDB6C5B68184750A600202C
:10E3F000014BDB6C9B68184750A60020014BDB6C7F
:10E40000DB68184750A600202DE9F041114C04F1BB
:10E41000500884F851101746002502234246FF2178
:10E42000064684F85050FCF7D7F980B14246304692
:10E430000223FF21FCF748FA48B194F8502094F8E1
:10E44000513003EB022328463B80BDE8F0816FF09A
:10E450000C00FAE750A60020014BD868704700BFB7
:10E4600000160020044B93F8503113B1034B186988
:10E4700070476FF00100704750A600200016002082
:10E48000437A5A1C0344D2B242729972037A93427D
:10E4900000D97047002AFCD010B5044604F10A01E7
:10E4A000D0E9003098470023637210BD2A4ED6F899
:10E4B0005451D6F8600108B52FF00EF928462FF018
:10E4C0000BF9D6F8600141798B073ED5002108464B
:10E4D000FEF7D2FF00210120FEF7CEFF1F4CD6F839
:10E4E000600103685B689847D0B92B6828465B6871
:10E4F00098470028F3D0D4F89C202B68B4F8A010DB
:10E50000DB685183284698470146D6F860010268C7
:10E5100013689847D4F89C30B4F8A0201A83DEE73B
:10E52000D6F86001D4F8D8200368B4F8DC10DB68B2
:10E53000518398472B6801461B6828469847D4F8B2
:10E54000D830B4F8DC201A83CFE7036841F0020129
:10E550009B699847BAE700BF50A600200C2900200D
:10E5600070B50568E8690C461646A0B3D0F80130CE
:10E57000CCB1D0F805209FED1B7ADFED1B5ADFED03
:10E580001B6A07EE902AF8EE677AB7EE006A77EE1C
:10E59000C77A77EEA77A87EEA57A77EE467A67EEA6
:10E5A000E67AC4ED007AAEB107EE903A9FED107AAC
:10E5B000DFED106A9FED106AF8EEE77A67EE877A72
:10E5C00087EEA67ADFED0D6A77EE467A77EEA67AC9
:10E5D000C6ED007A70BD09211420FAF719FAE86136
:10E5E000C4E700BF9AC9CC449AC94C460E76D745B9
:10E5F0000000484300E0FF44000048423393884352
:10E6000070B50668F46982B00CB300250423257048
:10E610000DEB03023046FF21FCF756F9A8B19DF837
:10E6200004108B091CD19DF805209DF806509DF81B
:10E63000073002EB012292B203EB0523C4F8052058
:10E640005B1101222270C4F8013002B070BD054692
:10E6500009211420FAF7DCF9F06104462E68D4E7AA
:10E66000034A04210320FAF7E1F8284602B070BDFE
:10E670001051080870B50668F06982B00D4614465E
:10E68000002848D0D0F80530DFED266A9FED267AC5
:10E6900007EE903AF8EE677A77EEE67AF3EE096ADB
:10E6A00067EE877AB2EE047A67EEA67AF4EEC77A5E
:10E6B000F1EE10FA22DCBAEE047AF4EEC77AF1EE4B
:10E6C00010FA1BD4D0F801302DB19FED187A67EE07
:10E6D000877AC5ED007A7CB107EE903A9FED146A17
:10E6E000DFED146AB8EE677ADFED137AE7EE067AAB
:10E6F00077EEA67AC4ED007A02B070BD17EE900AEC
:10E7000063F054FF0D4ACDE9000104210320FAF71C
:10E710008DF802B070BD09211420FAF779F9F06183
:10E72000B0E700BF00000046000080380AD77843F9
:10E730000319C83D33938843000048C23451080888
:10E7400030B52DED028B574C94F8AC31022B85B0CF
:10E7500019D0DFED557A79B19FED547A9FED546A67
:10E76000DFED546A67EEA77A67EE877A87EE867ADE
:10E7700077EE267AC1ED007A0AB14F4B136005B0EF
:10E78000BDEC028B30BD94F850326BBB4B4B1B6819
:10E790009B072DD5B4F9343200EE103AB4F9323279
:10E7A000B8EEC00A07EE103A20EE000AB8EEC77ABB
:10E7B000B4F93632A7EE070A07EE903AF8EEE77A98
:10E7C000A7EEA70AB5EEC00AF1EE10FAC1DBB5EE6E
:10E7D000400AF1EE10FA5BD4F1EEC07AF4EE677AFB
:10E7E000F1EE10FAB7D7B4E7344B1B68980704D49E
:10E7F000D4F84C32D3ED347AADE7314D0DF10E0043
:10E80000CDE9001229F094FEBDF80E30D5F8EC03E6
:10E81000DFED2C5ADFED2C6A9FED2C7A1B1A07EEE8
:10E82000903AF8EEE77AB0EE408A87EEA56ADDE925
:10E830000012A6EE267AFDEEC77AB0EE470A17EE72
:10E84000903A2033402B20D8F9F77EFDDDE9001205
:10E850001F4BD4ED847A6C7CA3F144001D462C3B05
:10E86000002C08BF034695ED007AD3ED056AA8EEAB
:10E87000407A37EEA60A20EE000AA7EE070AB5EEA8
:10E88000C00AF1EE10FAA2DA63E79FED070ADFE7AC
:10E89000CDE9001265F066FBDDE90012F0EE407A8A
:10E8A0009CE700BF50A6002000000000CDCC9C3F9C
:10E8B00000409C4682E6C54733139043A0000010F9
:10E8C00018FF00200000C84235FA8E3CDB0FC93F1C
:10E8D0001803012030B50C4D83B055F8303001914C
:10E8E00083B107EE901A93ED047A93ED030AF8EEE4
:10E8F000E77A0446A7EE870A65F026FA55F8343021
:10E900009B68186003B030BD485E0020F0B54D4EE6
:10E9100096F8483083B03BB196F85152012D044629
:10E920005ED0022D3ED00DB103B0F0BD012280219A
:10E930000068454FFBF70AF801223870FF21206874
:10E94000FBF704F82A46387029462068FAF7FEFFDC
:10E9500096F85222387091212068FAF7F7FF29467D
:10E96000387001222068FAF7F1FF2A463870FF213B
:10E970002068FAF7EBFF2A46387080212068FAF702
:10E98000E5FF29460346012220683B70FAF7DEFFC7
:10E990002E4A38701268C6F85422012386F8513284
:10E9A00003B0F0BD0068284F01AA1321FCF7DCFE7C
:10E9B0009DF8043038705B0725D1D6F85832002B0B
:10E9C000B2D0224AD6F85412126892B2521A934226
:10E9D000AAD24FF0FF3200237A6086F85132A3E7C3
:10E9E00001AA0068184F0021FCF7BEFE9DF8043014
:10E9F0003870DA07E1D4154A02231268C6F85422A7
:10EA000086F8513290E720682B4601AA1E21FBF7B9
:10EA10005BFFBDF8043002460B2120683A700122EA
:10EA20005CBAFAF793FF0A4B3870A4B2A3FB043424
:10EA3000E408012200237C6086F8492086F85132E0
:10EA400072E700BF50A60020001600200428002016
:10EA5000CDCCCCCCF0B541F0010285B000212A4FDD
:10EA60002A4D2B4E0446FAF771FF3B68C6F8543224
:10EA7000287016E0A368DB070DF10F024FF01301B9
:10EA800020465EBF0DF10F0293212046FCF718FED1
:10EA90009DF80F30287013F007030ED1D6F85822D6
:10EAA0004ABB2379012B18D0022BE3D09DF80F30FD
:10EAB000002013F007032870F0D001220B2120461C
:10EAC000FAF744FF00220346114620462B70FAF75E
:10EAD0003DFF2870012005B0F0BDA268617C94F96B
:10EAE000100002F0010201920DF10F0200921322B8
:10EAF000F5F704FECCE73968D6F8540289B2091A52
:10EB00008A42CED21846E6E70428002000160020EC
:10EB100050A6002010B5174C84F85110017984F8E4
:10EB2000522001294FF0000282B084F8502012D008
:10EB300002290CD1032304F15002FF21FBF7F6FD5B
:10EB4000002814BF00206FF00C0002B010BD6FF061
:10EB50000C0002B010BD8268417C90F91000503466
:10EB600002F00102CDE900420323FF22F5F792FDF6
:10EB7000E6E700BF50A6002000680379012B0BD008
:10EB8000022B08D183680F4A13F0010316D000232B
:10EB90005121FBF7CBBD704700B58368094A417C22
:10EBA00090F9100083B003F00103CDE900230023A6
:10EBB0005122F5F76FFD03B05DF804FBD121FBF79F
:10EBC000B5BD00BFACA8002030B5184D95F84A304F
:10EBD00083B00BB903B030BD04460DF105010068E8
:10EBE00061F0C8FD9DF8053073B901212068104A15
:10EBF00085F852104FF406440323FF21A5F8504036
:10EC0000FBF7EAFD03B030BD0DF106029621206846
:10EC1000FFF7FAFB074ABDF806300749A2FB0323BA
:10EC2000DB0801228B6085F84B20DEE750A6002030
:10EC3000A0A60020CDCCCCCC0016002030B50446D8
:10EC400000680379012B85B029D0022B1ED1826880
:10EC500012F0010F18BF512103AA08BFD121FBF701
:10EC6000DDFD98B1BDF80C30194A5BBA9BB2D36098
:10EC7000D368B3F5C87F0EDC1649174AD1F85C3269
:10EC800015683233AB4218D305B030BD104B6FF06E
:10EC90000102DA60F0E74FF0FF33D360ECE78368FE
:10ECA000417C90F9100003F00103019303AB009342
:10ECB00051220223F5F722FDD3E701F51772C1F8BF
:10ECC0005C52206800235121FBF786FD05B030BD62
:10ECD0000016002050A600200428002000B500687F
:10ECE0000379012B85B008D0022B2FD0204B0022B6
:10ECF00083F8502105B05DF804FB8368417C90F9EE
:10ED0000100003F0010303AACDE90023022300222F
:10ED1000F5F7F4FC164B83F850010028EAD0BDF853
:10ED20000C305BBA9BB2B3F5FA6F1AD21149124A92
:10ED3000A1FB0313DB0807EE903AF8EEE77AFDEE4D
:10ED4000E77AC2ED047A05B05DF804FB826812F040
:10ED5000010F18BF002103AA08BF8021FBF75EFD49
:10ED6000D8E7054B4FF0FF321A6105B05DF804FBA0
:10ED700050A60020CDCCCCCC0016002010B50068E9
:10ED80000379012B84B00C461DD0022B18D1826868
:10ED900012F0010F14BF0021802103AAFBF73EFDF2
:10EDA00060B15CB19DF80D309DF90C20DB0903EBDF
:10EDB000830302EB820203EB4203238004B010BD05
:10EDC000002004B010BD8368417C90F9100003F06E
:10EDD0000103019303AB009300220223F5F78EFC9D
:10EDE0000028DED1EAE700BF2DE9F843DFF86480B0
:10EDF00004460F461646002540F6340920462021D9
:10EE00006AF0ABFE0446D0B103461C4613F8010B72
:10EE10002028FAD02046FAF7F7FA4845A8BF484616
:10EE2000B0F5617FB8BF4FF46170A0F56170A8FBC9
:10EE30000030C0084DB178703378013333700DB9AC
:10EE40000125DBE72046BDE8F883387033780133CD
:10EE50003370F4E71F85EB5130B583B005460846A3
:10EE6000019163F037FA0199044602462846F9F702
:10EE700077FF20B92A5DA2F13001092902D80020CC
:10EE800003B030BD22F02002413A192AF8D90134EA
:10EE9000281903B030BD00BF10B4474C00232246F0
:10EEA00092F90410012902F10C022AD00133052B3A
:10EEB000F6D12246002392F90410032902F10C0234
:10EEC00035D00133052BF6D1002394F90420052A0F
:10EED00004F10C0441D00133052BF6D1374B5B68AC
:10EEE000DB0351D40179A1F13403012B1BD901F0CB
:10EEF000EF01A1F12000B0FA80F040095DF8044B69
:10EF000070472F4A03EB430302EB8303D3F86032CD
:10EF10000BB32C4B93F83D2093F83CC003799A42F5
:10EF200001D06345C5D101205DF8044B7047244AE8
:10EF300003EB430302EB8303D3F86032002BC4D00E
:10EF4000214B027993F83D1093F83C309142EAD07E
:10EF50009A42B9D1E7E72246ADE7194A03EB4303EA
:10EF600002EB8303D3F86032002BB7D0174B027942
:10EF700093F83D1093F83C309142D4D09A42D2D0CD
:10EF80000E4B5B68DB03ADD5114C22460023117993
:10EF9000212902F1140207D001330C2BA2D01179E0
:10EFA000212902F11402F7D103EB8303026854F81C
:10EFB00023309A4296D1B6E7B0A80020A0000010F6
:10EFC00050A60020200300206C050020B807002078
:10EFD000040A00200D4B10B503F1F00C4FF0000EA9
:10EFE00002E014339C450FD01A688242F9D1DA68E6
:10EFF0008A4218BFD9600EF1010403F1140318BF4F
:10F000005FFA84FE9C45EFD1704610BD040A0020D3
:10F010002DE9F04F3D4EDFF80091DFF800813C4DC7
:10F0200083B04FF0000B0190B2465F46DAF8004023
:10F030004046002101E055F83100844203D00131FF
:10F040000E29F8D1FF21494491F8A012012944D09A
:10F05000022909D1DAF80C10480705D521F004017E
:10F0600041F00801CAF80C105046FFF715FF48B9E7
:10F07000264B0BEB8B0103EB8101C96801F00C00FF
:10F08000042835D00BF1010BBBF10C0F0AF1140A67
:10F09000CCD1204C3046FFF7FFFEC0B9F3685907CA
:10F0A00003F00C0213D5042A11D07A1CD5B2019AB0
:10F0B00023F0080040F00400BA42014623F00403A4
:10F0C0001ED9F0603068FFF785FF2844C7B21436B8
:10F0D000B442DFD103B0BDE8F08FDAF80C100B07B3
:10F0E000C2D521F0080141F00401CAF80C10BBE7B9
:10F0F0002046FFF76FFF0137FFB20744FFB2C1E7B9
:10F100003068F3601946FFF765FFE0E7040A002066
:10F110004CAD0708F40A002050A600200000014072
:10F1200038B50446BDF810502160084619B119469B
:10F13000F3F766FE20682946F3F7DEFE2368596878
:10F140000B68B3F844206FEA42426FEA524292B22F
:10F15000A3F844201A8892B242F001021A804A7938
:10F16000032A17D8DFE802F0110C0702403300220F
:10F17000A3601A6038BD3C330022A3601A6038BD1A
:10F1800038330022A3601A6038BD34330022A360F4
:10F190001A6038BD0023A3601B60FFDE2DE9F04F2D
:10F1A00085B00646BDF838A09DF83CB089461746A4
:10F1B0009846F3F7B1FD0546002842D0274A92F859
:10F1C000AE42092C38D804EB440302EB4313002170
:10F1D000C3F8B01283F8B412631CDBB282F8AE320B
:10F1E00004EB440402F52C723079039302EB4414CF
:10F1F000FDF70CFD50B3039B80F8069002210372CB
:10F20000C1710390BBF1000F12D11121FAF722FD59
:10F21000039A136892885A832046CDF800A043468B
:10F220003A462946FFF77CFF204605B0BDE8F08F3F
:10F23000327AFDF7EFFEEFE7094A00210420F9F7E3
:10F24000F5FA0024204605B0BDE8F08FBBF1000FB1
:10F25000E2D11121FAF7FEFCDEE700BF50A6002044
:10F26000585108082DE9F0473E4D95F8703682B0A8
:10F270003BB93D4A0221042002B0BDE8F047F9F74E
:10F28000D5BA95F8717695F872360137FF1A102FB6
:10F290000DDD10230221009385F87316334A3B4697
:10F2A00000210420F9F7C2FA02B0BDE8F08795F812
:10F2B0007C36012B064611D0022B0BD160F076FF75
:10F2C0002B4BC5F8803695F87C1611F0FD040BD059
:10F2D000284ACFE7284BC5F88036F4E760F066FF90
:10F2E000264BC5F88036EEE77368BB422FDB002F54
:10F2F000DADDDFF89880DFF898A0DFF884902C360C
:10F3000004E00134BC4248F8040BCDD0DAF80430F4
:10F31000B5F874160091C3F300720192B5F8763611
:10F32000174AB9FBF3F356F8040F9BB20321FFF71A
:10F3300035FF0028E5D1134A05260146234604205F
:10F3400085F8736602B0BDE8F047F9F76FBA04209C
:10F3500000930D4A85F873063B462146F9F766FA95
:10F36000A2E700BF50A6002094510808B051080839
:10F3700041E300083C5208082DE3000881210308FE
:10F3800040420F0014520808DC51080858A600201B
:10F39000A000001030B503682C4C2DED028BA34269
:10F3A00083B0F0EE408AB0EE608A13D004F580643A
:10F3B000A3420FD004F57054A3420BD004F580642F
:10F3C000A34207D004F58064A34203D0204B1C68FD
:10F3D000640801E01E4B1C680192B4FBF1F202F5D7
:10F3E0007F420023FF32120C0093B4FBF2F4B4FB13
:10F3F000F1F52246ABB20221FFF7D0FEC0B1B5EE67
:10F40000408AF1EE10FA17D007EE904AF8EE677ACC
:10F4100027EE888A9FED0F7AC8EE076A01230371F1
:10F4200027EE667AC0ED046AA8EEA77A80ED037A2B
:10F4300003B0BDEC028B30BD07EE905AB8EE678A80
:10F4400007EE904AF8EE677AE4E700BF000001405B
:10F45000F40A002000007A442DE9F04F2DED028BD4
:10F46000A74B93F80080B8F10C0F9BB000F30D810F
:10F47000A44BA54D9B792B70032B20D91A1F022A70
:10F4800000F2FC80052B00F02D81062B0CBF4FF401
:10F490007A544FF47A649D4A9D49DFF8C8C20392BA
:10F4A00016469C4AC6F884260027002200264A6099
:10F4B000CCE90067984AB2FBF4F20A6005E0934A8F
:10F4C00003921146954AC1F88426954A12F81330E2
:10F4D000002B00F00A8103684345C0F26981B8F14E
:10F4E000000F00F09F80DFF88092DFF880A29FED90
:10F4F0008D8A00F1040B0027D9F804202B785BF8E3
:10F50000046FC2F30072062B00F2DA80DFE803F02A
:10F51000A99C8F7604040400052B00F0CF8082495B
:10F520008248062B08BF01460024019200940A4637
:10F53000142302213046FFF731FE0290002800F02C
:10F54000BA807B4B31681A787A4E22B9AAE001342E
:10F55000944200F0A7802301F3589942F7D1E2B218
:10F56000130104930298744C016806914FF4907350
:10F5700003FB02420B68D1F804C05C6E049BC265B9
:10F58000F318DCF80000079205949A60002C00F054
:10F59000EF80B0F84430694A6FEA43436FEA53435F
:10F5A0009BB2A0F8443003889BB243F080030380F1
:10F5B0009CF8063013F0040F9CF80530D15C028CE7
:10F5C00014BF042301238B409BB292B222EA0302B0
:10F5D0000284028C92B21343038403889BB243F0EB
:10F5E00001030380059B002B00F0F980029A0123A0
:10F5F0001371029B4AF83730FB000BE0414BDFED03
:10F60000500A9988B0EE600A3046FFF7C3FE4AF808
:10F610003700FB005AF80330002B54D00137B845AF
:10F620007FF46AAF1BB0BDEC028BBDE8F08FDFED5D
:10F63000450A9FED450A30464FF4FA61FFF7AAFEEE
:10F64000FB004AF83700E5E7DFED400A3046B0EE50
:10F65000600A4FF47A71FFF79DFEFB004AF837000D
:10F66000D8E79FED300AF0EE480A30464FF4C871F3
:10F67000FFF790FEFB004AF83700CBE7234A0392DE
:10F680001146334AC1F884261FE72049314A0C232A
:10F690000120009381F87306434600210420F9F706
:10F6A000C5F8BFE713010493F1502149531C072A01
:10F6B0000B707FF657AF002302939AE7264933E792
:10F6C00000234AF83730039C244A052084F8730647
:10F6D0003B46002104201BB0BDEC028BBDE8F04F7F
:10F6E000F9F7A4B84FF4FA54D5E61D4A02210420D4
:10F6F0001BB0BDEC028BBDE8F04FF9F797B800BF27
:10F700009800001010600020015E002050A600202C
:10F71000085E002059E3000840420F00D5E80008C9
:10F720000CAE07086F12833AC0C62D00001BB7004D
:10F73000A85E0020AC5E0020D8AC0020E8AD070831
:10F7400000000000ACC5A737ACC5A7366F1203395F
:10F7500029E3000878520808808D5B0000530808F0
:10F76000A4520808105E0020A0000010485E00208F
:10F77000DCF81030484C059A190B1B0ACDE908C07B
:10F7800008469C46530104EB421EE35880EA1331BD
:10F790008CEA132301F0030103F00F030B4302F182
:10F7A000010211D0102AEDD1069A0023D36020E780
:10F7B00003980093032180F87316384A43460021CA
:10F7C0000420F9F733F82DE7069BC3F80CE09EF808
:10F7D0001C30DDE908C0002B3FF4DBAE09E7069BD7
:10F7E000069CD8682E4B42682E499A422E4A136BCB
:10F7F0000CBF43F4001343F4800313630723838394
:10F8000003222346F3F7E6FDE3689868F4F70AF865
:10F81000E368626898680799036823F0010303604E
:10F820001368127C0D914C330C93204B53F822300B
:10F830000B930023CDE91633CDE9183310931493BD
:10F8400012230F934FF4806311934FF4804C4FF4C5
:10F850008053CDE9123C40230E930BA94FF40033A3
:10F8600015935FF0C3FC2246E4680499A36810680E
:10F870000692314456681A6842F010021A604466D3
:10F8800074790B4A32F81420A0F868208A81069A0D
:10F890004B6001231374A9E6F80A0020C45208083B
:10F8A00000600240A102000800380240ECAD0708E9
:10F8B000F4AC070810B5104CD4E90423A16882B059
:10F8C00002FB03F38B428DF8070012D06368E068F7
:10F8D0000DF10701184467F043F863682269A168D5
:10F8E00013446269B3FBF1F0013201FB1033636032
:10F8F000626102B010BD00BF205E002010B5142070
:10F90000FDF784F990B1044601214FF40873C380D8
:10F910000172FAF79FF92168114BA08848830022F1
:10F9200083F88C2FC3F8884F83F88D2F2520FDF79F
:10F930006DF9044690B14FF408720223C28003723D
:10F940000121FAF787F92168054BA0884883002236
:10F9500083F8942FC3F8904F83F8952F10BD00BF04
:10F9600050A6002010B50379012B84B00C4621D09D
:10F97000022B1DD18368DB070DF10F024CBF012163
:10F980008121FBF79DFE9DF80F30114A1070C3F3E3
:10F99000C002C3F3001CC3F38001A270C3F3801242
:10F9A000DB0984F800C06170E270237104B010BDFF
:10F9B0000020E8E782680DF10F0102F00102CDE9B5
:10F9C00000121A46417C90F91000F4F797FEDAE72E
:10F9D000001600202DE9F04383B014460F4601AA1B
:10F9E00050210546FBF7C0FE9DF804303C4EDFF881
:10F9F000F490307001335B00DBB201AA2380462112
:10FA00002846FBF7B1FE2378DFF8DC80307009FB75
:10FA100003F303F5FA73A8FB03239DF80420990967
:10FA20000132DB0902FB0133A280A8FB03239B09FF
:10FA300001AAE360512102232846FAF745FF237803
:10FA4000BDF80410307009FB03F349BA03F5FA73EB
:10FA5000A8FB0323CAB2C1F307218A40013292B244
:10FA60009909DB0902FB0133E280A8FB03239B0910
:10FA7000238201AA70212846FBF776FE9DF8043008
:10FA8000307001335B00DBB201AA63807121022375
:10FA90002846FAF719FFBDF80420F978307052BAF9
:10FAA000D3B2C2F30722934001339AB2228119B133
:10FAB000E388D31A9AB22281A1780A4B0A4803FB41
:10FAC00001F101F5FA71A0FB01139909DB0902FBB1
:10FAD0000133A0FB03239B09638203B0BDE8F083DD
:10FAE00000160020002F3A00D34D62102DE9F0439C
:10FAF000A84FA94CDFF8A4828FB006464FF000094A
:10FB00004FF4FA7309AA89210068C7F8583287F8B8
:10FB10004890FBF729FE9DF82420207042F0010256
:10FB200089213068F9F712FF4A4620708821306831
:10FB3000F9F70CFF0122207080213068F9F706FFE9
:10FB400001222070FF213068F9F700FF4A4620703B
:10FB500049463068F9F7FAFE09AA20709121306809
:10FB6000FBF702FE9DF824302070012249463068E0
:10FB700087F85232F9F7EAFE4A462070FF213068D2
:10FB8000F9F7E4FE4A46207080213068F9F7DEFE7E
:10FB900009AA207060213068FBF7E6FD9DF824205B
:10FBA000207042F0120260213068F9F7CFFE202564
:10FBB0000223207009AA442130688DF825508DF861
:10FBC0002490FAF709FEFF22207001213068F9F72E
:10FBD000BDFE35682070012280212846F9F7B6FE67
:10FBE00001222070FF212846F9F7B0FE4A46207016
:10FBF00049462846F9F7AAFE06222070FF2128462A
:10FC0000F9F7A4FE09AA207083212846FBF7ACFD72
:10FC10009DF82420207042F0040283212846F9F741
:10FC200095FE07222070FF212846F9F78FFE01225A
:10FC3000207081212846F9F789FE01222070802159
:10FC40002846F9F783FE6B22207094212846F9F7A5
:10FC50007DFE4A46207083212846F9F777FED8F8C2
:10FC600000302070C7F8543214E0AB68DB0709AAF3
:10FC70004FF0830128465EBF09AA83212846FBF77F
:10FC80001FFD9DF82430207083B9D7F85832002B1F
:10FC900040F00F832B79012B00F0FE82022BE4D081
:10FCA0009DF8243000202070002BEED0012283210B
:10FCB0002846F9F74BFE09AA207092212846FBF747
:10FCC00053FD00222070812128469DF82490F9F7E9
:10FCD0003DFE06222070FF212846F9F737FE09AACB
:10FCE000207083212846FBF73FFD9DF824202070DB
:10FCF00002F0FB0283212846F9F728FE012220703A
:10FD0000FF212846F9F722FE012220700021284613
:10FD1000F9F71CFE00222070FF212846F9F716FE95
:10FD20000022207080212846F9F710FE062320705B
:10FD300007AAB0213068FAF7C7FD01222070FF2121
:10FD40003068F9F703FE002220704F213068F9F780
:10FD5000FDFD2C2220704E213068F9F7F7FD0022BE
:10FD60002070FF213068F9F7F1FDB4222070B62130
:10FD70003068F9F7EBFD4FEAD918B8F1000F4FF0F2
:10FD80000005207018BF4FF00C0809F07F0EAC463C
:10FD9000012017E050A600200016002004280020B3
:10FDA000F44503F0070317D011F81C2C42FA03F3B3
:10FDB000DB070CF1010105F1010548BF5FFA81FC89
:10FDC000302D12D0EBB20EAA02EBD301984503F00E
:10FDD000070200FA02F2E3D911F81C3C013523EACC
:10FDE0000202302D01F81C2CECD1062307AAB02109
:10FDF0003068FAF7F1FC01222070FF213068F9F732
:10FE0000A5FD0022114620703068F9F79FFD002201
:10FE10002070FF213068F9F799FD00222070092138
:10FE20003068F9F793FD0022207010213068F9F74F
:10FE30008DFD0022207011213068F9F787FD012225
:10FE4000207024213068F9F781FDFF2220702521E0
:10FE50003068F9F77BFD0022207075213068F9F7D2
:10FE600075FD01222070FF213068F9F76FFD2C220B
:10FE700020704E213068F9F769FD0022207048217A
:10FE80003068F9F763FD2946207020223068F9F7C1
:10FE90005DFD00222070FF213068F9F757FD2946EB
:10FEA000207009223068F9F751FD0022207054219A
:10FEB0003068F9F74BFD0422207031213068F9F7E2
:10FEC00045FD0322207032213068F9F73FFD83227F
:10FED000207040213068F9F739FD25222070462135
:10FEE0003068F9F733FD0022207060213068F9F79F
:10FEF0002DFD0022207027213068F9F727FD06220A
:10FF0000207050213068F9F721FD00222070512126
:10FF10003068F9F71BFD9622207052213068F9F7FE
:10FF200015FD0822207056213068F9F70FFD2A468A
:10FF3000207057213068F9F709FD002220706121F7
:10FF40003068F9F703FD0022207062213068F9F76C
:10FF5000FDFC0022207064213068F9F7F7FC0022D4
:10FF6000207065213068F9F7F1FCA022207066212D
:10FF70003068F9F7EBFC01222070FF213068F9F7B7
:10FF8000E5FC3222207022213068F9F7DFFC1422D0
:10FF9000207047213068F9F7D9FCFF2220704921F1
:10FFA0003068F9F7D3FC002220704A213068F9F755
:10FFB000CDFC00222070FF213068F9F7C7FC0A222F
:10FFC00020707A213068F9F7C1FC002220707B2173
:10FFD0003068F9F7BBFC2122207078213068F9F7EE
:10FFE000B5FC01222070FF213068F9F7AFFC342204
:10FFF000207023213068F9F7A9FC002220704221EB
:020000040801F1
:100000003068F9F7A3FCFF22207044213068F9F72B
:100010009DFC2622207045213068F9F797FC0522C7
:10002000207046213068F9F791FC4022114620707B
:100030003068F9F78BFC062220700E213068F9F742
:1000400085FC1A22207020213068F9F77FFC4022BD
:10005000207043213068F9F779FC00222070FF21DD
:100060003068F9F773FC0322207034213068F9F707
:100070006DFC4422207035213068F9F767FC0122BD
:100080002070FF213068F9F761FC042220703121D3
:100090003068F9F75BFC092220704B213068F9F7D2
:1000A00055FC052220704C213068F9F74FFC0422E2
:1000B00020704D213068F9F749FC00222070FF21A3
:1000C0003068F9F743FC0022207044213068F9F7CA
:1000D0003DFC2022207045213068F9F737FC0822CA
:1000E000207047213068F9F731FC28222070482120
:1000F0003068F9F72BFC0022207067213068F9F78F
:1001000025FC0422207070213068F9F71FFC0122C1
:10011000207071213068F9F719FCFE2220707221DD
:100120003068F9F713FC0022207076213068F9F767
:100130000DFC0022207077213068F9F707FC0122BE
:100140002070FF213068F9F701FC012220700D2199
:100150003068F9F7FBFB00222070FF213068F9F7C7
:10016000F5FB0122207080213068F9F7EFFBF822BF
:10017000207001213068F9F7E9FB01222070FF218E
:100180003068F9F7E3FB012220708E213068F9F71F
:10019000DDFB0122207000213068F9F7D7FB002237
:1001A0002070FF213068F9F7D1FB002220708021F8
:1001B0003068F9F7CBFB042220700A213068F9F788
:1001C000C5FB3568207009AA84212846FBF7CCFAC4
:1001D0009DF82420207002F0EF0284212846F9F7D0
:1001E000B5FB012220700B213068F9F7AFFB05A9A0
:1001F000207030680390FFF7B5FB039809AA05A9A2
:10020000FFF7E8FB9DF81430002B65D00C9B03F63C
:1002100084539DF81620002A55D00C9A02F2B2227F
:1002200003EB42039DF8172022B1BDF8342002F5FC
:10023000257213449DF8182022B1BDF8362002F231
:100240002622134401213068C7F8A83FE822F9F7B5
:100250007DFBD7F8A81F207044F61F6399423068D1
:1002600002D960F0C1FA306801221146F9F76EFB3D
:10027000402120703068FEF7EDFB50B1012130685D
:100280000222F9F763FB002120703068FEF7E2FBE1
:1002900028BB0FB0BDE8F083AA68697C95F910000F
:1002A00002F00102019209AA00928322F4F726FAD1
:1002B000E7E4D8F80020D7F8541292B2521A9342C9
:1002C000BFF4E8ACE5E79DF81520002AAAD00C9A07
:1002D00002F525721344A5E740F6363399E7E82284
:1002E00001213068F9F732FB002502234FF0200C82
:1002F00009AA2070442130688DF825C08DF824505B
:10030000FAF76AFAD6F80080207005A94046FFF790
:1003100029FB09AA05A94046FFF75CFB502257219B
:100320004046F9F713FB0822207056214046F9F7A2
:100330000DFB0822207050214046F9F707FBBDF85D
:10034000342020704FF47A7148F20E6301FB0233BF
:100350007C4A934240F2F2807B4AA2FB03231B0CAF
:100360005A1E32F0FF0309D02B465208013322F007
:10037000FF019BB20029F8D11B029BB21343C3F3C8
:100380000722DBB28DF810208DF8113004AA022369
:1003900051214046FAF720FA0C9A20704FF47A71F6
:1003A00048F20E6301FB0233684A934200F2C480B4
:1003B000654AA2FB0332120C013AD2B246214046F2
:1003C000F9F7C4FAD7F8A81F207044F61F639942C2
:1003D00002D9404660F008FA04AA01214046FBF722
:1003E000C3F902222070012140469DF81050F9F710
:1003F000ADFA002120704046FEF72CFB2A46012171
:100400004046F9F7A3FA3568207005A92846FFF79A
:10041000A9FA09AA05A92846FFF7DCFA48221146DD
:100420002846F9F793FA0822207047212846F9F761
:100430008DFA0322207032212846F9F787FA072225
:10044000207030212846F9F781FA01222070FF211F
:100450002846F9F77BFA2022207030212846F9F748
:1004600075FA00222070FF212846F9F76FFA06225C
:10047000207070212846F9F769FABDF83610344A21
:10048000207046F644034FF47A7000FB0133A2FB60
:1004900003239DF817201B0B1AB1BDF82A20134423
:1004A0009BB2002B46D05A1E32F0FF0309D0002326
:1004B0005208013322F0FF019BB20029F8D11B0240
:1004C0009BB21343C3F30722DBB28DF810208DF8E3
:1004D00011307121022304AA2846FAF77DF9D7F8D2
:1004E000A81F207044F61F63994202D9284660F085
:1004F0007BF904AA01212846FBF736F90222207075
:10050000012128469DF81060F9F720FA002120709B
:100510002846FEF79FFA324601212846F9F716FAD7
:10052000642201232070C7F8582287F848300FB0A2
:10053000BDE8F0831A46C8E7FF223FE72B462A466C
:1005400020E700BF1B0C0100950370F41B280D0170
:100550004963A41310B5174C84F85110017952BAAD
:10056000A4F8522001294FF0000282B084F85020F4
:1005700012D002290CD1042304F15002FF21FAF712
:10058000D5F8002814BF00206FF00C0002B010BD99
:100590006FF00C0002B010BD8268417C90F9100031
:1005A000503402F00102CDE900420423FF22F4F7A7
:1005B00071F8E6E750A600202DE9F04FA24FA34DB9
:1005C000066800213C4685B0834685F84A105A37B4
:1005D000C4F12D0905F1500A884615E0022A0FD111
:1005E000B26812F0010F4FF0030352464FF0FF01C3
:1005F000304601BF03235246FF213046FAF796F8F2
:10060000BC421AD014F8011F327985F8521009EB58
:100610000403012A85F8508085F85130DED1B36893
:10062000717C96F9100003F00103CDE900A3FF22CD
:100630000323F4F72FF8BC42E4D14FF40743A5F8A5
:100640005030402385F8523052460323FF21304674
:10065000FAF7C2F800238DF80E300DF10E01304686
:1006600060F088F89DF80E30002BF6D04FF406406D
:10067000A5F850000120764A85F852000323FF2197
:100680003046FAF7A9F84FF40740714AA5F8500030
:1006900000240323FF21304685F85240FAF79CF8E6
:1006A0004FF40060A5F850000920694A85F852000F
:1006B0000323FF213046FAF78FF84FF43063A5F893
:1006C0005030634A85F8524030460323FF21FAF741
:1006D00083F800287FD0DBF800600DF10E025E2168
:1006E0003046FDF791FEBDF80E30B3F5D77F00F030
:1006F000A38079D8512B75D040F29480AD2B00F0B7
:100700009B80D62B40F08A80212408BB0A224B21F3
:100710003046FEF7FFF90F2260213046FEF7FAF966
:100720000D2263213046FEF7F5F9B82269213046E3
:10073000FEF7F0F940F60D7278213046FFF70AFF18
:1007400040F60E627A213046FFF704FF002875D08C
:10075000DBF8000021215FF05DFFDBF800400DF1C8
:100760000E02DE212046FDF74FFEBDF80E309FED54
:10077000397AC3F30903ADF80E3003EB8303DB00D2
:1007800007EE903AF8EEE77A204667EE877A06237E
:10079000FCEEE77A4FF4D84417EE902A110E85F854
:1007A0005210110C52BA85F85310A5F85420FF21AD
:1007B0005246A5F85040FAF70FF84FF4074140238E
:1007C000DBF80000A5F8501085F85230524603239C
:1007D000FF21FAF701F885F84A0005B0BDE8F08F6F
:1007E0001E2BB5D1142490E740F2E132934221D080
:1007F0000AD940F28F42934203D040F29152934281
:10080000A6D14FF4FA7480E740F2D922934211D076
:1008100040F2E122934209D1642476E7602B3FF451
:1008200073AF95E71D2BDBD10F246EE7B3F5E67FA1
:10083000F2D08DE7C82468E7322466E721463046C7
:100840005FF0E8FE84E700BFC0B4070850A60020B0
:10085000A0A600209A99893F03682DE9F041DF693D
:100860001FB13B46BDE8F0411847002A164611DD8E
:1008700004460D460E4400E023689B6820469847D6
:100880000028F9D0236815F8011B1B6820469847FB
:10089000AE42F1D1BDE8F081DEE700BF224B1B681C
:1008A00013F0100F214B03D0B3F8AC2F520717D41D
:1008B00093F8C62F02BB93F8D42FD3F8D03F52B190
:1008C00043B120B11A689B88138370474BB31A68F1
:1008D0009B885383704780F00100002BF1D1F9E72A
:1008E00093F8C62FB2B993F8D42FD3F8D03F002A8B
:1008F000ECD1002BE6D17047D3F8C82F002AE9D0FD
:1009000058B19268B3F8CC1F094BB3FBF1F35B10FD
:1009100013607047D3F8C82F22B1936800221A6081
:1009200070477047704700BF9C00001050A6002021
:1009300040420F00BFF34F8F0549064BCA6802F4CF
:10094000E0621343CB60BFF34F8F00BFFDE700BFF2
:1009500000ED00E00400FA0508B572B600224FF081
:10096000FF31930003F1604303F561430132082A2C
:10097000C3F88010C3F88011F3D1FFF7DBFF00BF8D
:10098000012108B50846F4F719F8FFF7E5FF00BFA5
:1009900000B583B00D49002200920091009B043302
:1009A0000093009B1B68012B02D003B05DF804FB91
:1009B00001920191019B064904330193019B1A6046
:1009C0000B6883F308884B689847FEE7502800407F
:1009D0000000FF1F10B4EFF31183102282F312887E
:1009E000094C0A4822684FF0E021013222608A69EE
:1009F000C0F8D82F0022C0F8DC2F0A69DBB283F3DD
:100A000011885DF8044B70470428002050A6002090
:100A100030B4EFF31182102383F312884FF0E023F8
:100A2000D2B29969186910F4803F0D481EBF0121A8
:100A3000C0F8DC1F99690B4B1D68D0F8DC3F82F3CE
:100A40001188094804684FF47A7202FB04F02B44C1
:100A5000401A0021B0FBF4F030BCE3FB0201704708
:100A600050A60020042800208C340020124B5B6824
:100A7000C3F30803FBB9EFF31183E3B930B40F4AB2
:100A80000F4C4FF0E02C1168DCF8180013688B4213
:100A9000F9D1D4F8D81F8142F5D30A4A15684FF42A
:100AA0007A7404FB05F20021101AB0FBF5F0E3FBA9
:100AB000040130BC7047ABE700ED00E004280020E3
:100AC00050A600208C34002090B170B5461EFFF770
:100AD000CDFF04460D46FFF7C9FF031B61EB05027E
:100AE000B3F57A7F72F10003F5D3013EEFD270BD0A
:100AF000704700BF70B5006801220921F8F726FF92
:100B00006426FFF7B3FF04460D46FFF7AFFF031B54
:100B100061EB0502B3F57A7F72F10003F5D3013E74
:100B2000EFD170BD2DE9804883B0431C0193DFF8FD
:100B30003C810A230093D8F89C10D8F8D830B8F834
:100B4000A000B8F8DC20DDF804B048834FF0320A8A
:100B50001A834FF005094C69204214BF488308836B
:100B600059690A4214BF5A831A830120FFF796FE7F
:100B700056465746FFF77AFF04460D46FFF776FFC5
:100B8000001B61EB0501B0F57A7F71F10003F5D32D
:100B9000013FEFD1D8F89C30B8F8A02059690A423B
:100BA00014BF5A831A83D8F8D830B8F8DC205969B2
:100BB0000A4214BF5A831A830020FFF76FFEFFF723
:100BC00055FF04460D46FFF751FF001B61EB050181
:100BD000B0F57A7F71F10003F5D3013EEFD1B9F1A1
:100BE000000F0BD0B9F1010910D0B8F8A000D8F867
:100BF0009C10B8F8DC20D8F8D830ACE70BF1FF3BFC
:100C0000BBF1000F19D04FF00009EEE74FF4FA7670
:100C1000FFF72CFF04460D46FFF728FF001B61EB92
:100C20000501B0F57A7F71F10003F5D3013EEFD1F4
:100C30004FF0FA0ABBF1000FE5D14FF47A76FFF7D7
:100C400015FF04460D46FFF711FF031B61EB05017D
:100C5000B3F57A7F71F10003F5D3013EEFD1009B2C
:100C6000013B00937FF467AFFFF78AFE0C29002059
:100C700070B110B504798C4209D3447994429646F8
:100C800005D30368DB6813B1BDE81040184710BDF9
:100C9000704700BF18B103681B6A03B118470020F2
:100CA000704700BF10B50C4620B10368DB6A0BB17A
:100CB000984768B9074B0020C4E90000C4E9020066
:100CC000C4E906332D2130222061217584F82020CB
:100CD00010BD00BF54A908080178F9B1F8B5104F4C
:100CE0000546002602E015F8011FB1B1D7F8E04F24
:100CF000637A5A1C2344D2B262729972237A934265
:100D0000F1D8002AEFD004F10A01D4E90030984765
:100D1000667215F8011F0029E8D1F8BD704700BFC1
:100D200050A6002070B504460F48FFF7D5FF2046B7
:100D3000FFF7D2FF0D48FFF7CFFF0D4BB3F8E46F7D
:100D400016B970BD013EFCD0FFF790FE04460D467B
:100D5000FFF78CFE031B61EB0502B3F57A7F72F19E
:100D60000003F5D3EEE700BF2853080884B4080851
:100D700050A6002030B583B00F4C01900F48009171
:100D8000FFF7AAFFDDE900320D49D4F8E00F61F06A
:100D900063F8D4F8E05F6A7A32B12B68686805F1CD
:100DA0000A01984700236B7294F8E63F13B10123C0
:100DB00084F8E73F03B030BD50A600203053080848
:100DC00081E400080FB470B582B006A951F8040B95
:100DD0000191FFF7CFFF0E48FFF77EFF0D4BB3F8F1
:100DE000E46F36B902B0BDE8704004B07047013E10
:100DF000F8D0FFF73BFE04460D46FFF737FE031B16
:100E000061EB0502B3F57A7F72F10003F5D3EEE7EB
:100E100084B4080850A6002000283DD00378002B99
:100E20003AD02DE9F04F87B05A4905AA66F0A6FDE1
:100E30000446002800F0A2804FF0000BDFF88091FC
:100E4000DFF88081DFF880A15D465F464FF0FF3616
:100E50000BE0BBF1000F26D04E4905AA002066F03A
:100E60008DFD0BF1010B044610B3BBF1010F15D042
:100E7000BBF1020FEDD14946204668F0C8FE0028BC
:100E80006ED045F001054146204668F0C0FE0028BE
:100E90005FD045F00205DFE73F4893E72046F8F7CB
:100EA000B3FA0746D8E72046F8F7AEFA0646D3E786
:100EB00070B23A4A002392F90010814225D00133E2
:100EC000052B02F10C02F6D1002F50D0002D08BFE7
:100ED00003250023EDB2CDE9015300971A461946C8
:100EE0002CF062FB044600284ED02D48DFF8DC8051
:100EF0003A463146F7F766FC31462A48F7F762FC76
:100F0000D8F8540121465CF035FBDFF8C08003EBD4
:100F1000430308EB8303D3F8EC4F002CD4D02248D2
:100F20003146F7F74FFC5DB16179A94208D01F48FF
:100F30002A46F7F747FC2368E9B29B6920469847A1
:100F4000E36A002BD8D01A48F7F73CFC0023E36291
:100F5000D2E72046514668F05AFE002899D17BE737
:100F60001449204668F053FE00288AD18BE71248C6
:100F70003146F7F727FC07B0BDE8F08F4FF0FF30A0
:100F800025462746064694E731460C48F7F71AFCF3
:100F9000F1E700BFE4AA08083054080838B600207A
:100FA0009053080800540808B0530808C8530808AC
:100FB000E8530808206C08084853080870530808CC
:100FC0003C530808405308084453080850A6002022
:100FD000002868D02DE9F04F90F800C085B0044695
:100FE000BCF1000F2AD000F100475A4E8646023F5E
:100FF00001466346722207E0984526D1B94212D0D5
:1010000011F8013F16F8012FA3F14105192DA2F1A6
:10101000410098BF2033192802F12008ECD99A42E8
:1010200013D1002AEAD14C4C0023C4F8203E84F8A6
:10103000273EA4F8283E05B0BDE8F08F002101202E
:1010400005B0BDE8F04F5CF0EFBA444E2146634670
:101050006C2207E098452AD1B94212D011F8013F1D
:1010600016F8012FA3F14105192DA2F1410098BFF7
:101070002033192802F12008ECD99A4217D1002A0E
:10108000EAD1374B1B685B07D5D4334C94F9263E25
:10109000002BD0D194F9213E002BC5DC05B0BDE872
:1010A000F04F53F091BA002101205CF0BDBA2D48F9
:1010B000732307E065455BD1774513D01EF801CF58
:1010C00010F8013FACF141011929A3F1410298BF89
:1010D0000CF1200C192A03F12005EBD9634547D107
:1010E000002BE9D11C4B002293F9270E83F8202E08
:1010F0001C46164693F8D2140129A1F1030509D024
:10110000052D07D90EB184F8270E174805B0BDE8A4
:10111000F04F57E693F8D314A52903F1140303D035
:101120000132782AE6D1EDE7012803D0013840B238
:101130000126F5E70D4984F8200E0023013284F8DA
:10114000212E01F8D43C84F8273E05B0BDE8F04FCD
:1011500051F09AB83C54080818FF0020445408087D
:101160009C000010A86308083054080848B7002005
:10117000DFF880A22046F8F747F91AF9D47C07FA7D
:1011800080F5772D064600F2D1802046202168F0B8
:10119000E4FC8046002800F01C810346984613F8C2
:1011A000012B202AFAD04046F8F72EF901245FFAE5
:1011B00080F94046202168F0D0FC8046002800F0ED
:1011C0000D810346984613F8012B202AFAD0404699
:1011D000F8F71AF901340090E4B24046202168F093
:1011E000BCFC8046002800F0F7800346984613F8C0
:1011F000012B202AFAD04046F8F706F90134019075
:10120000E4B24046202168F0A8FC8046002800F0A7
:10121000BF800346984613F8012B202AFAD0404697
:10122000F8F7F2F801340290E4B24046202168F069
:1012300094FC8046002800F0A9800346984613F8E5
:10124000012B202AFAD04046F8F7DEF801340FFAD5
:1012500080FBE4B24046202168F07FFC0246002873
:1012600000F0B58003461A4613F8011B2029FAD076
:1012700010460392F8F7C8F80134039A0FFA80F881
:10128000E4B21046202168F068FC002856D00346DE
:101290001A46013311782029FAD010460392F8F744
:1012A000B3F8039A03461BB210462021039368F05B
:1012B00054FC039B002800F0938002461046013244
:1012C00001782029FAD00393F8F79EF804F0FD0482
:1012D000042C039B08BFC2B27FF417AFB9F1010F12
:1012E00004D9A9F1030105293FF60FAF22B1A52AC0
:1012F0002FD0482A7FF409AF3DB33B4905EB850564
:1013000001EB850181F8D2940098C1F8C0040198DE
:10131000C1F8C4040298C1F8C804A1F8CCB4A1F87B
:10132000CE84A1F8D03481F8D32484E62F49304804
:101330007723002205B0BDE8F04F43E55FFA88F25D
:1013400003468046062CC9D0DFE6274981F8275E90
:10135000D8E7FDB9244C0099C4F8C0140199C4F829
:10136000C4140299A4F8D03484F8D294C4F8C814F0
:10137000A4F8CCB4A4F8CE8484F8D3240123013794
:101380003E440AF8D46C84F8273E54E6834661E76D
:1013900002904AE7144C009805EB850504EB8501A3
:1013A000A1F8D03494F8273EC1F8C0040198C1F8E0
:1013B000C4040133029881F8D294C1F8C804A1F89A
:1013C000CCB4A1F8CE8481F8D3245BB2D7E78046B1
:1013D00057E704468146ECE6019012E70090FCE6F0
:1013E0000134E4B20246ADE718FF00204C5408086F
:1013F0005854080848B700202DE9F04782B03E490C
:1014000001AA66F0BBFA002872D04FF0000A4FF034
:10141000FF34394DD1465646D0462746BAF1040F1F
:1014200009D8DFE80AF0443E380E03000378482B61
:1014300046D0562B41D03148FFF7C4FC02B0BDE87E
:10144000F087F7F7E1FF3F280646F4D8002001AA0D
:10145000294666F093FA0AF1010A0028DED1BAF1B2
:10146000040F3AD02FDDBAF1050FE4D1244AB301BD
:1014700003F47C6308F03F0843EA0803B9F1000F66
:1014800001D043F40053962101FB074402EB4404CE
:1014900024F8D03CD2E7F7F7B7FF3F288046D5D9EC
:1014A000C9E7F7F7B1FF95280446CFD9C3E7F7F7A7
:1014B000ABFF03280746C9D9BDE74FF00109C5E7CF
:1014C0004FF00009C2E7BAF1020FB4DC0D49234620
:1014D0003A4601205CF02EF9B0E7094A962303FB57
:1014E000074302EB430333F8D09CC9F34039BEE70E
:1014F0004FF0FF373C46E9E7E4AA080830540808F3
:1015000048B7002078B6002080B51948194DFFF77C
:10151000E3FB1948FFF7E0FBD5F8E04F627A32B100
:101520002146606851F80A3B984700236372D5F85A
:1015300054713B6838465B699847B0B90A26FFF793
:1015400095FA04460D46FFF791FA031B61EB05027D
:10155000B3F57A7F72F10003F5D3013EEFD13B681A
:1015600038465B6998470028E8D0012007F0C6FD9F
:101570007854080850A600209454080830B42F4C22
:1015800094F8E033012B86B002D006B030BC70472F
:1015900094F8E5330A2B04D0294806B030BCFFF795
:1015A0009BBB41218DF80110264900231520097DA0
:1015B0008DF80200CDE90333EB20CDE90133A622FB
:1015C0008DF803008DF80410B22003218DF805007A
:1015D0008DF814308DF800208DF80610EC460DF1D2
:1015E000120541F2210083EA0223082213F4004F7E
:1015F00080EA43010ABF5B008BB29BB2013AF5D18E
:10160000654502D01CF8012FEDE7C3F307228DF8E2
:1016100014308DF81320EC461523C4F85034BCE880
:101620000F00094D0FC59CE8030045F8040B07485F
:10163000297006B030BCFFF74FBB00BF48B7002091
:10164000A05408080016002048BB0020B054080829
:10165000F8B52F482F4FFFF73FFB2F48FFF73CFB14
:10166000B7F8E46F002E44D1D7F8E04F627A32B178
:101670002146606851F80A3B984700236372274B64
:10168000002583F85454C3F8945483F8985423F0F5
:10169000ADF82348FFF720FBD7F8E04F627A2AB174
:1016A0002146606851F80A3B98476572D7F8547133
:1016B0003B6838465B699847B0B90A26FFF7D6F908
:1016C00004460D46FFF7D2F9031B61EB0502B3F5A3
:1016D0007A7F72F10003F5D3013EEFD13B683846C3
:1016E0005B6998470028E8D0002007F007FD013E1D
:1016F000BAD0FFF7BBF904460D46FFF7B7F9031B55
:1017000061EB0502B3F57A7F72F10003F5D3EEE7E2
:10171000CC54080850A6002084B4080848B700201C
:1017200094540808F8B530490522044668F02AFAAE
:1017300018BB2E4E96F8E63F23B9012286F8E62F15
:1017400086F8E73F2A48FFF7C7FA2A48FFF7C4FAA6
:10175000B6F8E46F16B9F8BD013EFCD0FFF786F984
:1017600004460D46FFF782F9031B61EB0502B3F552
:101770007A7F72F10003F5D3EEE71F49032220467A
:1017800068F000FA50BB194E96F8E63F13B196F890
:10179000E73FFBB91948FFF79FFA1648FFF79CFA95
:1017A000B6F8E47F3FB9002386F8E63F86F8E73FC6
:1017B000F8BD013FF7D0FFF759F904460D46FFF792
:1017C00055F9031B61EB0502B3F57A7F72F1000353
:1017D000F5D3EEE70A48FFF7F5FAE4E7BDE8F8408D
:1017E0000848FFF7EFBA00BFF854080850A60020D9
:1017F0000055080884B40808EC7408085055080817
:101800001855080864550808F8B52C4C94F8E63FBC
:101810001BB194F8E73F002B44D1294D29480126FC
:10182000FFF75AFA85F89F6485F8D464F7F78CFEC1
:10183000254B85F8CA641B682448C5F8AC340026DB
:1018400085F8D46485F89F64FFF746FAD4F8E05F22
:101850006A7A02BBD4F854713B6838465B69984792
:10186000B0B90A24FFF702F905460E46FFF7FEF865
:10187000401B61EB0601B0F57A7F71F10003F5D3EF
:10188000013CEFD13B6838465B6998470028E8D0B7
:10189000002007F033FCD5E9003005F10A01984734
:1018A0006E72D7E70A48FFF78DFA0A48FFF78AFAFF
:1018B000002384F8E63F84F8E73FF8BD50A60020F7
:1018C00048B70020945508080428002094540808BC
:1018D0001855080874550808F8B5284C284F0126F3
:1018E00005462848FFF7F8F906F01AFA84F89F64CD
:1018F00084F8D464F7F728FE234A2449126884F850
:10190000CA6400232846C4F8AC2484F8D43484F88C
:101910009F3487F8E73FFDF79FFA00B1F8BD044612
:101920001B48FFF7D9F9D7F8E05F6A7A2AB1D5E901
:10193000003005F10A0198476C72D7F854713B6882
:1019400038465B699847B0B90A26FFF78FF8044616
:101950000D46FFF78BF8031B61EB0502B3F57A7FA9
:1019600072F10003F5D3013EEFD13B6838465B6965
:1019700098470028E8D0002007F0C0FB48B70020B7
:1019800050A600209C55080804280020B4550808DB
:101990009454080870B50C48FFF79EF90B4BB3F848
:1019A000E46F16B970BD013EFCD0FFF75FF8044646
:1019B0000D46FFF75BF8031B61EB0502B3F57A7F79
:1019C00072F10003F5D3EEE784B4080850A60020B6
:1019D000800601D5002933D10CB470B5194C1A49D1
:1019E000D4F8E00F82B007AB069A019360F034FAA6
:1019F000D4F8E05F6A7A32B12B68686805F10A01B1
:101A0000984700236B721148FFF766F9B4F8E46F4A
:101A10003EB9012002B0BDE8704002B07047013EFF
:101A2000F7D0FFF723F804460D46FFF71FF8031B16
:101A300061EB0502B3F57A7F72F10003F5D3EEE7AF
:101A40000020704750A6002081E4000884B40808F4
:101A5000F0B5044683B070B302785AB300F1004089
:101A6000434D21460238722307E0974237D188421E
:101A700014D011F8012F15F8013FA2F1410EBEF16B
:101A8000190FA3F1410C98BF2032BCF1190F03F1DB
:101A90002007EAD9934222D1002BE8D1354B364AB0
:101AA000C3F8D824C3F8DC24C3F8E024C3F8E42442
:101AB00003B0F0BD1446314D314E35F8241005EB1E
:101AC000840332465888CDE90010012023460021C6
:101AD0000444FFF77DFF042CEFD103B0F0BD204696
:101AE000F7F792FC032805462FD82046202168F0FE
:101AF00034F80446002839D003461C4613F8012B5D
:101B0000202AFAD02046F7F77FFC0127064620213D
:101B1000204668F022F8034688B11846013302785F
:101B2000202AFAD0F7F770FC4FB1A6F2EE2240F26D
:101B3000DC539A4203D8A0F2EE229A420ED9114801
:101B400003B0BDE8F040FFF73DB90F490F4803234C
:101B5000002203B0BDE8F040FFF734B9054B03EBBA
:101B60008505A5F8D864A5F8DA04A1E70746CEE70D
:101B70003C54080848B70020E803D00720BC0020E8
:101B8000C055080830540808D455080858540808A7
:101B90002DE9F04387B040B3037807462BB300F13B
:101BA0000040564E39460238722207E09C4532D139
:101BB000814212D011F8013F16F8012FA3F141051F
:101BC000192DA2F1410498BF2033192C02F1200CE9
:101BD000ECD99A421FD1002AEAD14948602200215B
:101BE00007B0BDE8F04367F059B8454D454F0024B4
:101BF000D5E9010615F80C1B0091CDE9010601207D
:101C000023463A4604440021FFF7E2FE082CEFD1B8
